:020000040800F2
:1000000000500020994D0108394E01088137010840
:10001000394E0108394E0108394E01080000000030
:10002000000000000000000000000000394E010840
:10003000394E010800000000394E0108D3D10008F4
:10004000394E0108394E0108394E0108394E010870
:10005000394E0108394E0108CD9E0008C99E00089E
:10006000394E0108394E0108394E0108394E010850
:10007000394E0108394E01080DBE0008394E0108FD
:1000800085E90008394E0108394E0108394E01084A
:10009000394E0108394E0108394E0108C59E000845
:1000A000394E010861CD0008394E010871CD0008B4
:1000B00051CD000841CD000831CD00082944000889
:1000C0002D4400082144000825440008394E010849
:1000D000394E010805BE0008FDBD0008F5BD000849
:1000E000E1D10008394E0108394E01080000000036
:1000F0000000000000000000000000000000000000
:0C01000000000000000000005FF808F1A3
:100110002DE9F04F754B764EA3B03360002373602A
:1001200011F06AFE18B911F089FE08F06FFF09F0AE
:100130000FF8704A704C1378704D43F00103137040
:1001400000230A930B930C934FF4E0130D93236851
:10015000A87B43F480332360A36943F01003A361B9
:10016000236803F400330B930A9B01330A930B9B20
:100170001BB90A9BB3F5A06FF2D123685E4913F453
:10018000003301D0022315E00A6842F001020A6040
:100190000A93236803F002030B930A9B01330A932B
:1001A0000B9B1BB90A9BB3F5A06FF2D123689B0789
:1001B00039D501230C93524B52491A6842F0100270
:1001C0001A601A6822F003021A601A6842F00202EA
:1001D0001A606368636063686360636843F48063A4
:1001E0006360494B1A68043B22F070425A60474AE8
:1001F0001160616821F47C116160596841F000412F
:100200005960D96821F40041D9609B681F0449BF37
:100210003F4B4FF4E01313604FF480130D930C9B8E
:10022000012B01D117E0FEE7022B18D168B10D9B1D
:10023000B3F5801F02D14FF4A01305E00D9BB3F579
:10024000E01F02D14FF400130D930D9963680B4327
:1002500043F4803302E0636843F46013636023680F
:1002600043F0807323602168234B8901FBD55968D3
:1002700021F003015960596841F002015960636837
:100280001D4903F00C03082BF9D14B68DFF88C8073
:1002900003F00C03042B03D0082B03D0194B12E0FE
:1002A000136810E04B684868C3F38343C70303F146
:1002B000020301D4174905E0496811F4003F1168B1
:1002C00018BF49084B43C8F8003063681249C3F3AC
:1002D00003130B44197ED8F80030CB40C8F8003027
:1002E0001368084A93421BD101221DE0F3870008DE
:1002F00050090020BC33002000100240FC280020E0
:100300000020024000127A00041001403C0000204E
:10031000001BB70000093D00009D010858000020A7
:100320008A4A934202D10222894B1A70DFF878A2DE
:10033000884BDFF878C2CAF80C30A3690DF1880B3E
:1003400043F00103A361636A834FB360636A60464D
:1003500043F080736362A3694FF0000943F01C030C
:10036000A3614FF6FF732BF82C3D5946CDF80CC016
:100370008DF85E900EF011FC384659460EF00DFCDB
:10038000594676480EF009FC754A5846536843F0C2
:100390000073536010F0BEF8724A179B4946B3FBD6
:1003A000F2F3714A714813600C2216F0D0FFD8F8AE
:1003B00000304FF47A72B3FBF2F36D4A013B5360A5
:1003C000F0238AF823300723C2F808901360AB6843
:1003D000DFF8DC91DFF8DC81C9F8003098E80F0025
:1003E0008BE80F00A3694FF0100A43F00803A361E4
:1003F000A369179843F00803A36108233B6118A978
:10040000C7F810A00EF0C9FB19981AA90EF0C5FB89
:10041000D9F80020100713D5564B93F89021012AE4
:100420000ED8554993F89121896811F0805300F056
:10043000F28505E04F4B002283F8912109F04AF83C
:1004400064200CF0BCFEA0224C48002116F07FFF77
:10045000E369002243F00703E361A36943F4006307
:1004600043F00C03A361444B4FF0000803F10C016F
:1004700002F8018001320E2AF5D1FF229A76DA764F
:100480001A775A773E4B3F4A41461A603E483C2213
:10049000D9F8004016F05BFF4146C4F380170523EE
:1004A0003A4ADFF8E4E0885C0C224A4302F80E0086
:1004B00047B91E3801289FBFFF2003F1FF3302F820
:1004C0000E00DBB201310529EAD1314A95F805A0C9
:1004D0001370304B304983F800A0304B264A33620A
:1004E000C0330B602E4BA10603EBCA035B7848BFF9
:1004F00001235362002340F2DC512A4A22F81310F0
:100500000133082BF7D110A800211C2216F01FFF81
:1005100014F4007CDFF8A09004F400684ED0A3042B
:100520000AD4B8F1000F0AD095F8842109F10C0320
:10053000012A08BF4B4604E0CDF8109002E009F113
:100540000C030493CDF858B03AE000BF001BB7008D
:10055000E73300200005FA05000C014000100140BF
:100560000000014040420F0054220020A01800204B
:1005700010E000E0FC280020500900206822002044
:10058000E8180020E22A0020EC180020E9C4010845
:1005900089100020600400208423002010290020FE
:1005A00050C10108F40F002000ED00E000080140F8
:1005B0009C280020289D0108009D0108CDF810C04E
:1005C000BAF10E0F04D00AF0EF0ABAF1080F02D107
:1005D00001238DF852300120CDF814C007F0FAF84D
:1005E000DDF814C018B14088003018BF0120C4F3F2
:1005F00040038DF84630C4F3403300F001008DF81D
:100600004030C4F3C0338DF845008DF848708DF844
:100610004330B8F1000F07D095F8848108F1FF3717
:10062000D7F1000848EB0708C4F300438DF84930C0
:100630001CF1000318BF01238DF84A30736AB5F826
:100640004801003318BF01238DF84B30C4F3005329
:100650008DF84C30B5F84A31ADF85600ADF8503051
:10066000E004B5F8563148BFBA48ADF84E30C4F38F
:10067000804348BFB0F850018DF84730B5F8543189
:1006800048BFADF85600B3F5FA7FADF8543084BFDB
:100690000023ADF8563095F8CC31AF4886F82830B5
:1006A000002386F8293043709DF8523004F0010190
:1006B000002BC4F3C0028DF844808DF841108DF8F2
:1006C00042200CBF0023022301B902B1013309EB20
:1006D0008309D9F838309A1E1A33079300230692FB
:1006E0000593069B33F8024F06934FF6FF739C4227
:1006F00000F08E819DF84520E3B2240AE5B21AB1DC
:100700009A1E012A40F27F819DF8482032B1934918
:100710001A018958924A914200F075819DF849006A
:1007200030B18E491A0189588D4A914200F06B818F
:100730009DF8462052B18949039E01EB03114A6896
:10074000B24203D10A89102A00F05D819DF843204E
:1007500052B18249039E01EB03114A68B24203D1B0
:100760000A89022A00F04F819DF8442052B17B494A
:100770007C4E01EB03114A68B24203D10A89022A76
:1007800000F04181169E7EB1744F326807EB03176B
:100790007968914208D13A89B188914200F0338159
:1007A000F188914200F02F81022C02D19DF8402067
:1007B00003E0012C04D19DF84120002A00F02381A0
:1007C0009DF84B20654C1E015AB19DF8522042B94C
:1007D000A3F10802012A04D8A25963498A4208BF3A
:1007E00004259DF84C20344452B19DF852203AB96A
:1007F00010B10C3B012B01E0043B032B40F2EB80DA
:10080000012D48D1594FDFF854A1FF2387F87030EC
:1008100087F871300AEB06035A7B586803F1080920
:100820001B894FF00008ADF85C3017A9022387F848
:100830007480C7F880408DF85F308DF85E2087F8AF
:100840002C80C7F83080C7F83480C7F83880C7F8E4
:100850006C8087F8728087F873800EF09EF95AF8E2
:10086000060099F80210424609F07DF920464146FB
:100870002A460BF01BFA3E4BC7F88C80C7F8843031
:100880003C4B2046C7F8883007F1840107F1880205
:100890000BF054FAB7E0022D4CD19DF814204FF024
:1008A0001C0C0CFB02FC314B002703EB0C080893DB
:1008B0009DF814304FF0010988F87530274B88F8FF
:1008C00076709A19517B506802F1080A12898DF8E6
:1008D0005E1088F87E7017A988F87490C8F8804078
:1008E000CDF824C0ADF85C208DF85F500EF055F9BE
:1008F0001A4B9AF8021098593A4609F034F92046F2
:1009000039464A460BF0D2F91B49089BDDF824C052
:10091000C8F8841019496344C8F8881003F18401A9
:10092000C8F88C7020460A1D0BF008FA059B4B4452
:10093000059368E0032D4CD19DF847300B4D104EC8
:1009400003B395F82A70204608214FF6FF72002362
:1009500033E000BFFC2800207909002008BF01080F
:1009600000040040000C0140002C01405009002010
:10097000D5950008B5960008A19B0008AB95000826
:10098000E4260020BDF8542095F82A70B2F5FA7FCD
:10099000BDF856300BD986492046B1FBF2F208214A
:1009A00092B209F035F9834B46F827000AE08249F4
:1009B0002046B1FBF2F2012192B209F029F97F4BF6
:1009C00046F82700C36095F82A30013385F82A30AD
:1009D00019E0042D17D1BDF84E20774B784D93FBCD
:1009E000F2F22046BDF85030012192B295F829600C
:1009F00009F00EF995F8293005EB86060133C6F8A3
:100A0000540185F82930069B079A93427FF469AE1A
:100A10006B4D6C4B95F82920002485F874216A4AA7
:100A20001C7016789846A6F11702022A19D82B6A6C
:100A30000021185903EB040913F05EF910B16B6A39
:100A40005BBB25E0614F99E80F00274487E80F0062
:100A500098F8003010340133C02C88F80030E6D10B
:100A6000EDE75B4B13F836E003EBC603D3F804C0A5
:100A700088F800E0BCF1000FE1D07445DFDA534F95
:100A800023011F4463440FCB013487E80F00F4E7D0
:100A9000504F3B68DA0424D41DE04F4B4F4A13F803
:100AA000360003EBC6035C681070002CF0D0002306
:100AB0008342EDDAC3EBC3016218D2F800C0DFF85D
:100AC00044E1013341F80EC001EB0E079188B98073
:100AD0009279BA71ECE706F0EF03082B404B25D171
:100AE00026E098F80030012BF5D93E4C04EB0313B7
:100AF00003F1100810344445EDD054F8100C4FF0B9
:100B00007C5112F065FF4FF07C5144F8100C54F802
:100B1000140C12F05DFF4FF07C5144F8140C54F8A3
:100B20000C0C12F055FF44F80C0CE3E70E2E08D124
:100B30001A78182E42F010021A7008D10CF0D2FD6B
:100B400005E01A78192E22F010021A70F5E70CF061
:100B5000ADFD3B68244C5B035EBF244B01221A7041
:100B6000234B24481A78994642F004021A70224A0C
:100B700011789046022934BF142310238DF85E307B
:100B80004FF002038DF85F30A3694FF4805243F0B9
:100B90000403ADF85C2038BF0026A36128BF0126FE
:100BA00017A90DF0FAFF154B76B3154A2DE000BFDB
:100BB00000127A00D596000840420F00C596000842
:100BC00050090020E0260020600400209C03002043
:100BD00050C101089C2800202CA8010810230020E7
:100BE000CC100020A403002000100240C808002000
:100BF000BC33002000080140E7330020CC33002044
:100C000081CD000811230020714A00201A600CF0E9
:100C1000F5FA704B704E93E80300A3698BE803006C
:100C200043F00803A361179818A90DF0B6FFE36914
:100C3000304643F48043E3612369594643F48043DB
:100C4000236118238DF85E304FF42043ADF85C30FB
:100C500003238DF85F300DF0A0FF04224FF4804392
:100C6000304659468DF85E2003924FF4805AADF815
:100C70005C300DF092FF1023304659468DF85E30FF
:100C8000ADF85CA00DF089FF2369322043F4804366
:100C90002361236923F480432361504B198801F4B5
:100CA000415141F4457141F003011980998B21F4C0
:100CB00000610904090C998307211982198889B2F6
:100CC00041F0400119809F23C6F810A08DF83C30F8
:100CD00000238DF83D308DF83E308DF83F300CF01C
:100CE0006EFA039AC6F814A058460FA911F00CFC2E
:100CF000C6F810A09DF85E309DF85D201B0243EA07
:100D000002439DF85F201343354A934215D03220A9
:100D10000CF055FAC6F814A0F52011F02BFCFF20BA
:100D200011F028FC7028C6F810A006D198F8003001
:100D3000022B02BF2B4B03221A7098F80030032BB2
:100D40000CBF1F20022006F0C8FC98F80030032BCF
:100D500003D001200EF072F907E0022006F03AFD00
:100D60000028F6D04388002BF3D03E684FF0100BDC
:100D700006F40043039306F4006305931A4B002125
:100D800018465A46069398F8008016F0E0FA4FF697
:100D9000FF72069BADF83C2002224FF0000A16EAD3
:100DA00002018DF83E208DF83FA01E4620D022A9DA
:100DB00021F84CBD0D480FF059FD04233370072274
:100DC000012386F801A0B370F2709A4611E000BFCB
:100DD00095CD0008489D0108000C014000380040F6
:100DE00015202000E7330020C8250020000801401E
:100DF0008A46B8F1010F12D9202222A921F84C2DE0
:100E00009F480FF033FD052201233272B3720AF1BD
:100E10000102072386F809A0F3725FFA82FA039BA6
:100E20008BB122A9022221F84C2D95480FF01EFD0E
:100E300001220AEB0201072386F805A03271B27184
:100E4000F3715FFA81FA059B93B1022222A921F87E
:100E50004C2D8C480FF00AFD092201233273B37325
:100E60000AF10102072386F80DA0F3735FFA82FAF4
:100E70006268854842F4404262606269DFF8088235
:100E800042F001026261A26942F40072A2610FF0B5
:100E9000C9FA7E4A002417927D4ABAF1010F1892CE
:100EA00094BF224680221C924FF480721D924FF410
:100EB00080621E92202240461F9217A94FF40052D2
:100EC00020921994CDF868A01B9421940AF09EFDFD
:100ED000D8F800206F4942F00102C8F800204A68A3
:100EE000BAF1010F22F4702294BF0020012022F4F5
:100EF000807242EA00224A608868674A0AF1FF333A
:100F0000024042F4602242F002028A60CA6ADBB206
:100F100022F4700242EA0353CB6201233219917822
:100F2000002963D0305D591C0928C9B2D278DFF896
:100F300064C112D9A0F10A0EDCF80CA00EEB4E0E23
:100F40004FF0070808FA0EF82AEA080802FA0EF22B
:100F500048EA0202CCF80C200FE0DCF8108000EB2D
:100F6000400A4FF0070E0EFA0AFE28EA0E0E02FAA9
:100F70000AF24EEA0202CCF81020062BDFF814E148
:100F800010D8013BDEF8342003EB83034FF01F0C35
:100F90000CFA03FC22EA0C0200FA03F31343CEF826
:100FA000343022E00C2B10D8073BDEF8302003EB66
:100FB00083034FF01F0C0CFA03FC22EA0C0200FA28
:100FC00003F31343CEF830300FE0A3F10D02DEF847
:100FD0002C8002EB82021F23934028EA030C00FAC4
:100FE00002F34CEA0303CEF82C300B460434102CE9
:100FF00094D1284B9A6842F480729A609A6842F0C1
:1010000001029A609A6842F008029A609968214A3F
:101010000C0743D5FAE7013A092A3FF611AAD8F896
:101020002C0004935946C7F814A0CBF8000003988D
:101030000DF0B3FD039B3C201A46082313610CF00E
:10104000BEF8049BC7F810A01F4695F891319F4247
:10105000BFF6F0A9039BDFF82CA04FF00808CAF8F0
:1010600010807820C3F814800CF09EF8039BCAF817
:1010700014807820C3F810800CF096F80137E4E76C
:1010800000080140000C0140080002404C240140CF
:10109000D825002000240140FDF7F1FF936843F0BC
:1010A00004039360BF4B9E6816F00406FAD1BE4C51
:1010B0009A68B4F85C0142F4A0029A60002840F0FB
:1010C0001086B4F95E31002B40F00B86B4F9603124
:1010D000002B40F006863B6898031FD5C8200CF013
:1010E0006EF8AE200DF015FF08B10DF017FF85F872
:1010F0007501C8200CF063F8AC4B0021C5F87831BD
:10110000AB4D0C22284616F022F90223EB7006F0B4
:1011100055FF0CF02DF8A74B0344AB60A64DB4F877
:101120000CE02B68B4F8640194F8631194F86B2117
:10113000B3F95630CDF800E094F80FE0CDF804E0B4
:1011400009F092FF10B903200CF0B4F899F80030C0
:10115000102243F0020389F80030984B4FF00A0840
:101160005A6108221A61DFF854921920D9F80C301C
:1011700008F1FF3883F01003C9F80C30D9F80C30AF
:1011800083F00803C9F80C300CF019F801200CF0BA
:1011900035F819200CF013F800200CF02FF818F097
:1011A000FF08E0D10823C9F810304FF0100A844B33
:1011B000C9F810A01A68984612F0080F09D0814BA0
:1011C000C9F814A01B6898477F4B0122C9F810A0EA
:1011D0001A707E4BDFF81C921B68187B12F0A4FB80
:1011E0007B4912F0F5FB07F0EDFD8246B9F80000EF
:1011F00012F09AFB514612F0EBFB16F0B5FA754B64
:101200001880B9F8000012F08FFB0146724812F006
:1012100093FC724912F090FC714B6D491860714B50
:10122000186912F0D5FB704912F0D2FB6F4BFF2109
:1012300018606F4B1A22184616F089F8DFF8B8E1EB
:10124000002273460270D8F80020012112F0020F2C
:101250008EF800101FBF417003218EF8001002218C
:1012600018BF8170510741BF9EF8001001F1010EB7
:1012700083F800E04FF0030E48BF00F801E012F0E1
:101280000A0F0ED01A7804218154511CC9B24FF0B4
:10129000050E00F801E0D11C02321970D2B206210D
:1012A000815439688F0641BF1A78571C1F70072771
:1012B00048BF87540A0608D51A7809278754971C0F
:1012C00001321F70D2B20A2787546779082F01D0E4
:1012D0000E2F08D11A7802F1010E83F800E04FF0CA
:1012E0000B0E00F802E01A7811F4803F4FF00C0C5E
:1012F00000F802C002F1010E1CBFDFF8FCC0023290
:101300005FFA8EFE83F800E01FBF8CF80020384A99
:101310004FF00E0C02F80EC04A0748BF1A784FF083
:10132000120C41BF02F1010E83F800E04FF0100EE5
:1013300000F802E01A7811F4806F02F1010E5FFAF2
:101340008EFE83F800E000F802C00ED094F810C2C0
:10135000BCF1000F09D0DFF8A0C002328CF80020E9
:10136000234A4FF0130C02F80EC01A7811F4007FD4
:101370004FF0140C00F802C002F1010E1CBFDFF8A0
:1013800078C002325FFA8EFE83F800E01FBF8CF84F
:101390000020174A4FF0150C02F80EC0182F41D14B
:1013A0002CE000BF00240140FC280020842A0020FB
:1013B000E8230020404B4C0004100020000C0140AA
:1013C000C8100020D8180020080100209023002019
:1013D00035FA8E3CB42300200AE81C4100401C462C
:1013E0001402002030180020BD3786358C230020E1
:1013F000CD0F00201C000020CC0F00201A784FF0E9
:10140000160E00F802E002F1010E5FFA8EFE4FF0B8
:10141000170C00F80EC002F1030E0232D2B283F8AC
:1014200000E087540F0341BF1A78511C197019232B
:1014300048BF835400219822A24815F088FF09F084
:101440008AFDA14AA14BA2491A6000234B800B716F
:10145000B4F896019F490A6081B29F4A22F813109E
:101460000133122BF9D19D4F3B68D9045CBFB4F80E
:101470009C1111801B0740F1D58094F89031062B08
:1014800000F2CA80DFE803F0040430566D89890059
:101490009349944A012B0A60934C9448944908D18B
:1014A0004FF0030E84F800E007240B7004700C2347
:1014B00006E0022323700323037000230B7007232D
:1014C00013708C4A8C4B40201A6006F05DFA00289D
:1014D00000F0A28001234FF0000B90F900004021A2
:1014E0008DE80808854A39E012F01EFA844912F0A6
:1014F0006FFA844912F062F912F056FC0023824A16
:1015000042F823000133122BF9D17B4A7F49402056
:101510001160744A137006F037FA00287CD001235A
:101520004FF0070A90F9000040218DE80804784A3E
:10153000784B6BE0784A704B40201A60694B102260
:101540001A7006F021FA002866D001234FF0000936
:1015500090F900008DE80802704A40214FF4E13311
:1015600054E06F4A644B40201A605E4B08221A70A8
:1015700006F00AFA00284FD001234FF0000C90F932
:10158000000040218DE80810664A4FF4E13306F070
:10159000D1F8654BC3F87C013AE052490C22062B86
:1015A000DFF8B8C1DFF8B8E1604C61480A700FD0CD
:1015B000002323708CF800308EF800301B2303705A
:1015C0005C4B4FF4E1341A705B4B05221A700CE04F
:1015D000002121708CF800108EF80010212101707C
:1015E0005449564C0A70544A1370554A424B402095
:1015F0001A6006F0C9F978B101234FF0000E90F996
:1016000000008DE8084023464E4A402106F092F83B
:10161000003018BF012028B9082007F0C5FC364B60
:1016200000221A603B682F4A13F4804F1FBF082125
:1016300011704548304918BF086042F20101194055
:1016400079B1980441BF0821117040482A4948BF28
:101650000860D90741BF0C2111703D48264948BF99
:10166000086011781C06A1F10401517040F1B580A9
:101670002D48DFF8F0A04FF00009364CC0F880A1EB
:101680004946152200F5C270DFF8DCB084F80190FD
:10169000C4F80490C4F8089015F059FEAAF10503A7
:1016A0004846CBF800300BF072F82B4B02201B6839
:1016B000E36006F069F9002858D1802007F074FC37
:1016C00084E000BF8C170020842A0020E00E002058
:1016D000B4330020F4320020D82800209C280020B9
:1016E000DC00002088330020D8000020E00000202B
:1016F0000325002079020108843300208D030108AE
:10170000CDCCCC3F0000B04494320020452E0108DF
:1017100019300108A0860100352E0108612F01084B
:10172000A1020108D9030108500900205C2500200E
:101730005E250020012500205F25002090D00300B9
:10174000CD010108B9020108712E01088D2E010892
:101750007D2E010830020020C02800200225002034
:101760005D250020E22A00205002002090F805E0CC
:101770006378C8490C2202FB03125278724504D0E8
:101780000133DBB2042BF4D900236370DBF80030A3
:1017900062781B7890F90000002B4FF00C0303FBDC
:1017A000021314BF4FF0030E4FF0010E00225B78BE
:1017B000CDF800E00192022105F0BCFFB64B1860A5
:1017C00000283FF47AAF01200AF0E1FF2868B34B0C
:1017D00000F5C5721A600BF081F83B68980553D587
:1017E000AF4AB04C049B102523609369AE4843F088
:1017F00001039361049B0EA91B888DF83A50ADF844
:10180000383002238DF83B300DF0C7F92368A64825
:101810005B880EA9ADF8383004238DF83A300DF00E
:10182000BCF923680120197A0DF0A2F923689F4AB8
:101830005B684FF00009536117A88DF861500125CE
:1018400017938DF860908DF862500EF0D1FF2368E9
:101850000FA85B7A8DF83E908DF83C3003238DF80D
:101860003D308DF83F5010F031FE914B914A1B688E
:101870003C3B1360D8F800304FF0FF3243F01003C8
:10188000C8F800308C4B1A608C4B8D4A8D4C13601D
:101890008D4A803313603B680025D903257040F1E1
:1018A000AF8040F22A39DFF854A2DFF8F4B10FF02C
:1018B000ABFE4FF001084A465046294684F80080A6
:1018C00015F045FDDBF81830804843F00403CBF8F1
:1018D00018304023ADF8383018238DF83B300EA96E
:1018E00003238DF83A300EF0C1FFDBF81C30784A44
:1018F00043F00203CBF81C30764B774C1B68ABF6F9
:10190000947BB3FBF2F32288013B22F45C72120455
:10191000120C22809BB21D22A2852385A4F814807C
:10192000238C23F001031B041B0C2384238CA1882C
:10193000228B23F0020322F0730212041B04120C08
:101940001B0C89B242F0600243EA0803A1802283A3
:10195000A5862384238B23F008031B041B0C43F070
:1019600008032383B4F844306FEA43436FEA5343D8
:101970009BB2A4F84430DBF8A83F43EA0803CBF855
:10198000A83F58460EF04EFD544BCDF860A017937B
:1019900080231C934FF480734FF0100A1D93584618
:1019A0004FF4005317A920931B951E951F95219561
:1019B000CDF864A0CDF868900AF028F8A3890FA8A4
:1019C0009BB243F40073A381DBF8003043F00203C1
:1019D000CBF800308DF83CA08DF83D808DF83E505E
:1019E0008DF83F8010F072FD3D4B1A683D4B43F877
:1019F00026200136202EF7D10CF0DCFF0CF0DAFFA8
:101A00003B685A0540F18C80374C384BD4F8C4649D
:101A100004201E6005F0B8FF0421C4F8C80405F0D6
:101A20008FFF334B84F8CC0408201E6005F0ACFF18
:101A30000821C4F8D00405F083FF2E4D84F8D404A7
:101A4000002128462C2215F082FC8E236B704FF06B
:101A50007C09E0234FF07D08EB7085F8009085F855
:101A60002B80254D2C220021284615F070FC8A235E
:101A70006B701020A023EB7085F8009085F82B8008
:101A8000C4F8D86405F080FF1021C4F8DC0405F028
:101A900057FF35E018990108E42300203C0F00208F
:101AA000001002402C020020000C01400004014004
:101AB000C028002028020020241000201C2B002019
:101AC00090110020C90800202824002000080140AF
:101AD00000366E015800002000040040340400402D
:101AE000509D0108CA08002050090020BC100020A9
:101AF00014110020E410002019110020E90A002030
:101B000084F8E0042020C4F8E46405F03DFF2021BF
:101B1000C4F8E80405F014FF84F8EC0406F04EF96C
:101B2000804B814C1B78022B65D1804A002513889D
:101B3000322023F040031B041B0C138013884FF446
:101B4000805623F038031B041B0C138013889BB2B0
:101B500043F0400313809F238DF83C308DF83D50B7
:101B60008DF83E508DF83F500BF029FB8DF85D50FD
:101B70006F4D04226E6117A80FA910F0C5FC2E61ED
:101B80009DF85E309DF85D201B0243EA02429DF8FD
:101B90005F301343674A934219D00AD8A2F51A421C
:101BA000033A93420CD002F51A420232934209D012
:101BB0001CE0614A934205D00132934207D015E000
:101BC000202300E0802323804FF4807302E04FF451
:101BD000807323806380A38822881B02A360534301
:101BE000E360564B012283F8ED2404E000232380B8
:101BF0006380A360E360E46804B3240C26464FF0DE
:101C00000008A04514DA08EB04056D100DF15C091D
:101C10002804494610220DF02DF9002359F82320FD
:101C200001325AD10133042BF8D12E462C46E8E775
:101C30000BF018F8414B3604C3F8F0643B68404A97
:101C400013F4002318BF012313700BF091FA3D4BDE
:101C500018603D4B5A791946052A02BF3B4B4FF499
:101C6000C8721A803A4B4FF47A721A80394BC822E4
:101C70001A80394A137843F008031370374A1378EF
:101C800023F00203137040F602033A6813406BB16D
:101C90003348344B1860344B03201870334B012009
:101CA000187033480023038032480380930341BFF8
:101CB000314B04221A71DA7844BF42F00102DA7023
:101CC0008B6801223B602D4B1A702D4A137863F00C
:101CD0007F03137023B0BDE8F08F05F1010825469E
:101CE000A4E7284B00221A7000B211F01DFE26490D
:101CF00011F06EFE1790B4F95E0111F015FE224945
:101D000011F066FE1890B4F9600111F00DFE1E4945
:101D100011F05EFE1D49199017A807F05DF8FFF756
:101D2000DAB900BFE73300200C0000200038004083
:101D3000000C014018BA20001740EF0050090020A5
:101D4000D0300020D4020020FC280020F20E002019
:101D5000DE330020DC330020CC100020E5330020EF
:101D6000762A0020B4100020181100204D00002019
:101D7000600E0020620E0020E8230020C80800202A
:101D8000BC3300204000002035FA8E3CA425002002
:101D9000B54B2DE9F04FB3F90610B44B85B01F6871
:101DA00001937A8991420EDBB1F5FA6FFC79BFBFDE
:101DB0008B1A6343A2F5FA6493FBF4F4ACBFC4F14D
:101DC0006404643400E06424A94BAA4AB3F896B1D1
:101DD00093F9623112689BB2029215460393002276
:101DE00040F2E630A04B4FEA420C33F912E0CBEB65
:101DF0000E0303F2F316864203D8002BB8BF5B42F2
:101E000001E04FF4FA73022A2ED0029E96F8116177
:101E10001EB1B342CCBF9B1B0023642093FBF0F8A0
:101E2000954E6FF0630A36F818900AFB083A08F1ED
:101E3000010836F918600FFA89F8C8EB060606FBA8
:101E40000AF696FBF0F68D484E4420F80C60BE185A
:101E50003679642073438A4E93FBF6F364339BB266
:101E6000634393FBF0F02CE0029890F812611EB1EE
:101E7000B342CCBF9B1B0023642093FBF0F0DFF840
:101E80002C926FF0630808FB003A39F910600130BA
:101E900039F91000002BA0EB060000FB0AFA9AFBB0
:101EA000F8FA0398C6EB0A0A0AFB00FA7348B8BFAF
:101EB0005B42A0F804A0B8794343714893FBF0F06B
:101EC00064306B784FF06408434393FBF8F36D4E36
:101ED000022AB354EB7A6C4E00FB03F393FBF8F346
:101EE000B3546B7D654E00FB03F090FBF8F0674B3D
:101EF0009854674B0ED1DE4583F802800DDB5C4CB5
:101F0000B4F89821914214DBB1F5FA6FA8BF4FF4F1
:101F1000FA610FE0DE459C5404DA36F80C305B427F
:101F200026F80C300132032A05F101057FF458AF81
:101F3000E5E71146891A4FF47A735943C2F5FA62FC
:101F4000B1FBF2F1642391FBF3F2DFF874E16FF07F
:101F500063073EF8120007FB021101323EF912201E
:101F600007B2D21B514391FBF3F30344F380494B77
:101F7000424D1B885F063BD5474A484B10881B885B
:101F8000181A00B211F0D0FC454911F021FD0746A6
:101F900006F018FF8046384606F0A1FE0746B5F960
:101FA000020011F0C1FC8146B5F9000011F0BCFC43
:101FB0004146824611F00CFD39468346484611F0F1
:101FC00007FD0146584611F0F9FB11F0C7FE4146E6
:101FD0002880484611F0FCFC39468046504611F0F6
:101FE000F7FC0146404611F0EBFB11F0B7FE6880AC
:101FF0002C4D2B68980740F19E8045F207212A4B13
:102000002A4F1A687B69D31A8B4240F394807A6115
:102010000EF09AFD264BDFF8AC901A789846032A0A
:10202000B9F8003050D10A2B58D90023282088F85D
:1020300000300BF0C4F80EF087FD1E4B18880EF030
:102040006DFD1D4B1A68D37890FBF3F00130082822
:102050001A4BA8BF08201870537980B243433B83C2
:1020600013795843788339E0D82800202C100020B9
:10207000FC28002004100020AE110020AC1000202D
:102080000CFEFFFF60240020560E00207424002068
:10209000A82100208C110020360F0020A410002061
:1020A00035FA8E3C9C280020C4330020480E0020C6
:1020B00018110020E0250020B41000204D00002061
:1020C00096110020B81000200A2B07D803239B4A42
:1020D00088F80030002313703B837B8398F800302E
:1020E000974A012B0CD002D3022B1BD023E03A8B52
:1020F000B9F800309A421EDD012388F800300FE065
:10210000B9F800107B8B8B4202DD022313700FE0C5
:102110008C4B1B8B0133994202DD002313700AE0C4
:10212000082006E07B8BB9F8002001339A42E3DCFB
:1021300007200BF081F82D68290575D5824B814F5A
:102140001A68FB69C3EB020845F2072398456BDD6B
:10215000B6F906304FF47A71A3F57A7B7B4BFA61BE
:10216000D3F8009098FBF1F899F80A30B4F85201CE
:10217000012B774E03D040D3022B1FD03FE0754B8D
:10218000386A5A7B744B4FF0080E33F8122090FBDC
:10219000FEF392B2C01A83183B6293FBFEF3BA843B
:1021A00040F6E4429BB25343B9F80820C2EB133324
:1021B0004B43B9F9062093FBF2F31FE0674BB9F8E4
:1021C00008A01B78C6F800A05A0718D510F039FCF3
:1021D00020B915F0100F18BF4FF0000B0BFB0BF1DF
:1021E000322391FBF3F3B9F906205B445A434FF4D1
:1021F0007A7392FBF3F3534400E0002333603368B7
:10220000D7E90A0103FB08F84FF47A7398FBF3F857
:1022100010EB080041EBE8710023C7E90A01504ABE
:1022200011F0E2FD4F4B18604F4E3368DB0427D5A9
:102230002F0622D54D4B1B789D071ED54C4B187889
:1022400004281AD900224B4B0521D718951C4FF0B2
:102250000A0E122AD154E9B287F801E004D0B0EB9B
:10226000510F2A46EFD800E014215A18322002F804
:10227000010CFF225A540F2000E00A200AF0DCFF74
:102280003D4D2A68002A51D03C4B3D4F18683968B3
:10229000984681424AD83B4BDFF8F490197852684F
:1022A000E1B94FF0010A83F800A0B9F80030D35C1F
:1022B00023B350460AF0A2FF334B83F800A011F07D
:1022C0003FF8B9F80030CBB92B681B78053B534574
:1022D00014D80AF04DFF2D4B18600FE04FF0000AA4
:1022E00083F800A0B9F80030D35C3BB150460AF047
:1022F00085FF254B83F800A011F022F82B68B9F870
:1023000000205B6822499B5CFE2B02D100230B80DE
:102310000CE0FF2B02D10AF077FF07E0D8F80000AD
:102320000A2505FB030301323B600A800B4D2B7825
:10233000580731D5174B08225A616BE04D00002039
:1023400018110020480E0020C4330020B4100020D3
:10235000C0100020C8250020D8250020E53300202B
:10236000407E0500C4100020C80F0020CC100020C3
:10237000D21000202427002064220020C028002042
:102380005C220020582200208B3300208432002061
:1023900060220020000C01403268D1075CBF43F08E
:1023A00001032B70984B1B781F075EBF2B7823F01F
:1023B00001032B70D60248BF2B78944A44BF23F008
:1023C00001032B70924B1B6813F0040F02D091494C
:1023D000098851B99049098809B1980705D48F4BEC
:1023E0001B88003318BF012333B1022313702B78ED
:1023F00023F001032B7004E02978C90758BF02239A
:1024000013700AF0B5FE864B1B68C01A002801DB6A
:1024100010F096FF05F0D2FC824B1E789846002EF5
:1024200000F0AB80804E3368002B00F0E786306808
:102430000AF094FF002800F0E1867B4B7B4C186883
:102440000AF089FF092801D03F2850D14FF0000A37
:102450005746D4F80090764DB9F1000F05D0754875
:1024600029684A4614F0C0FF10B9AA4607B92F469A
:10247000714B10359D42EFD3C7B1D7F800E0DAF8C1
:1024800000C023681EF803501CF80300A8420DD1B9
:102490005A1C684938B92D2B05D8644D2A6020256F
:1024A000CD54885402E0CD542260EAE723680BB192
:1024B000574511D061480EF093FD574507D857F89E
:1024C000100B0EF08DFD09200EF082FDF5E75C4843
:1024D0000EF086FD4FF0000923689945A7D2554BB1
:1024E00013F809000EF074FD09F10109F4E72368FF
:1024F000002B40F06886042840F0A6864D480BF07B
:102500001DFD00F07BBED9F80000DFF844A10AF001
:1025100025FF40B3DAF800000AF01DFFDBF80030B9
:10252000024693F84810002935D1242840F09280C3
:10253000012283F84820DBF80030DFF810A193F87F
:102540004820062ADFD193F8490002F0C7FF8146F0
:10255000002800F0A3803B6898790EF08EFC3B6861
:10256000002283F84820374B93F83530002B40F099
:1025700018864C36982E00F04186334BF21892F8AC
:102580004A100129F5D1314FF3583A60304ABB4621
:1025900013609146B7E7012904D14D2814BF0022EA
:1025A0000222C6E7022904D13C2814BF00220322DC
:1025B000BFE703290CD140284FF0000102D983F86E
:1025C0004810B8E758711971D97198710422B0E7B1
:1025D000042906D1997983F849004A409A71052265
:1025E000A7E70529A7D1587919798842987906D99A
:1025F00050409871481C18710B441A729BE7904226
:102600000CBF0622002294E7CC1000208B33002060
:10261000C8100020DC330020F20E0020DE33002042
:102620008C330020E9330020DC2600202424002005
:102630008CA50108F42300206CA70108E8BF01085D
:10264000EDBF0108480E00208C1700206C110020FF
:10265000701100202B7858073FF56DAF232ADAF868
:1026600000300ED1012188F80010AE49AE480B6051
:10267000AE4902920B630EF0B3FCAD480EF0B0FC15
:10268000029AAC4B1B681B78934201BFAA4AAB4B22
:102690001A60AB4A04BFAB4BDA604CE7DAF80020B3
:1026A00092F849304A2B00F038815CD8332B00F087
:1026B0009E8421D8292B00F0388409D8252B00F0DE
:1026C0000F84272B00F01384232B40F0B9853CE2C4
:1026D0002D2B00F03B8407D82B2B40F0B1850EF05A
:1026E000AFFB607100F058BD2F2B00F00885312B37
:1026F00000F01A8500F0A4BD3E2B00F004811DD827
:10270000372B00F0C48404D8352B00F0578200F03A
:1027100097BD392B00F0F8833C2B40F09185DFF812
:102720002892D9F800A00EF08BFB8AF80000D9F8A7
:10273000003018780BF03EFA00F02EBD432B00F06D
:10274000838406D8412B40F07B854FF0000900F0D0
:1027500053BC442B00F01C85482B40F071850AF0D7
:10276000BFFA00F019BDD02B00F0338368D8CA2B14
:1027700000F0F2801CD84E2B00F00B8410D84C2BAC
:1027800040F05E850EF05CFB84F8CE010EF058FB45
:1027900084F8CF010EF05EFBA4F8D00100F0FCBC81
:1027A000C82B00F08380C92B00F0348300F048BDB3
:1027B000CD2B00F0198304D8CC2B00F0278200F039
:1027C0003FBDCE2B00F01983CF2B40F039850EF0A2
:1027D00041FB6FF4AF6283189BB2C62B98BFA4F87D
:1027E00096010EF037FBA4F844010EF033FBA4F879
:1027F00046010EF02FFBA4F848010EF02BFBA4F8C5
:10280000D0010EF01DFB84F8E1010EF019FB0EF073
:1028100017FB84F8E2010EF013FB84F885010EF03B
:102820000FFB84F892010EF00BFB474BD3F800909E
:102830000EF010FB00EB80004000A9F8560063E3A7
:10284000D62B00F04B820AD8D22B19D0C0F00983C6
:10285000D32B25D0D42B00F04C8200F0F1BCEF2B11
:1028600041D005D8D82B40F0EB844FF00009FFE0B1
:10287000F22B00F08682FA2B00F0C88200F0E0BC58
:102880002B78590700F188840EF0DAFA022884F8D0
:10289000A80740F2A4822D4B002283F8A8279EE2CD
:1028A0000EF0D8FA2A4B188000F076BC92F805900A
:1028B0004FEA5909B9F1120F03D909F071F800F084
:1028C0006BBC4FF0000ACA4507D20EF0C3FA214B89
:1028D00023F81A000AF1010AF5E7144B012283F8E4
:1028E000342000F059BCDFF86090D9F800A00EF059
:1028F000B1FAAAF85A00D9F800900EF0ABFAA9F88C
:10290000580000F049BC0EF09BFA84F8D4010EF098
:1029100097FA84F8D30100F03FBC0EF09BFAA08137
:1029200000F03ABCDC2600201DC00108480E002043
:10293000EDBF0108E8180020EFBEADDEF04F00202B
:102940000400FA0500ED00E004100020FC2800203F
:10295000340F0020D8280020D64B1A689A461278E7
:10296000022A6AD1DAF8003009F1080B02930EF05E
:1029700067FA10F0D5FFD04911F0DEF8029B43F85A
:102980002B00DAF800B00EF05BFA09F10A030BEB4A
:10299000830B10F0C5FFC94911F0CEF8DAF800300A
:1029A000CBF8040002930EF04BFA10F0B9FFC449C3
:1029B00011F0C2F809F10E0B029B09F10109B9F1FE
:1029C000030F43F82B00CDD1B9F1070FDAF800B0AF
:1029D0001AD10EF035FA10F0A3FFB74911F0ACF898
:1029E000CBF84400DAF800B00EF02AFA10F098FFA5
:1029F000B14911F0A1F8CBF84800DAF800B00EF0B8
:102A00001FFA8BF84C0012E00EF01AFACB448BF848
:102A10000100DAF800B00EF013FACB448BF80B008B
:102A2000DAF800B00EF00CFACB448BF8150009F17F
:102A30000109B9F10A0FC7D1AEE3DAF800B00EF020
:102A4000FFF9CB448BF80100DAF800B00EF0F8F98A
:102A5000CB448BF80B00DAF800B00EF0F1F9CB4460
:102A600009F10109B9F10A0F8BF81500E5D193E3DB
:102A7000DFF840A209F1080BDAF8003002930EF0FB
:102A8000E9F910F04DFF8E4911F056F8029B43F81A
:102A90002B00DAF800B00EF0DDF909F10A030BEBB8
:102AA000830B10F03DFF864911F046F8DAF800304C
:102AB000CBF8040002930EF0CDF910F031FF8049FD
:102AC00011F03AF809F10E0B029B09F10109B9F175
:102AD000030F43F82B00CBD1B9F1070FDAF800B0A0
:102AE0001AD10EF0B7F910F01BFF754911F024F858
:102AF000CBF84400DAF800B00EF0ACF910F010FF9B
:102B00006F4911F019F8CBF84800DAF800B00EF070
:102B1000A1F98BF84C0012E00EF09CF9CB448BF835
:102B20000100DAF800B00EF095F9CB448BF80B00F9
:102B3000DAF800B00EF08EF9CB448BF8150009F1ED
:102B40000109B9F10A0FC7D126E30EF079F913286C
:102B500083463FF6B2AEDFF85CA1DAF800900EF0E3
:102B60006FF9002357490C2202FB0312117A8142AC
:102B700020D1137809EB8B0989F879300EF060F9D0
:102B800089F87A000EF05CF989F87B000EF058F9AC
:102B90004D4A4E4B89F87C001A60DAF800004C4B25
:102BA00000211860793004F07BFF4A4B80F001006F
:102BB0001870F1E201331B2BD4D17EE60EF040F900
:102BC0000B2882463FF679AE3A4BD3F800900EF0D0
:102BD00037F903283FF671AE062303FB0A9989F8FB
:102BE000CE000EF02DF989F8C9000EF029F989F808
:102BF000CA000EF025F989F8CB000EF021F989F80A
:102C0000CC000EF01DF989F8CD00C5E25379092BEF
:102C10007FF653AE019BD3F800900EF011F9019BA3
:102C200089F80000D3F800900EF00AF989F8010045
:102C30000EF006F9019B64281B68A8BF6420187178
:102C40000EF0FEF8019B64281B68A8BF6420587131
:102C50000EF0F6F8019BFF281B68A8BFFF209871B3
:102C60000EF0EEF8019B6428D3F8009028BF642092
:102C700089F807000EF0E4F8019B89F80200D3F808
:102C800000900EF0DDF8019B89F80300D3F8009066
:102C90000EF0E0F83B68A9F80A005B790A2B40F2D5
:102CA0007B820D4BD3F800900EF0CAF889F808002B
:102CB00072E200BF04100020000020410000C84262
:102CC00000007A44309E0108402A00202C0F00208A
:102CD000300F0020080000202C1000200EF0BAF861
:102CE000CB4B23F8190009F10109B9F1080FF5D10F
:102CF00052E253790F2B7FF4E0AD0EF0A1F80728D4
:102D000081463FF6DAADDFF834A3DAF800B00EF012
:102D1000A1F80E2303FB09F9CB44ABF81901DAF84B
:102D200000B00EF097F8CB44ABF81B01DAF800B016
:102D30000EF090F8CB44ABF81D01DAF800B00EF0BD
:102D40007FF8CB448BF81F01DAF800B00EF078F86A
:102D5000CB448BF82001DAF800B00EF071F8CB44C8
:102D60008BF82101DAF800B00EF06AF8CB448BF84A
:102D70002201DAF800A00EF077F8D144C9F8230157
:102D80000AE20EF05DF80F2881463FF696AD0EF090
:102D900057F8C9EBC909A14489F8D4000EF050F8DE
:102DA00089F8D5000EF04CF889F8D6000EF048F8F6
:102DB00089F8D7000EF044F889F8D8000EF040F8F2
:102DC00089F8D9000EF03CF889F8DA000AF08AFC9C
:102DD000E2E12B785B0700F1DF810FF02FF806F0BE
:102DE00015F906F0B5F9D7E12B78580700F1D48131
:102DF000884B4FF4C8721A80CEE12B78590700F146
:102E0000CB81854A137843F0040328E02B785A07D6
:102E1000E5D515E20EF014F87F4B1A7810B142F0A8
:102E2000020201E022F002021A700EF009F87B4B58
:102E3000DFF80C9218700EF017F8C9F800000EF0C9
:102E400013F8C9F804000EF005F8754B18800EF061
:102E500001F8744B744A1880137843F0020313701E
:102E60009AE10DF0EDFF02900DF0FEFF83460DF0AC
:102E7000FBFF82460DF0F8FF81460DF0EBFF0DF0F1
:102E8000E9FF0DF0DDFF029BA3B9684B1020C3F8EA
:102E900000B0C3F804A006F066F85F4A137843F068
:102EA00001031370B9F1000F00F07681604BC3F895
:102EB000009071E1102B40F06F815E4BC3F800B0C1
:102EC000C3F804A0B9F1000F02D0594BC3F8009029
:102ED0005848594B0222011D1A7009F0B9FC5BE1F8
:102EE000A0600DF0C1FFA3681843A06054E10DF08D
:102EF000B1FFA4F85C010DF0ADFFA4F85E010DF088
:102F0000A9FFA4F8600147E10DF09AFF84F87A0167
:102F10000DF096FF84F87E010DF092FF84F87D019C
:102F20000DF08EFF84F87F0136E10DF093FFA4F8D9
:102F300080010DF08FFFA4F882010DF081FF84F86D
:102F400084010DF087FFA4F8860125E10DF078FFDC
:102F500084F890010DF07EFFA4F89A010DF07AFF3D
:102F6000A4F896010DF076FFA4F898010DF068FF23
:102F7000DAF8003084F891015B79082B40F20C817B
:102F80000DF068FFA4F89C010DF064FFA4F89E0109
:102F900002E192F805900323B9FBF3F9B9F10E0FA2
:102FA0003FF68BACDFF89CA04FF0040BCB4580F0D4
:102FB000F3800DF045FF8AF8A0010DF04BFF40F2C1
:102FC000ED23984205DD40F6CA039842A8BF184693
:102FD00001E040F2EE20A0F2EE20192390FBF3F086
:102FE0000BF1010B8AF8A1010AF1020ADEE70DF0EC
:102FF00027FF84F89201CFE00DF022FF04EB0903D4
:1030000009F10109B9F1080F83F88801F4D1C3E08F
:10301000C2260020F20E0020CC100020D21000208A
:10302000D0100020CE1000203210002034100020DC
:10303000441000203C100020380F00200410002015
:10304000D4100020FC2800200DF0FAFEC4F80890EF
:1030500060710DF009FFA3681843A0600DF0F0FE49
:1030600084F890010DF0F6FEA4F85C010DF0F2FE7C
:10307000A4F85E010DF0EEFEA4F860010DF0EAFE8A
:10308000A4F880010DF0E6FEA4F8820184E05379F3
:103090004FF0070AB3FBFAF2C2EBC2029A1A12F01F
:1030A000FF0F7FF40AACB3FBFAFA0AF1FF3A5FFABA
:1030B0008AFABAF1FF0F6FD00DF0C2FE5FFA80FB03
:1030C0004FFA8BF004F086FB814600283FF4F5AB05
:1030D00080F800B00DF0BEFEA9F802000DF0B0FEC1
:1030E00089F804000DF0ACFE89F805000DF0A8FE8B
:1030F00089F807000DF0A4FE89F80600D5E7DFF88F
:103100005C9209F1400A0DF0A5FEA9F8A0020DF0AD
:1031100097FE89F8A2020DF093FE09F1040989F8DF
:103120009F02D145EFD137E00DF08AFE1F2881467E
:103130003FF6C3AB3B685B79082B7FF4BEAB0DF069
:1031400089FE09F1880904EB890A00F03F00AAF81A
:1031500002000DF07FFEBAF80230800100F4FE504C
:103160001843AAF802000DF06BFE000104F82900D4
:103170000DF066FE14F8293000F00F00184304F833
:1031800029000DF05DFE8AF801000EF03DFA03E023
:103190005F4B012283F8352000200DF09DFEFFF7E4
:1031A000DAB95C4B98590AF0D0F818B932200AF015
:1031B00006F8F6E70AF054FA05F0FEFE564A574BB9
:1031C000DA60FFF7D6B90C2840D00A2847D1544D11
:1031D00054480DF005FF2846232114F0EEF808B1FD
:1031E000401B20602368002B5CD14D480021302219
:1031F000236014F0ACF898F8003053BB4A4B1B68BE
:103200009B0614D5494B42491B688A6B9A1A002ABF
:103210000DDB474A1278042A09D903F5123303F566
:10322000F873444A8B63D36883F01003D360424B36
:103230009B68002B69D0414805B0BDE8F04F1847A6
:1032400008F0AEFBFFF787B90C2804D13C480DF01D
:10325000C7FE3C480DE07F2812D1FFF7E8B80D28E3
:10326000B5D07F2809D12E4A013B00213648236082
:10327000D1540DF0B5FEFFF7DAB82F2B3FF6D7A8E3
:10328000A0F12002D2B25E2A3FF6D1A813B92028BD
:103290003FF4CDA85A1C2260214AD0540DF098FE6C
:1032A000FFF7C5B85A1EA95C202901D113469AE739
:1032B0001B4A00212360D154244B254DD3F800A094
:1032C000D5F800B0DFF85890584614F084F8074657
:1032D00059463A46484614F087F81E4A28B919F864
:1032E000073053445B785B0703D010359542E7D332
:1032F00006E0954204D2781CEB684844984702E007
:1033000015480DF06DFE00236FE705B0BDE8F08FA6
:10331000480E00208C1700200400FA0500ED00E0A4
:10332000F423002029CF0108C8100020C433002056
:10333000D2100020000C014030180020840E002024
:10334000F2BF0108EDBF010819C0010860000020AC
:103350008CA501086CA70108FDBF0108FC2800200E
:103360009148F0B50368914A9C8AA4B2E1B211F089
:10337000010F2ED0198821F400610904090C19806D
:10338000198889B241F48061198000211170517847
:1033900099B1917811B9D178FF290ED1012191709D
:1033A0001179022901BF198889B241F4006119809D
:1033B000517941F001011982E1E0517901F0FE01FA
:1033C0001982D378FF2B00F0DA80784BFF21197037
:1033D000D5E08E073AD5BFF35F8F1479E4B2012CA4
:1033E00013D1517889B1917879B1198821F480612C
:1033F0000904090C1980BFF35F8F198B1988947128
:1034000089B241F4007119801BE0198BBFF35F8F03
:1034100014796649022C0AD14C7844B1897831B1CB
:10342000198821F480610904090C1980A1E014793C
:103430005E49032C05D14C781CB18978002940F0F5
:103440009880998889B241F4806197E04D0756D5FC
:10345000012191715178002937D09178002934D019
:1034600011791C88022911781DD924F48064240460
:10347000240C1C801E8A9568CCB2F6B249B26E54F8
:10348000198889B241F4007119800168A31C137076
:103490000B8A0134DBB264B22B558B889BB243F4A8
:1034A00080638B8026E0A4B244F400741C801D8AE3
:1034B0009668CCB2EDB249B275541B8A611C49B210
:1034C000DBB203347354147014E09178374C09B9AB
:1034D000217B41B1198889B241F4007119801378B8
:1034E0000133137006E0198889B241F480711980A4
:1034F0000123A37001680B88DB05FCD43FE001F0D9
:10350000400101F0FF05E1B114781F8A9668E5B229
:10351000691C64B2FFB23755C9B21679117049B24D
:10352000CC1CA64201BF9C8824F480642404240C93
:1035300008BF9C8013798B4221D11C4B02351D7032
:103540001DE027061BD511784CB2661C0AD0156900
:1035500001312C5DC9B21C821479117049B28C42C0
:103560000DD106E0D17815701982517809B9117919
:1035700029B9998821F480610904090C998013798B
:1035800092F9004001339C4208490CD100238B7012
:103590008B7933B101688B8823F440731B041B0CB7
:1035A0008B8000231375F0BD44240020880E00207A
:1035B0006B4B6C4A2DE9F04F5E8994694FEA062AFD
:1035C000B4EB0A0A9C884FF000054FEA04481C89B6
:1035D0004FF0000BA4FB0A6765EB0B0B04FB0B77AA
:1035E000F40944EA476418EB04065C884FF00009CC
:1035F0004FEAE7154FEAC438DC8849EB050787B086
:10360000CDE90467A4FB0A6704FB0B77340A44EA9C
:10361000076418EB04064FEA27259C894FF0000940
:1036200049EB0507CDE90067AAFB046704FB0B77AC
:10363000F40D44EA472414F5FA664FEAE75545F1DC
:103640000007B6F5FA6F77F10003CDE902679646F9
:1036500066DADDE90489A4FB046704FB05F34FF097
:10366000050C07EB4307A6FB0C230CFB07335F108D
:103670004FEA3206B8EB06084FEA920646EA83762E
:1036800069EB07099F10DDE90023921B63EB070339
:10369000CDE90023DDE90267334A4FF0FF3396425C
:1036A00077EB0303CDE9048927DA40F6AC52002317
:1036B000A4185D4104FB05F3A4FB04456FF006026A
:1036C00005EB4305664202FB0566A4FB0223334477
:1036D00018EB020649EB0307CDE904670B26A4FBB0
:1036E000062306FB0533DDE900455B104FEA320295
:1036F000A41A65EB0305CDE90045DDE902450AFBA7
:103700000BF3AAFB0AAB0BEB430B4FEADA7242EA6C
:103710004B02A41A4FEAEB7365EB0305CDE90245B2
:10372000DEF81C40009B019DA4FB032304FB053332
:103730004FEA525848EAC3284FEA6359DDE90423A7
:10374000B8EB020269EB03039946D30B43EA494302
:1037500000B1036009B1029B0B6007B0BDE8F08FB8
:1037600050180020880E002024FAFFFF2DE9F04FAA
:10377000DFF8589285B00746D9F820000E4610F0C1
:10378000D3F88E4C8046208810F0CAF84FF05C5178
:103790000546404610F01CF94FF064518246284619
:1037A00010F016F90146504610F008F84FF062513B
:1037B0008246404610F00CF94FF06A518046284688
:1037C00010F006F9014640460FF0F8FF0546B4F93F
:1037D000020010F0A9F80146284610F0F9F8514609
:1037E0000546504610F0F4F88046B4F9040010F095
:1037F0009BF80146404610F0EBF8014628460FF0D2
:10380000DFFF804610F0AAFA6D490546A0614046E8
:1038100010F092F9D9F8243080462846019310F030
:1038200083F84FF07C5110F0D3F866490FF0C6FFD3
:103830000546E389B4F90A00029310F075F82946A9
:1038400010F0C6F8294610F0C3F84FF0585110F0A8
:10385000BFF88146B4F90800B4F810B0B4F80CA071
:1038600010F062F8294610F0B3F8014648460FF010
:10387000A7FF4FF0585110F0ABF84FF0605110F027
:10388000A7F84FF07E510FF09BFF8146E08810F0C3
:1038900047F80146484610F09BF80021814610F099
:1038A0002BFA00287BD12946284610F091F8039086
:1038B0000FFA8BF010F038F8039B0146184610F011
:1038C00087F84FF0605110F083F88346BDF9080087
:1038D00010F02AF80146284610F07AF801460FF059
:1038E0006FFF014658460FF06BFF4FF07A5110F012
:1038F0006FF88346019810F017F801464FF0934097
:103900000FF05CFF05460FFA8AF010F00DF84FF04B
:103910008F4110F05DF8014658460FF051FF4FF00F
:10392000665110F055F8014628460FF047FF26492A
:1039300010F04EF8494610F0FFF80546B4F91600AD
:103940000FF0F2FF294610F043F8294610F040F836
:103950004FF0405110F03CF88146B4F914000FF0DC
:10396000E3FF0146284610F033F84FF0605110F0A5
:103970002FF8014648460FF023FF8146B4F91200A4
:103980000FF0D2FF014648460FF01AFF4FF0765174
:1039900010F01EF8014628460FF012FF00E000204C
:1039A00017B110F0DBF938602EB1404610F0D6F9AF
:1039B00064235843306005B0BDE8F08FB018002094
:1039C0000000A04500007A470050C345880E002043
:1039D000704770472DE9F041324C334D62892B8D91
:1039E000B4F904809A1A2389B4F902E05A43B4F96D
:1039F0001230D613B4F91420DB02324493FBF2F2F6
:103A000032440A26E2615643A2F57A6202FB02F3CF
:103A1000B4F90EC002FB0EFE02FB08F2B4F90C80F2
:103A20001B130CFB03FC03FB08F31B1403EB6232B8
:103A30000232E388921002F5004253434CF25032B6
:103A4000B4F920704FEAEE2EB4F900400EEBEC2CE6
:103A50000CEB8404BC40ED6A0234A5EBA4043A41AB
:103A600062434FEAD3384EBFB2FBF8F35400B4FBC5
:103A7000F8F340F6DE3448BF5B001A12524362434B
:103A80000A4C08365C43241404EB224202F6CF624F
:103A9000361103EB221300B1036001B10E60BDE8E3
:103AA000F08100BF64180020880E002043E3FFFF70
:103AB000024B4FF480521A80704700BF1C00002058
:103AC00010B5224C2368998A89B211F4706F1EBF19
:103AD0001F4A012082F8300011F4E06F2BD01A8BBE
:103AE0009A88890522F480624FEA02424FEA124224
:103AF0009A8020D41A8892051DD41A88D0050FD533
:103B00001A88D105FCD41A8892B242F400721A8045
:103B10001A889205FCD40F4B18780BF08FFA0AE044
:103B20001A8892B242F400721A809A8822F4407283
:103B30001204120C9A802268938A23F470631B0487
:103B40001B0C9382024B00221A7510BD44240020E6
:103B5000880E002048240020054A08B51388013348
:103B60009BB21380034B18780BF068FA002008BD55
:103B7000C60F00204824002008B54FF480400CF008
:103B800067FE012801BF044B4FF480425A61034B8A
:103B900008BF83F8310008BD00040140880E0020F2
:103BA00010B5054C236818690CF052FE18B1236853
:103BB0001A69024B5A6110BD4818002000040140E8
:103BC00070B50E46054C4FF4805565610EF0D2FC81
:103BD00030460EF0CFFC256170BD00BF000C0140E7
:103BE0001D4B07B51A681D4B9A420ED14FF4005376
:103BF000ADF8043002238DF80730042318480DEB8C
:103C000003018DF806300AF0C8FF80216B20FFF712
:103C1000D7FF642009F0D3FA00216B20FFF7D0FF13
:103C2000642009F0CCFA6B200121FFF7C9FF1B20AB
:103C30001821FFF7C5FF1C201021FFF7C1FF094B1A
:103C40001A201978FFF7BCFF19200021FFF7B8FFF1
:103C500003B05DF804FB00BF3C000020001BB70070
:103C60000010014023000020F0B5264D85B095F8E6
:103C70003230002B44D1244C2368002B40D01A68EA
:103C8000224E12B1B1690A43B2619A889868ADF8C0
:103C9000002002228DF80320694604228DF80220BC
:103CA0000AF07BFFB369002743F00103B361236887
:103CB0000126197D187B0AF05BFF154809F030FBDF
:103CC0002368144A1B695361029308230DEB030018
:103CD0008DF80D308DF80C708DF80E600CF088FDAD
:103CE000236801A85B7D8DF806708DF804300323EE
:103CF0008DF805308DF807600EF0E8FB85F832602E
:103D000005B0F0BD880E00204818002000100240C9
:103D1000A13B00080004014008B5FFF7A5FF074BD1
:103D20001B7813B1012B03D008BD4FF4006201E0F2
:103D30004FF48052024B1A8008BD00BF4D1800207E
:103D40001C00002010B51E4C4000C0B2A3602361CF
:103D50001C4B6071E17001200021217360702271A1
:103D60002075186884F8301040B383889B0515D4FB
:103D70000388D9050DD447F230530288920502D545
:103D8000013BFAD112E08BB103889BB243F48073FC
:103D9000038083889BB243F44073838047F230539F
:103DA000227D12B1013BFBD100E013B9BDE8104008
:103DB000D2E6034B93F8300080F0010010BD00BF45
:103DC000880E00204424002007B5002101AB032207
:103DD0007720FFF7B7FF9DF805309DF804001B0220
:103DE00043EA00439DF80600184303B05DF804FB66
:103DF00008B5FFF7E9FF014BD86108BD880E002028
:103E000008B5FFF7E1FF014B986108BD880E00205F
:103E100007B5F7216B4606227620FFF793FF9DF842
:103E200000309DF801101B0343EA01139DF80210B6
:103E3000094A43EA111353629DF803309DF80410B8
:103E40001B0343EA01139DF8051043EA11131362A3
:103E500003B05DF804FB00BF880E002013B5104CC2
:103E600094F831301BB9A38E0133A38616E00322E8
:103E700001AB7720F621FFF765FF9DF805309DF82F
:103E800004201B0243EA02439DF806201343054A1F
:103E9000B2F92020C2F10802D340E36202B010BDA3
:103EA000880E00206418002013B50B4C94F83130B4
:103EB0001BB9A38E0133A3860CE0022201AB77204D
:103EC000F621FFF73FFF9DF804209DF8053043EAF7
:103ED0000223238502B010BD880E002013B50122F5
:103EE0000DF1070304463A216820FFF72BFF9DF8E8
:103EF000073003B10123237002B010BD13B50622B1
:103F00000446432168206B46FFF71CFFA0B19DF8D3
:103F100000209DF8013043EA022323809DF802200F
:103F20009DF8033043EA022363809DF804209DF846
:103F3000053043EA0223A38002B010BD13B5062268
:103F400004463B2168206B46FFF7FCFEA0B19DF8BC
:103F500000209DF8013043EA022323809DF80220CF
:103F60009DF8033043EA022363809DF804209DF806
:103F7000053043EA0223A38002B010BD13B501222D
:103F80000DF1070304461A216820FFF7DBFE9DF8B8
:103F9000073003B10123237002B010BD13B5022214
:103FA000044601AB1B216820FFF7CCFE9DF80420DE
:103FB0009DF8053043EA022303F54E534FF48C720B
:103FC000103393FBF2F32333238002B010BD13B5FB
:103FD00004466B461D2106226820FFF7B3FE9DF8BC
:103FE00000209DF8013043EA022323809DF802203F
:103FF0009DF8033043EA022363809DF804209DF876
:10400000053043EA0223A38002B010BD13B5062297
:1040100004466B4601211C20FFF794FE9DF80130F9
:104020009DF80020042143EA022242F38D0292FB14
:10403000F1F29DF8023022809DF8032042EA03222B
:1040400042F38D0292FBF1F29DF8043062809DF8FC
:10405000052042EA032343F38D0393FBF1F3A3808E
:1040600002B010BD13B504466B460221062218208B
:10407000FFF768FE9DF800309DF801209B0803EBD8
:10408000022323809DF802309DF803209B0803EB58
:10409000022363809DF804309DF805209B0803EB04
:1040A0000223A38002B010BD2F4B2DE9F3411B78F2
:1040B0000546002B39D0002426462746A046082274
:1040C0006B4653203221FFF73DFE9DF801209DF8FD
:1040D0000030013403EB02231BB29DF80320984407
:1040E0009DF80230E4B203EB02231BB21F449DF89B
:1040F00005209DF80430202C03EB02231BB21E4444
:104100009DF8073003F07F0301D0002BD7D198FB37
:10411000F4F897FBF4F796FBF4F6144BA5F800803F
:104120006F80AE8083F836401AE006226B4653203B
:104130003221FFF707FE9DF801209DF8003003EBC8
:1041400002232B809DF803209DF8023003EB02230D
:104150006B809DF805209DF8043003EB0223AB80B3
:1041600002B0BDE8F08100BF4C180020880E00208E
:1041700013B5204B400002ACC0B2587104F8012DB9
:10418000D970012200211A7359701A711A751A4ACE
:104190001C6110689C6083F8301040B382889205DF
:1041A00015D40288D4050DD447F230520188890510
:1041B00002D5013AFAD112E08AB1028892B242F4F1
:1041C00080720280828892B242F44072828047F20A
:1041D0003052197D11B1013AFBD100E012B9FFF75D
:1041E000BBFC04E0034B93F8300080F0010002B008
:1041F00010BD00BF880E00204424002077204821F5
:104200000122B5E7772058210122B1E77620F42179
:104210003122ADE7064B002193F82020054B920197
:10422000343283F831107720F42102F0FC029FE74A
:1042300064180020880E0020034B002283F83120F0
:104240007720F4212E2293E7880E002008B5FFF78F
:104250000BFD6B2180226820FFF78AFF642008F0A5
:10426000AEFF6B2103226820FFF782FF0F2008F0CA
:10427000A6FF124B19211A786820FFF779FF0F204B
:1042800008F09DFF0E4B1A211A786820FFF770FF87
:104290001B2118226820FFF76BFF1C2110226820C9
:1042A000FFF766FF372102226820FFF761FFBDE8B4
:1042B00008406820382101225AE700BFCC180020AE
:1042C0002100002008B5192008F079FF6820152189
:1042D0000022FFF74DFF10B9032008F0EBFF0C4B55
:1042E00016211A78682042F01802FFF741FF1721C3
:1042F00000226820FFF73CFF3D2101226820FFF7E4
:1043000037FFBDE8084068203E21012230E700BFAA
:104310002200002013B500222A211C20FFF728FFCD
:104320000E2102221C20FFF723FF0F2103221C2055
:10433000FFF71EFF2B2112221C20FFF719FF164A40
:1043400002249369154843F0040393612023ADF8D8
:10435000043004230DEB03018DF806308DF807407F
:104360000AF01BFC22462C211C20FFF701FF2D2107
:1043700001221C20FFF7FCFE2E2100221C20FFF74B
:10438000F7FE2A2105221C20FFF7F2FE044B4FF412
:1043900080721A8002B010BD001002400008014077
:1043A0001C00002008B50F2108221820FFF7E0FEAE
:1043B0000E2218201021FFF7DBFE024B4FF4805233
:1043C0001A8008BD1C00002008B5134B53201B7831
:1043D0002D2108227BB1FFF7CBFE31210A22532089
:1043E000FFF7C6FE2C210C225320FFF7C1FE5320FD
:1043F0003821902209E0FFF7BBFE31210A22532029
:10440000FFF7B6FE53202C210A22FFF7B1FE40F23F
:104410000912024B1A8008BD4C1800201C00002015
:10442000FEF79EBFFFF74CBBFEF79ABFFFF748BBF6
:10443000F8B50F461646074C4FF48055656140F0BD
:1044400080000EF097F83846002132460EF05CF8F6
:104450002561F8BD000C014013B5012204460DF1A1
:1044600007013820FFF7E4FF9DF8073003B101236F
:10447000237002B010BD13B50446694643200622DE
:10448000FFF7D6FF9DF800209DF8013043EA022394
:1044900023809DF802209DF8033043EA02236380C5
:1044A0009DF804209DF8053043EA0223A38002B062
:1044B00010BD13B5044669463B200622FFF7B8FF3E
:1044C0009DF800209DF8013043EA022323809DF8E7
:1044D00002209DF8033043EA022363809DF8042004
:1044E0009DF8053043EA0223A38002B010BD07B552
:1044F000232008F064FE6820752101220DF10703D6
:10450000FFF720FC28B19DF80700A0F1680358428E
:10451000584103B05DF804FB2DE9F04FA04EA14DCA
:104520003368A14C03F59C43203323602B889F4ABA
:1045300001332B8042F20103116889B00B4092468F
:104540001BB19B4A1378013313700EF037FEDAF873
:104550000030DF0405D5974B1B68D80701D40EF057
:1045600035FC954B37681A68907AB8B19349137B3C
:10457000013831F810001BB1C0F53B60083080B243
:1045800000B2A0F57A70B0F57A7FA8BF4FF47A70C8
:1045900020EAE0700FF0C8F9894930E0DAF800301D
:1045A000190435D56368804EFB1A002B30DB07F504
:1045B0009C4320337360834BD27A5979824B33F812
:1045C0001130317A9BB293FBF2F3013101F00F020B
:1045D00032723244537203467C4A825C0130134487
:1045E00010289BB2F8D11BB293FBF0F000B2642804
:1045F000A8BF642020EAE0700FF096F974490FF02C
:104600009BFA74490FF0E4F90FF0CEFB724B18805F
:10461000DAF80030694E13F4807F00F081806F4B30
:104620009F4204D92B7913B95E4B01221A71B5F957
:1046300000E06B4ABEF1140F1778CCBF4FF0000EAC
:104640004FF0010E574BC7F38007BEF1000F06D0A5
:104650004FF0000883F8068083F8058001E04FF0F2
:104660000308E369A8790193D4F820C0B5F9009054
:1046700069796B883288032848D8DFE800F0020E99
:104680001B36BEF1000F02D0328000222BE0002F3B
:1046900040F086863280AF713AE09CF8000000EB73
:1046A0008000814502DC328001221CE001206FB3D2
:1046B00000F0E6BE47B1019A4FF00208D28972803D
:1046C000B280BCF80200F0809CF800B09CF80100B9
:1046D000584400EB8000814500F36586002F00F010
:1046E000628632800222AA7112E032800322AA710D
:1046F00069716B8077B13A4A137843F00203137003
:10470000284B00225A710EF061FB03E03280A87141
:1047100069716B80B8F1000F02D0404608F08CFD43
:10472000304FB7F852010EF08CF90197834668B903
:104730000FF00CF82C4B0022C3F800B0C3F804B003
:10474000C3F808B0294B1A605A609A60244F3B782E
:104750005B0763D5DAF80030D8065FD5244B1B78A9
:10476000D9065BD4234B1B7893B1019B93F8D431CA
:10477000BBF1000F42D173B11F4B1A68636A9B1AD9
:10478000002B08DA0EF022FB074B83F828B045E037
:10479000BBF1000F3AD1102008F04EFD01233BE0A1
:1047A000C4330020B4330020C40E00209C28002015
:1047B000F8320020C80F0020F4320020D828002052
:1047C00000007A44C8250020D8250020CD0E002006
:1047D0000000C84200C07F4428100020404B4C001D
:1047E000E5330020FC280020D421002054240020A0
:1047F000CC10002008000020C028002033B1904ACF
:104800004FF47A71126801FB0323636294F8283035
:1048100023B108F0F9FC002384F82830019B93F8B9
:10482000D2310293019B93F8D311B3F898E1B3F816
:104830009AC10023184636F9132080087245C4BF78
:1048400060F07F00C0B201336245B8BF40F0400065
:10485000042BF0D194F829307A4A834205D192F89A
:104860002A30F92B04D8013300E0002382F82A30E3
:10487000754B84F829001A78DFF8E4819946DAB993
:10488000D8F80030DA0708D5BBF1000F14D13B7817
:10489000DB0711D50EF0EEF80EE03B7858070BD58C
:1048A0006A4B1B7843B16B7933B911B10EF08EFAB4
:1048B00002E0BBF1000FF9D094F82A30614A142BC2
:1048C000DFF8A0B140F08F80029B003318BF0123B6
:1048D000029399F8003063B392F829305F2B11D11D
:1048E0003B7803F0040303F0FF0113B10EF06EFAFE
:1048F00008E00B200491039208F09EFC039A0499AF
:1049000082F82A10029BA3B194F829307D2B10D194
:104910003B7803F0040303F0FF0213B10EF056FAE4
:1049200007E00B20039208F087FC464B039A83F8BC
:104930002A203B7803F0040303F0FF01002B52D13F
:1049400094F829303F4A572B16D1414B4FF47A72D5
:104950001A80DAF80030190601D508F00FF83D4B3F
:104960001B685A0742BF3C4A0A21118013F0080312
:1049700039D13A4A138036E0DAF80000400717D5FB
:104980005A2B15D192F82B302BB1012382F82B1022
:1049900082F82C3027E092F82D3083F0010382F862
:1049A0002D300BB10C2000E00D2008F045FC1AE082
:1049B0005D2B00F0FB845B2B00F0FA845E2B02D1B0
:1049C000032000F0F6BC562B01D104F083FD99F8CA
:1049D0000030002B00F0028594F829306F2B40F056
:1049E000F8840EF047F8DAF800305A074BD594F8FF
:1049F0002D30144A93B13B785B070FD5019BB6F974
:104A00000610B3F89831994208DDD8F8003013F059
:104A1000010302BF3221118682F82D30D8F8003010
:104A2000D80321D594F83220064B22B993F82B20D5
:104A30000AB932221A86012384F8323023E000BFFB
:104A4000C0280020C40E0020080000208A33002067
:104A5000DE330020C8100020DC330020A41000202A
:104A6000C80F00200410002094F82B30AC4A53B13A
:104A70003B7803F0040303F0FF0123B9012382F81C
:104A80002B1082F82C30DBF800700023C8F80030BF
:104A900007F17B0607F1CB093278737816F8010C21
:104AA0009A420DD2314602F0D7FF48B116F8022CD7
:104AB000012303FA02F2D8F800301343C8F800309B
:104AC00004364E45E8D1974B1B784BB1964EDFF834
:104AD00080823368954F13F0020F40F025831DE369
:104AE00007F1CA0607F589773278737816F8010C52
:104AF0009A4222D2314602F0AFFFF0B196F804E0BC
:104B00000C21B37801FB0E41894A013B03EB4303BF
:104B100013448A6B96F803809A4281480DD08B63C8
:104B2000002390F86420CB63012303FA0EF322EAFA
:104B3000030381F8348080F864300636BE42D3D156
:104B40007C4BDFF810921F687B4B4FF0000B1B680B
:104B500002937A4B1B780393D9F80030002B00F0B6
:104B6000D48293F80080B8F1000F00F0CE82D9F81B
:104B7000042002998A1A002A0CDB01F5FA72C9F89E
:104B8000042094F86410012202FA0BF221EA0202D6
:104B900084F86420039A002A00F0B78219F8042CE4
:104BA00059780432D2B2002940F07082644931F958
:104BB0001210644AB2F8962102F1C800814201DD68
:104BC0009E7814E0C83A914202DA99784E420EE09B
:104BD00094F86420012303FA0BF322EA030384F818
:104BE0006430029B03F5FA73C9F804308DE294F83F
:104BF000643043FA0BF3D90700F18782002ECCBF53
:104C00000220012008F03EFB08F1FF32444B132A3A
:104C100000F27382DFE812F0140021002E003D0044
:104C200056005D00DD004101A501D2010A027102BA
:104C30003D004C005D00DD004101AF001301770134
:104C4000397838460E44FA2EA8BFFA2626EAE676C8
:104C50003E7002F0E7FE012019E0797838460E44F4
:104C6000642EA8BF642626EAE6767E7002F0DAFE9D
:104C700002200CE0F97838460E44642EA8BF642662
:104C800026EAE676FE70996E02F084FE0320314635
:104C9000C0E179790D2031446429A8BF642121EA5B
:104CA000E171797108F050FAB8F10D0F00F025822A
:104CB00039790E2031446429A8BF642121EAE171C9
:104CC0003971A7E1B9790520314481F30801B9713F
:104CD000A0E1DB6E1A78022A3ED1304604930EF032
:104CE00023FE19490EF028FF049B596A05930EF024
:104CF00067FD002104900FF009F8059B48B9049A5C
:104D0000124910460FF020F8049A059B10B10F4A83
:104D100000E000225A620F20114608F001FA26E056
:104D2000C40E0020E9330020C80F00208C110020A1
:104D3000C49D01082C100020C02800208A330020C8
:104D4000D8280020FC280020000020410000C84294
:104D5000C8100020FC0E002099780F203144C8298B
:104D6000A8BFC82121EAE171997008F0EDF9B8F106
:104D70000F0F00F0C281A94BD3F86C8098F8003077
:104D8000022B1AD130460EF0CFFDA5490EF0D4FE0D
:104D9000D8F820100EF014FD002106460EF0B6FFE4
:104DA00030B930469F490EF0CFFF10B19D4E00E064
:104DB0000026C8F82060122058E198F8011012204F
:104DC0003144C829A8BFC82121EAE17188F801103F
:104DD00020E1DB6E1A78022A22D1304604930EF0CD
:104DE000A3FD90490EF0A8FE049B196B05930EF0ED
:104DF000E7FC002104900EF089FF059B48B9049A56
:104E0000884910460EF0A0FF049A059B10B1854A10
:104E100000E000221A631020114608F081F90AE030
:104E2000197B10203144C829A8BFC82121EAE171AB
:104E3000197308F089F9B8F1100F00F05E81774B13
:104E4000D3F86C8098F80030022B1AD130460EF05F
:104E50006BFD74490EF070FED8F82C100EF0B0FC0B
:104E6000002106460EF052FF30B930466D490EF073
:104E70006BFF10B16B4E00E00026C8F82C601320C9
:104E8000F4E098F80B1013203144C829A8BFC821BA
:104E900021EAE17188F80B10BCE0DB6E1A78022A77
:104EA00022D1304604930EF03FFD5F490EF044FEE0
:104EB000049BD96B05930EF083FC002104900EF047
:104EC00025FF059B48B9049A564910460EF03CFF51
:104ED000049A059B10B1534A00E00022DA631120C6
:104EE000114608F01DF90AE0997D11203144C829C6
:104EF000A8BFC82121EAE171997508F025F9B8F138
:104F0000110F00F0FA80454BD3F86C8098F8003010
:104F1000022B1AD130460EF007FD43490EF00CFE6D
:104F2000D8F838100EF04CFC002106460EF0EEFECC
:104F300030B930463B490EF007FF10B1394E00E062
:104F40000026C8F83860142090E098F81510142056
:104F50003144C829A8BFC82121EAE17188F8151099
:104F600058E0D3F86C8098F80030022B1AD1304604
:104F70000EF0DAFC2A490EF0DFFDD8F828100EF00A
:104F80001FFC002106460EF0C1FE30B9304625490F
:104F90000EF0DAFE10B1234E00E00026C8F82860BB
:104FA000092063E098F8031009203144C829A8BFFC
:104FB000C82121EAE17188F803102BE0D3F86C8056
:104FC00098F80030022B1AD130460EF0ADFC15498E
:104FD0000EF0B2FDD8F834100EF0F2FB00210646B8
:104FE0000EF094FE30B930460E490EF0ADFE10B111
:104FF0000C4E00E00026C8F834600A2036E098F82D
:105000000D100A203144C829A8BFC82121EAE17146
:1050100088F80D1008F098F86FE000BFC40E00206B
:10502000000020410000C84200007A44D3F86C80A0
:1050300098F80030022B1DD130460EF075FCB149B6
:105040000EF07AFDD8F840100EF0BAFB00210646AB
:105050000EF05CFE30B93046AB490EF075FE10B173
:10506000A94E00E00026C8F840600B20314608F049
:1050700057F842E098F817100B203144C829A8BF10
:10508000C82121EAE17188F81710C3E7012934D15A
:1050900098789E4B33F91230B3F5617F05DB40F60B
:1050A00033029342A8BF134601E04FF46173B8F195
:1050B0000C0F22D14FF4966292FBF0F0A3F56173CE
:1050C00093FBF0F3924ADEB21378B34215D0042E6C
:1050D00034BF334602231370019A08FB03238D4A21
:1050E00003F2AA7313600CF063FE4046314608F0E9
:1050F0002BF8701CC0B208F0C5F894F864200123A6
:1051000003FA0BF3134384F864300BF1010BBBF18A
:10511000040F09F10C097FF41FADD7E4DAF8003071
:10512000DA050FD56B796BB1D8F800309B0709D53C
:105130003B8813F001050AD10EF008FB012003F0B3
:1051400023FF04E0012003F00EFF012300E0002311
:10515000326855070CD55BB1012003F004FF3B8892
:10516000980708D40EF0F2FA022003F00DFF02E0D7
:10517000022003F0F8FE3B88674A13F0030F4FF05C
:10518000100114BF51611161D8F8002012F00A0F0C
:1051900023D03268D10609D55A070AD4042003F077
:1051A000F3FE5E4B1B88A4F8703002E0042003F08D
:1051B000DAFE33689B0606D53B885D0606D44020A0
:1051C00003F0E2FE02E0402003F0CDFE3368580613
:1051D00042BF524B1B88A4F87230D8F800309906B1
:1051E00008D433681A0540F1A9804FF4807003F0A9
:1051F000CBFEA7E04A4B1B789B074DD5494B1B784C
:10520000042B49D9336813F400780ED03B88DD06AF
:1052100036D4102003F0B8FE202003F0A4FE42484C
:10522000011D07F015FB022326E03D8805F010055F
:10523000ADB22DB1102003F096FE012584F87480E4
:105240003368580511D5A36F38495A89B1F9003030
:10525000002BB8BF5B42934207DAB1F90230002B52
:10526000B8BF5B429342C0F211813B88990608D5D2
:10527000202003F078FE002384F87430012500E03C
:10528000002594F87C30B3B90E2007F0D5FF284BE9
:10529000012283F87C200EE03B8803F03003002BD2
:1052A0009FD0102003F05FFE202003F05CFE00235F
:1052B00084F8743001E0002D93D0002005461D4B8A
:1052C000002423F815401C4B1A1D03F10A0122F893
:1052D00015400022425001444C608A6023F815407A
:1052E00003F132015A334250C250014403444C602E
:1052F0008A605C609A601430002D7FF472AF0125E3
:10530000DDE700BF00007A440000C842D828002032
:10531000C02600202C100020000C0140A41000200A
:10532000CC100020D210002034100020AC1000203F
:10533000C40E0020E0330020420F00204FF48070A4
:1053400003F011FE5D4B5A791C46082A01D00E2A43
:1053500002D1402003F007FEDAF800305A0540F190
:10536000AA8094F8103223B9554B1B7813F0040F20
:1053700002E0336813F4002F0BD0524B00221A7056
:105380003C2006F011FB002800F095800BF038FD62
:10539000F6E702F013FD09B0BDE8F04F05F0DBBD04
:1053A0000120FFF768B90320FFF765B9012000E08D
:1053B00002205FFA80F9019A09F1FF3382F8A837D9
:1053C00003F024FE03F0C4FE484607F05BFFFFF73E
:1053D0000ABB029A12B17E2B3FF403AB94F829303A
:1053E000972B05D1384B4FF4C872DA85FFF7FBBA1B
:1053F000A72B06D1354A137843F004031370FFF747
:10540000F2BA0022BB2B079201D1022303E0B72B93
:1054100004D14FF6FE73ADF81E3009E0BE2B01D16A
:10542000022303E0BD2B1AD14FF6FE73ADF81C30FA
:10543000DBF80020BDF81C10B2F858300B44A2F87D
:105440005830BDF81E10B2F85A300B44A2F85A304A
:1054500004F040F8002384F82A30FFF7C4BA792B0F
:1054600004D11B4AD37823F0010306E07A2B7FF4A2
:10547000BAAA174AD37843F00103D370FFF7B3BA3F
:10548000013301469BB20220FFF7F5B83B889B062B
:105490003FF5F7AE202003F077FD0E4B0E481A685B
:1054A0005B68011D4360026007F0D2F9064B0125DD
:1054B00083F87450E5E609B0BDE8F08FFC280020C1
:1054C000E5330020E4180020C40E0020CC1000209A
:1054D000E8230020D41000203C1000202DE9F047E4
:1054E0004B28A0B0044600F0498600F2B480302872
:1054F00000F0D48651D8222800F0958423D80328C0
:1055000000F0608114D8012800F05081022840F09A
:10551000308704200BF0E0FC43200BF0AEFC4C2065
:105520000BF0ABFC46200BF0A8FC4C2000F05BBE5F
:10553000042800F05181052840F01B871A200BF049
:10554000CBFC00245BE1282800F0E68515D8242850
:1055500000F0CD85262840F00C87B54C06200BF0D6
:10556000BBFCB4F85C010BF0BAFCB4F85E010BF0C4
:10557000B6FCB4F8600100F0B7BD2C2800F0DF8560
:105580002E2800F05B862A2840F0F38601200BF0DD
:10559000A3FCA74B587900F026BE3D2800F0F3820B
:1055A0001ED8362800F030860BD8322800F0158639
:1055B000342840F0DE8648200BF08EFC002500F0F9
:1055C00054BC3A2800F0B3823B2800F025843828E8
:1055D00040F0CF8604200BF07FFC954C00F08DBD91
:1055E000452800F0B38627D8402800F0FF854228E0
:1055F00040F0BF868E4C10200BF06EFC60790BF0F3
:105600003CFCA0680BF074FC94F890010BF035FCA6
:10561000B4F85C010BF063FCB4F85E010BF05FFCC6
:10562000B4F860010BF05BFCB4F880010BF057FCA0
:10563000B4F8820100F058BD472800F06586C0F03C
:105640005286492840F0958602200BF045FC784BA5
:10565000988900F049BD702800F0E88258D8692880
:1056600000F045822AD8652800F0FE8015D84D2824
:1056700000F09385642840F07C8607200BF02CFC1A
:10568000E7200BF0FAFB6A4B58790BF0F6FB002091
:105690000BF0F3FB042000F068BE672800F0AA813D
:1056A00000F2188212200BF017FC624B00241B88BA
:1056B000B3F5806F8CBF082501257EE16C2800F0D2
:1056C000298217D86A2800F095846B2840F051860B
:1056D00005200BF001FC584B18880BF000FC574BD1
:1056E00018880BF0FCFB564B93F86E0000F001009D
:1056F00000F079BD6E28524D00F0208200F26E82DB
:1057000006200BF0E9FBE86D0BF0F2FB4D4B0CE2D1
:10571000782800F07C8119D8742800F0C7830BD852
:10572000722800F02784732840F0238608200BF0AD
:10573000D3FB012400F057BC762800F07B8400F2F4
:10574000F9832F200BF0C8FB3F4C5DE3A42800F049
:10575000978414D87B2800F0FD82A02840F00986A9
:105760000C200BF0B9FB394B18680BF0C1FB384B20
:1057700018680BF0BDFB374B186800F0F6BDF12838
:1057800000F08181FE2800F0A284F02840F0F1852D
:105790002B4C04200BF0A0FB236CB3F85A000BF049
:1057A0009EFB236CB3F8580000F09EBC03200BF066
:1057B00093FB00200BF061FB20460BF05EFB0A2000
:1057C00000F011BD0BF088FB01200BF056FB092007
:1057D0000BF053FB00F052BC06200BF07DFB412088
:1057E0000BF04BFB46200BF048FB4E200BF045FB2B
:1057F00041200BF042FB184B187800F075BC174B9A
:10580000185D01340BF039FB0B2CF8D10024144B3C
:10581000185D01340BF031FB082CF8D10024114B3A
:10582000185D01340BF029FB072CF8D100F09FBD67
:10583000FC2800201C0000204611002048110020F8
:10584000C40F00209C100020FF9D0108E8F7FF1FF7
:10585000ECF7FF1FF0F7FF1FE733002060BC0108E3
:105860006CBC010841BC0108CC4C0B200BF034FB94
:1058700020880BF034FB608880B20BF030FBC84B03
:105880001B68C3F3C000C3F38002800040EA4200FB
:10589000C3F340021043C3F3401240EAC20003F0D6
:1058A000100318430BF01BFBBE4B1A88636812F001
:1058B000010F14BF4FF0020C4FF0000C12F0020F5A
:1058C00002F0080814BF4FF0040E4FF0000E03F46E
:1058D000475912F0040F14BF1027002749EA08099E
:1058E00012F0400F03F4804814BF2026002649EA36
:1058F000080912F0100F03F4004814BF4FF40075AC
:10590000002549EA080912F0200F03F4803814BF7B
:105910004FF48060002049EA080912F4807F03F404
:10592000003814BF4FF40061002149EA080912F45D
:10593000007F03F480289C4A49EA080903F4002800
:1059400049EA0809127803F4801849EA080903F0C3
:10595000007349EA0303C2F3800243EA020343EA05
:105960000C0343EA0E0E4EEA070746EA070645EA2D
:10597000060540EA050041EA00014FF00000034639
:1059800014BF4FF400184FF0000841EA0808217ACC
:105990008B420BD2854A9C5C012202FA04F414EA81
:1059A000080F1CBF9A4010430133F1E70BF0A0FA37
:1059B0007F4B93F8A80700F016BC7E4B33F9140018
:1059C000013490FBF5F080B20BF089FA032CF4D18E
:1059D000724CA08C0BF083FAE08C0BF080FA208DD7
:1059E0000BF07DFA608D0BF07AFAA08D0BF077FA50
:1059F000E08D79E310200BF06FFA00246E4B185DF8
:105A000001340BF03AFA102CF8D100F0B0BC702041
:105A10000BF062FA00260E247443604D01362B6CA5
:105A20002344B3F819010BF05AFA2B6C2344B3F852
:105A30001B010BF054FA2B6C2344B3F81D010BF03F
:105A40004EFA2B6C234493F81F010BF016FA2B6CC3
:105A5000234493F820010BF010FA2B6C234493F8A5
:105A600021010BF00AFA2B6C234493F822010BF06E
:105A700004FA2B6C1C44D4F823010BF039FA082EDD
:105A8000C9D100F074BC70200BF026FA484C04F128
:105A9000700594F8D4000BF0F0F994F8D5000BF0F1
:105AA000ECF994F8D6000BF0E8F994F8D7000BF075
:105AB000E4F994F8D8000BF0E0F994F8D9000BF071
:105AC000DCF9073494F8D3000BF0D7F9AC42E0D1FD
:105AD00000F04DBC10200BF0FFF90024374B185D8F
:105AE00001340BF0CAF9102CF8D100F040BC344D51
:105AF00000242878400000F0FE000BF0EDF92B7830
:105B00009C4280F034842F4B33F814000BF0E7F9FB
:105B10000134F4E72C4C06200BF0DEF920880BF062
:105B2000DEF960880BF0DBF9284B1888DCE20420F2
:105B30000BF0D2F9194B186E00F017BC07200BF0D0
:105B4000CBF9234B1888FF28A8BFFF20C0B20BF069
:105B500094F9204B186880F3100080B20BF0BFF965
:105B6000B5F864000BF0BBF9114B93F885211A4B83
:105B7000186822B10A23584380F3100001E000F3B3
:105B80000F0080B2B0E20A4C02200BF0A5F994F8A5
:105B9000D4010BF072F994F8D30124E3C40F002070
:105BA000C81000208C110020E5330020CD0F00200C
:105BB000FC28002096100020F40F00200810002080
:105BC00088330020D828002094280020A41000202A
:105BD000B8100020C4100020C01000200B200BF0D3
:105BE0007BF9AB6E002618780BF047F9AB6E58784E
:105BF0000BF043F9AB6EBE4C3344187901360BF011
:105C00003CF9032EF6D1A36ED8790BF036F9A36ECA
:105C100098780BF032F9A36ED8780BF02EF9A36EBA
:105C200058890BF05CF9A36E187ADCE2B04C1E20A8
:105C30000BF052F9236C00251B78022B77D1236CD3
:105C400005F1080253F82200AA490DF0C1FE11F037
:105C50008BFDFA28A8BFFA2020EAE070C0B20BF052
:105C60000CF9236CA44903EB8503D86A0DF0B0FE50
:105C700011F07AFDFA28A8BFFA2020EAE070C0B23D
:105C80000BF0FBF8236C05F10E0253F822009B4940
:105C90000DF09EFE11F068FD6428A8BF642020EA84
:105CA000E070C0B201350BF0E8F8032DC7D1072D25
:105CB000236C2AD1586C8F490DF08AFE11F054FDE7
:105CC000FA28A8BFFA2020EAE070C0B20BF0D5F89D
:105CD000236C8849986C0DF07BFE11F045FDFA2885
:105CE000A8BFFA2020EAE070C0B20BF0C6F8236C1F
:105CF00093F84C000DF014FE11F036FDFA28A8BF01
:105D0000FA2020EAE070C0B20BE02B4458780BF088
:105D1000B4F8236C2B44D87A0BF0AFF8236C2B44E7
:105D2000587D01350BF0A9F80A2DC0D11FE3236C73
:105D30002B4458780BF0A1F8236C2B44D87A0BF045
:105D40009CF8236C2B44587D01350BF096F80A2DF6
:105D5000EDD10CE33C200BF0BFF80024644D04F1BE
:105D600008022B6C654953F822000DF031FE11F04A
:105D7000FBFC80B20BF0B3F82B6C604903EB84039F
:105D8000D86A0DF025FE11F0EFFC80B20BF0A7F8F9
:105D90002B6C04F10E0253F8220058490DF018FE46
:105DA00011F0E2FC013480B20BF099F8032CD5D14C
:105DB000072C2B6C16D1586C50490DF009FE11F0D0
:105DC000D3FC80B20BF08BF82B6C4C49986C0DF027
:105DD000FFFD11F0C9FC80B20BF081F82B6C93F839
:105DE0004C000BE0234458780BF079F82B6C2344DB
:105DF000D87A0BF074F82B6C2344587D01340BF0E7
:105E00006EF80A2CD4D1B2E214F8010F002800F089
:105E1000AE820BF032F8F7E701200BF05DF8344B5F
:105E20001B6C1878DFE150200BF056F80025304B42
:105E30000C211C6C324B04EB850494F8792001355D
:105E400001FB023393F838000BF017F894F87A004E
:105E50000BF013F894F87B000BF00FF894F87C002B
:105E60000BF00BF8142DE2D181E2214B1C6C0623C0
:105E700003FB054494F8CE000AF0FFFF94F8C90034
:105E80000AF0FBFF94F8CA000AF0F7FF94F8CB0081
:105E90000AF0F3FF94F8CC000AF0EFFF013594F814
:105EA000CD000AF0EAFF0C2DDFD160E24FF00008D0
:105EB000012600270E4B1A7A974232DA0933FA5C30
:105EC00000240C2363430E4D05F13001595C9142CF
:105ED00007D12B44586B11F07EFA82462EB9B14699
:105EE00010E001341B2CECD119E0804417E000BF16
:105EF000C40F0020000020410000C84200007A4486
:105F0000009E0108D1450ADA0C2303FB04535B6BA6
:105F100013F809000AF0B1FF09F10109F2E70137AE
:105F2000C8E7002E00F023825FFA88F00AF0D4FF61
:105F30000026BEE7CC4D0024287A0AF0CDFF2B7A4C
:105F40009C4280F01482C94B0021E65C0C2202FBCB
:105F500001F3C74800F13007DA5DB24205D10344CE
:105F600093F838000AF089FF02E001311B29EDD1D6
:105F70000134E4E7BF4C16200AF0AEFFB4F89601F6
:105F80000AF0ADFFB4F844010AF0A9FFB4F84601E5
:105F90000AF0A5FFB4F848010AF0A1FFB4F8D00157
:105FA0000AF09DFF94F8E1010AF067FF00200AF073
:105FB00064FF94F8E2010AF060FF94F885010AF0AA
:105FC0005CFF94F892010AF058FF00200AF055FF98
:105FD000A54B0A201B6CB3F9563093FBF0F080B24E
:105FE0000AF07DFF89E0E0B201340AF046FF092C97
:105FF000F9D1BCE110200AF06FFF9F4B9F4C18783D
:1060000000F002000AF039FF9D4B18780AF035FFC6
:1060100020680AF06DFF60680AF06AFF994B1888E3
:106020000AF05DFF984B18880AF059FF8E4BB3F8C1
:106030006C0059E00AF004FF074612200AF04CFFFA
:10604000894C17B9266F656F05E0102F19BF002521
:106050002E46A66FE56F38460AF00FFF30460AF06D
:1060600047FF28460AF044FFD4F880000AF040FFBA
:1060700000200AF034FF00200AF031FF0020B2E0D7
:10608000794D002495F884002E4680000130C0B27E
:106090000AF022FF95F884000AF0EFFE96F88430AB
:1060A0009C4280F06481794D285D0AF0E6FE05F19E
:1060B0001003185D0AF0E1FE05F12003185D30358C
:1060C0000AF0DBFE285D0AF0D8FE0134E6E708207E
:1060D0000AF002FF00200AF002FF00200AF0FFFE93
:1060E00000200AF0FCFE00200AF0F9FE3FE1042047
:1060F0000AF0F2FE5F4B986837E194F87A010AF0F3
:10610000BCFE94F87E010AF0B8FE94F87D010AF016
:10611000B4FE94F87F0166E0564C07200AF0DCFEDE
:10612000B4F880010AF0DBFEB4F882010AF0D7FE71
:1061300094F884010AF0A1FEB4F88601D4E74D4C2E
:106140000C200AF0C9FE94F890010AF096FEB4F80B
:106150009A010AF0C4FEB4F896010AF0C0FEB4F841
:1061600098010AF0BCFE94F891010AF086FEB4F89A
:106170009C010AF0B4FEB4F89E01B5E73D4C042042
:106180000AF0AAFE94F8CE010AF077FE94F8CF0147
:106190000AF073FEB4F8D001A6E73D4C3D4D2078DF
:1061A0000426043800EB4000C0B20AF095FE2378C4
:1061B00002359E4280F0DB8015F8020C0AF05DFE8D
:1061C00015F8010C013600EB800000EB800000F2B6
:1061D000EE2080B20AF083FEE9E701200AF07CFE9F
:1061E000244B93F892010AF048FEC0E008200AF020
:1061F00073FE00241F4B234493F8880101340AF0F6
:106200003CFE082CF6D1B2E0174B1A4C93F8C500AF
:1062100004F12805C0EBC000C0B20AF05DFE94F89E
:10622000E80100231C4AD25C904200F0A4800C33A9
:106230003C2BF7D10834AC42F1D198E040200AF071
:106240004BFE0C4C04F14005B4F8A0020AF047FEE6
:1062500094F8A2020AF011FE043494F89F020AF0A6
:106260000CFEAC42F0D182E0C40F0020CD0F002024
:10627000009E0108FC280020CC100020D410002033
:10628000D2100020D0100020CE1000204910002095
:10629000883300209C2A0020EC180020E0200AF01F
:1062A0001BFE424C04F18005B4F82202043400F0D5
:1062B0003F000AF014FEB4F81E02C0F386100AF084
:1062C0000EFE94F81C0200090AF0D7FD94F81C0297
:1062D00000F00F000AF0D1FD94F81D020AF0CDFD88
:1062E000AC42E1D143E0324C0D200AF0F5FD08F05C
:1062F0008DFD0AF0C2FD20880AF0FAFDE0680AF080
:10630000F7FD06F0F5FB30E00AF0AEFD054684200F
:106310000AF0E2FD28460AF0EBFD254BDC6805F1AA
:106320008003A3428CBF641B802406F09BFC28469C
:106330002246694608F09EFD05460024AC4216DA66
:106340001DF804000AF099FD0134F7E713200AF064
:10635000C3FD0024174B185D01340AF08EFD0B2C91
:10636000F8D100200AF0C4FD00200AF0C1FD012090
:1063700018E0002016E00AF080FDB4F8EA010AF007
:10638000AEFD94F8EC010AF078FD94F8ED010AF006
:1063900074FD94F8EF010AF070FD94F8EE010AF034
:1063A0006CFD47E720B0BDE8F08700BFFC28002067
:1063B0000C00002060BC01082DE9F347C54C0646DF
:1063C0002378C54F002B00F0D9813A686368D31A4F
:1063D0007C2B40F2D381237A6260013323724FF029
:1063E000000808F12400BB4DC0B201F09BFC05F190
:1063F0000A0333F918000DF097FAB84B8146188854
:106400000DF092FA014648460DF096FBB4490DF0A6
:10641000DFFA0DF0A3FC08F1010800B201F070FCF6
:10642000B8F1030FDDD1302001F07CFCB5F910008C
:1064300001F066FC01F06EFC2B7A9A072CD141F238
:1064400088336A689A4218D9102001F06BFC686999
:106450004FF0640890FBF8F000B201F051FC2120ED
:1064600001F060FC686990FBF8F308FB130000285A
:10647000B8BF404200B201F043FC142001F052FCCE
:10648000B4F9180001F03CFC1C2001F04BFC00208A
:1064900001F036FC01F03EFC237ADFF838825B071E
:1064A00040F04981022001F03DFCD8F81C00642333
:1064B000323090FBF3F000B201F022FCB8F9265024
:1064C0004FF0050A95FBFAF5032001F02BFC854BF4
:1064D000ADB21B78DFF8209213F0040F0BD03046DA
:1064E0000CF0AFFA28B9D9F8003013F0100F18BF2C
:1064F000002528B205E0D8F828309889B0FBFAF0DA
:1065000000B201F0FDFBD9F800309E0765D5DFF839
:10651000EC91A28D99F800304FF0640808FB02322C
:106520005B00B2FBF3F3E68D06203601B6B246EA15
:106530000326B6B2C3F303231E4301F0F3FB30B2CC
:1065400001F0DEFBE38D99F8001001339BB293FB61
:10655000F1F201FB1233E385236B5E4D9B7B012B34
:1065600005D1392001F0DEFBB5F92C0019E0AD8D25
:106570006E235D43152695FBF6F53A20AEB201F089
:10658000D1FBB6FBF8F528B208FB156501F0B8FBA6
:106590003B2001F0C7FBA8B2451D0A2095FBF0F097
:1065A00000B201F0ADFB282001F0BCFB636B0A20B8
:1065B00093FBF0F000B201F0A3FB042001F0B2FB6A
:1065C000A36A9B8913B10AF083FA03E0414B986BED
:1065D00080F3100000B201F093FBE36B3D4E9D068B
:1065E00040F19F8096F8403098071DD5112001F0AA
:1065F00099FBB6F842004FF4F36568433A4B90FBC1
:10660000F3F000B201F07CFB192001F08BFBB6F82F
:1066100042004543642095FBF0F595FBF0F300FB49
:10662000135000B201F06CFB94F84030B4F84450C1
:1066300013F0020F08BF0025012001F073FB28B200
:1066400001F05EFB092001F06DFB002001F058FB1A
:10665000264B94F846501A88B2F5967F0AD91D4BFE
:106660001B7A03F00F03072B04D842F20F759542F3
:1066700028BF1546052001F055FB236B5B7B0BB94A
:1066800028B216E0A5F120000DF04EF918490DF0E2
:1066900053FA002105460DF039FB10B94FF07C513B
:1066A00001E04FF03F4128460DF08AF80DF056FB0F
:1066B00000B201F025FB94F84020064B910703D46B
:1066C00093F84720012A1BD1012384F84730094859
:1066D0002DE000BF8C100020C02800201C000020EE
:1066E00000007A44E5330020A08601004E0000201F
:1066F0006666E63FD41000209C2800204D00002054
:106700001D6BAF4968680DF063F90DF027FBAC49CC
:106710000090A8680DF05CF90DF020FB0190684630
:1067200005E0A84A92E803008DE80300684601F0FE
:1067300009FB01F0EFFA237A282B1FD1A24B00228C
:106740001A723B684FF47A70B3FBF0F83C261720BE
:1067500001F0E8FAB8FBF6F5B5FBF6F006FB1050D1
:10676000000200B201F0CCFA182001F0DBFA06FBBF
:10677000158000B201F0C4FA01F0CCFA94F8503060
:10678000914D002B00F0408106F0F2FC6B6D8F4ABA
:10679000C31A9342064640F2C280002385F85A305D
:1067A00085F85C30AB8DDAB21B0A85F8762085F867
:1067B000773085F86C2085F86D30D5F884203B68FB
:1067C0009A1AD5F88830D97B4FF47A734B439A42A2
:1067D0000ED37F4B1B68C5F8843095F88C30013B95
:1067E000012B9FBF102385F85A30022385F85C30B7
:1067F000626B0A20A36B92FBF0F293FBF0F384F838
:106800007420121284F8752084F8783094F84020AF
:106810001B1284F8793094F8463092076A4984F85C
:10682000A73003D42D2381F8A83077E0D4F848901E
:106830006848DFF8ACC199FBF0FA0CFB0A924FF004
:10684000060E042B0EFB02F28CBF3323322381F899
:10685000A830614BE76C92FBF3F197FBF0F003FB80
:106860001122642592FBF5F20CFB007C0EFB0CFE62
:1068700084F89920121284F89A209EFBF3F203FB0D
:1068800012E393FBF5F30AEB8A0A4FFA81F80AEB5D
:106890008A0A08EB8A0189B284F8971000EB80001D
:1068A000090A84F8981000EB800051B201EB8002D5
:1068B00092B284F89C20120A84F89D2084F89E30BD
:1068C000B4F842201B1284F89F302423534393FBD7
:1068D000F5F5B4F8BA300A2284F8A0301B0A84F81F
:1068E000A130B4F844304FEAD979B3FBF2F303F5A1
:1068F000FA739BB284F8A2301B0A84F8A330B4F870
:10690000BC30FF0F84F89450C5F3072584F89690A7
:1069100084F89B7084F8955084F8A930666594F8E3
:10692000BE80294DB8F1000F0DD1D5F8C40006F096
:1069300015FD012807D90228284F00F0388201F000
:10694000D1F90123BB70D4F8C8001F4D00285BD0DB
:1069500095F8BE703FB140F6B732D5F8D030F31A93
:1069600093420BD850E00123D5F8C400022185F8EA
:10697000BE3006F0E7FC85F8D47043E095F8CC30E3
:106980005BB9D5F8C4000121C5F8C83085F8BE3020
:1069900006F0D8FC01F0A6F934E0013BDBB285F843
:1069A000CC3095F8D41095F8D520DBB94B1C0132CA
:1069B00085F8D43085F8D520D5F8C40020E000BF94
:1069C0008096184B809F01088C1000203F0D03001B
:1069D000C02800208096980040420F001C00002034
:1069E000806967FF034613F8017B01327818394646
:1069F00085F8D400D5F8C400C5F8C83085F8D5208E
:106A000006F0AFFCC4F8D06094F8D6309C4DF3B1DA
:106A1000D5F8D830DBB1D5F8DC30C3B1C5F8E030FB
:106A20001B68984AC5F8E430D5F8E8301344187A62
:106A3000FEF754FDD5F8E03098790AF01EFAD5F843
:106A4000E8300133092B88BF0023C5F8E8308E4DAC
:106A500094F8EC202E688A4B002A00F0E281D3F8EB
:106A6000F020002A00F0DD8193F8F430013B012B87
:106A700000F2D781D4F8F000814F06F06FFCE0B14E
:106A8000D7F8F00006F067FC97F8F53080467E2BCB
:106A9000D5F800900ED102231B2887F8F43009D1D5
:106AA000D7F8F00006F05AFC20B90123C7F8F89097
:106AB00087F8FC3084F8F580DCE7D7F8F8202B68FD
:106AC0009B1A41F6583293421DD9032387F8F430BC
:106AD000A7E16E4A32F8130010B903464FF4036081
:106AE0000133B0F5C06FDBB275D01DD9B0F5006FC2
:106AF0007AD031D9B0F5036F3ED184F8FD30E36B25
:106B00005F4F99063FD494F8FC1094F8FD300029AB
:106B100000F04A812A68921B012ADAD984F8FD30F4
:106B2000002384F8FC307CE1B0F5007F42D007D828
:106B3000B0F5807F47D0B0F5887F00F08380E6E72E
:106B4000B0F5806F00F0A680B0F5826F00F0EB80AA
:106B5000B0F5047FDBD123E0B0F5E26F00F0828076
:106B6000B0F5E46F00F08380B0F5E06FCFD184F82A
:106B7000FD30B4F90A107EE0B0F5046F6BD0B0F5CB
:106B8000026FC4D1FAE097F840309A07BBD5B7F846
:106B9000421024234B436421123393FBF1F1FDE0B7
:106BA00084F8FD303A4B364F1B689B07ABD5BB8D45
:106BB0000A21F2E084F8FD30354B314F1B6819058E
:106BC000A1D5796BEAE084F8FD30E36B2C4F5A07CE
:106BD00099D57969E2E084F8FD302D4B284F1B6888
:106BE0001B0590D5B96BD9E0E16B254A8F0684F877
:106BF000FD3088D592F84010880784D5D90710D584
:106C0000D36C192283EAE371A1EBE37101EB51012B
:106C1000B1FBF2F1002BACBF41F0004141F040412B
:106C20000DE0936C192283EAE371A1EBE37101EBB0
:106C30005101B1FBF2F1002BB8BF41F080414FF49C
:106C400000608AE084F8FD30E36B0D4F5B077FF551
:106C50005AAF3969A2E084F8FD30B4F918306421E4
:106C600059437AE084F8FD30B4F90C1003E0B4F92C
:106C70000E1084F8FD302C2391FBF3F16DE000BF82
:106C80008C100020809F0108C028002030C101081E
:106C90009C28002084F8FD3094F8FE30624A0133CD
:106CA000DBB2032B88BF012382F8FE3042F210735F
:106CB00094F8FE1059435D4B1B78D80748BF01314B
:106CC0009A0748BF02315F07B4F8003148BF04316A
:106CD000D80748BF0A319A0748BF14311F0648BF7A
:106CE0002831D80548BF28315A0748BF64311F07EB
:106CF00048BFC831980548BF01F5C8719A0648BF1A
:106D000001F57A71DF0648BF01F5FA61580648BF00
:106D100001F57A614FF4806000F0B0FF424B002231
:106D200083F8FC20EFE6E16BDFF8FC8011F0200730
:106D300084F8FD3017D098F8402012F0020F14BFED
:106D40004FF47A71002112F0010F14BF4FF4FA636F
:106D500000230B4494F84610194400F08FFF0023E1
:106D600084F8FC30CFE6324B1B6819067FF5CBAEBA
:106D7000394600F083FF88F8FC70C4E684F8FD30E3
:106D8000E36B294F9A067FF5BEAE97F840309B071C
:106D90007FF5B9AEB7F844306421594300F06EFF77
:106DA000002387F8FC30AEE684F8FD3039E0BB788C
:106DB00023B1C5F8C06087F80280C4E5D5F8C030BB
:106DC000F31AB3F57A6FFFF4BEAD0123D5F8C40012
:106DD000BB7006F0C0FA0746D5F8C40006F0BBFA4F
:106DE0007F067FF4B0AD8A2802D08E280CD0AAE5A9
:106DF000EB6B98067FF5A7AD95F8BE30002B7FF4BE
:106E0000A2AD05F18D0306E095F8BE30002B7FF4AE
:106E10009AAD05F15803C5F8C8302D2385F8CC305C
:106E200091E502B0BDE8F0878C100020E53300202A
:106E30009C280020F8B504460E461746002520463B
:106E4000202110F0BAFA0446D0B10134204610F0E7
:106E500017FBB0F5617F05DB40F634039842A8BF0D
:106E6000184601E04FF46170A0F56170192390FBA2
:106E7000F3F00DB9307000E070703B7801333B7077
:106E80000DB90125DBE72046F8BD7FB5047806463D
:106E9000E4B9364B1921186800EB840090F87B5058
:106EA00090F879204D4305F5617590F87A3000959A
:106EB00090F87C00414301F5617101912C48214615
:106EC000013401F0DDFE142CE3D14CE010F0D8FACF
:106ED0001328054641DC254B701C1C68202100232B
:106EE0008DF80F3010F069FA1E35064670B1013684
:106EF000304610F0C5FA19289FBF04EB850358707F
:106F00009DF80F30013398BF8DF80F3030462021A7
:106F100010F053FA064670B10136304610F0B0FA60
:106F20000D289FBF04EB850398709DF80F30013347
:106F300098BF8DF80F3004EB85043046E11C0DF14D
:106F40000F02FFF777FF9DF80F30042B0BD0601C6A
:106F50000021042210F0FBF905E006480649002252
:106F6000132301F08DFE04B070BD00BF041000209B
:106F700020C2010835C2010854C2010801480AF0C4
:106F80002FB800BF5AC201082DE9F04304788FB032
:106F90000546002C59D17B4B0021142209A807AECD
:106FA000D3F8008010F0D3F907223046002110F00A
:106FB000CEF900231A46A70005A8059308EB07059C
:106FC00083807149B5F802E031F813C01CEA0E0F56
:106FD0000AD00E310DF1380C595C02F1010E6244F9
:106FE00002F81C1C5FFA8EF20133072BE9D1002155
:106FF0000B46664AB5F802E011F802C01CEA0E0F13
:107000000AD006320DF1380C8A5C03F1010E63449C
:1070100003F8242C5FFA8EF301310629E9D118F820
:1070200007308DE841006A785949029209A81A0987
:1070300003F00F0301F00FFE2146564809AA013460
:1070400001F01EFE202CA6D199E010F019FA1F289D
:10705000044600F3868028462021E4B210F0ADF902
:107060001F2C02D9FFF78AFF89E0464B451C1B689D
:10707000002103EB84042046042210F068F9002765
:10708000454B09AE304600210A2217F803905FFAFB
:1070900087F810F05CF9002315F8012B32B10A2BA8
:1070A00004D04A4502D0F2540133F5E74A455FD196
:1070B00008F1FF33032B09D8DFE803F01005023F86
:1070C0000DF1230134E00DF123011EE0304610F0F4
:1070D000D7F92378C0B243EA001006E0304610F03A
:1070E000CFF9237800F00F001843207031E001330E
:1070F000062B0AD0244800F11B069E5D9642F6D16D
:1071000003445A7D63881343638011F8012F02B34F
:107110000023EFE70133072B0AD01B4800F10E06CE
:107120009E5D9642F6D130F8132063881343638046
:1071300011F8012F6AB10023EFE7304610F0A0F9F3
:107140000F2804DC304610F09BF9607001E000234A
:1071500063700137052F93D101240AF055FA74B9F1
:1071600080E70E4900221F230D4801F089FD06E04B
:1071700020460021042210F0EAF80024EDE70FB0C9
:10718000BDE8F08390110020949F0108A99F010899
:1071900068C2010877C20108B59F010854C20108FE
:1071A00035C201082DE9F041047807467CB9344D19
:1071B0002146B5F8BC21B5F8BE313248013401F0A2
:1071C0005FFD042C05F10405F2D1BDE8F0812E49E4
:1071D00010F0C6F8B0B92A4B4FF47A714FF4FA6246
:1071E000A3F8BC11A3F8BE21A3F8C011A3F8C221D3
:1071F000A3F8C411A3F8C621A3F8C811A3F8CA21A3
:10720000BDE8F081384610F03BF9032805462ED83A
:107210003846202110F0D1F8044630B10134204620
:1072200010F02EF90127064600E0074620462021EF
:1072300010F0C3F810B9BDE8F0419FE6013010F03E
:107240001FF9012FF7D140F2DC53A6F2EE229A4249
:10725000F1D8A0F2EE229A42EDD88642EBDA084B42
:107260006E3503EB85039E80D880BDE8F08107482A
:10727000074900220323BDE8F04101F001BD00BF32
:10728000FC28002083C2010896C2010835C201080B
:1072900071D001082DE9FF4104780546002C34D156
:1072A0006E4809F09DFE6E4D686900210CF024FDCA
:1072B000002840F0CF8021466A4801F0E1FC68696F
:1072C000694601F063FB0146674801F0D9FCA869F3
:1072D000694601F05BFB0146634801F0D1FCE869B7
:1072E000694601F053FB01465F4801F0C9FC286A7A
:1072F000694601F04BFB013401465C4801F0C0FCDB
:107300000C2C05F11005CFD1A4E05949052210F04D
:107310006BF838B9524B002203441030C0285A6130
:10732000F8D197E028465349042210F05DF804464E
:107330002846002C3FD1202110F03FF8002800F013
:107340008980451C284610F046F807464A4B53F8FA
:1073500024601EB9494809F043FE7BE028463146C7
:10736000FAB210F041F801340028EFD13C4B002173
:10737000C2181030C02851619E46F7D1404B03EB34
:10738000C402D2F804C09846BCF1000F04D13146C3
:107390003C4801F075FC53E0002718F834309F4258
:1073A000F5DA3B010EEB0305143563440FCB0137CF
:1073B00085E80F00F1E710F063F80B28064643DC80
:1073C000284620210FF0F9FF054648B1013528462F
:1073D00001F046FA224B012403EB0613586100E04A
:1073E0000446284620210FF0E8FF054640B101354C
:1073F000284601F035FA1A4B013403EB0613986165
:10740000284620210FF0D9FF054640B10135284616
:1074100001F026FA124B013403EB0613D86128461B
:1074200020210FF0CAFF10B9FFF7A8FD12E00130CC
:1074300001F016FA0A4B032C03EB06163062F3D167
:107440001148FFF727FF05E01048114901220C23DE
:1074500001F016FC04B0BDE8F08100BF9CC2010839
:10746000FC280020B7C20108BDC20108CDCD01082B
:1074700096C20108C1C201086CA70108C6C2010872
:1074800050C10108D5C201081CC0010835C201085D
:1074900054C20108F0B5047887B0064614BB514BBE
:1074A00019201968062303FB041191F8CA5091F8BA
:1074B000CE20454305F5617591F8C930009591F8E6
:1074C000CB50C831684300F5617001900879029093
:1074D0004979454803912146013401F0D1FB0C2C38
:1074E000DDD17DE00FF0CCFF0B28044672DC3D4B74
:1074F000701C1D68202100238DF817300FF05DFFF0
:10750000064680B1013630460FF0BAFF03289FBF10
:10751000062303FB045383F8CE009DF817309CBF6D
:1075200001338DF81730304620210FF046FF074613
:1075300080B1013738460FF0A3FF0D289FBF062307
:1075400003FB045383F8C9009DF817309CBF013337
:107550008DF8173006266643A9193846CA310DF151
:107560001702FFF767FC20210FF027FF074670B1D5
:10757000013738460FF084FF14289FBF9DF817305D
:107580007619013386F8CC0098BF8DF8173038464D
:1075900020210FF012FF78B101300FF071FF0D289C
:1075A0009FBF062303FB045383F8CD009DF81730DB
:1075B0009CBF01338DF817309DF81730062B0FD084
:1075C000062202FB04500021C9300FF0C0FEFFF775
:1075D000D5FC05E00548064900220B2301F050FBCD
:1075E00007B0F0BD04100020E1C2010835C2010857
:1075F00054C20108F7B5047805464CB9204601A9E4
:107600000BF00EFA0134FFF7F5FF0E2CF6D150E027
:107610000FF036FFC6B20D2E47D8681C20210FF0A0
:10762000CCFE034650B15B780130682B07D0732B3A
:1076300001D1012704E0FFF7A1FC3AE000E00027B8
:1076400020210FF0BAFE1C4C06F1D005C8B1013064
:107650000FF016FF40F2ED2380B2984205DD40F6B0
:10766000CA039842A8BF184601E040F2EE20A0F2FB
:10767000EE20192290FBF2F004EB450304F815709C
:10768000587014F8153004EB45046278012B4FF064
:10769000190303FB02F331460CBF7322682203F285
:1076A000EE23064801F0ECFA03E005480E2101F054
:1076B000E7FA03B0F0BD00BFFC28002001C30108B9
:1076C00013C3010810B50446204605F03EFE18B964
:1076D0000A2005F074FDF7E710BD30B50949002216
:1076E0000B78094C1557854202BFFF25155503F14C
:1076F000FF3302F10C0208BFDBB23C2AF1D10B7060
:1077000030BD00BF89100020EC180020002208497D
:107710000C2303FB02135968814204D10022C26288
:107720001A725A6070470132052AF0D1704700BFC3
:10773000EC1800202DE9F743064689469DF828807D
:1077400011461A469DF82C3000250C2068431D4F29
:10775000C419C057B04202D1207A20B12BE00135C4
:10776000052DF2D127E0022E0FD005DC56B1012EF7
:1077700021D1009314480AE01E2E0DD01F2E1AD1DD
:10778000012009E00093114801E0114800934346AD
:1077900004F058FB044605E002F02AF9414604468D
:1077A00005F0D0FD4CB10C2303FB0575267185F85F
:1077B00008906C6001E0002000E0204603B0BDE8C6
:1077C000F08300BFEC180020004400400038014066
:1077D0000048004010B5084B0022196801EBC203B5
:1077E00093F90240844201D1981C10BD0132052A50
:1077F000F4D1002010BD00BFE8180020F0B50278D9
:1078000087B08AB94A4C04F1280694F8E82100238D
:10781000484950B2595681426ED00C333C2BF7D1B7
:107820000834B442F1D181E0002204920592451C53
:107830000FF026FEC4B260B2FFF7CCFF074618B1C6
:107840008DF81040012400E00446284620210FF066
:10785000B4FD054638B1013528460FF011FE01345C
:10786000ADF81200E4B20026284620210FF0A5FD55
:10787000B0B3451C28460FF003FE00222E495FFAE4
:1078800082FE51F82230834204D00132082AF5D119
:10789000002300E0734651F82320824220D1022EBB
:1078A0000FD0032E12D05A1E012ED2B204D0042AB9
:1078B00013D88DF814300EE0042A0ED88DF8153048
:1078C00009E0052B09D88DF8173004E09A1E052A27
:1078D00003D88DF816300134E4B20136042EC3D13A
:1078E000052C04D807B0BDE8F040FFF747BB04AB58
:1078F00003CB3860796019E094F8ED010E4B94F8F1
:10790000EC5153F82000B4F8EA21009094F8EF010C
:1079100053F82000019094F8EE0153F8200053F83A
:1079200025300290054801F0ABF979E707B0F0BDCA
:10793000FC280020EC180020F0A401082AC301084C
:1079400038B1438811EA030003D08B420CBF0120F9
:107950000220704730B50A4B0A491C680A79042A8C
:107960000AD81346551C04EBC303EAB29D8828428B
:10797000F5D00A71981C30BD0A71002030BD00BFDF
:10798000E818002090110020014B00221A71E1E755
:10799000901100202DE9F047877890F803C0BBB222
:1079A000C7F1640E03EB83065C42C3F178001C4D03
:1079B0005FFA8EFE7600CCF16408A4B280B2A3B266
:1079C0000FFA83F9B9F1000F04DC002B14BF3B461A
:1079D000012300E0734609FB09F25B4302FB0CF252
:1079E00092FBF3F3434403FB09F30A2293FBF2F304
:1079F00033449BB225F8023FB1F800904A880A341C
:107A0000C9EB020A1AB202FB0AF24FF47A7392FB34
:107A1000F3F3A4B24B4484422B80D0D1BDE8F0876D
:107A20009411002010B544780078002240F6C4116B
:107A300002FB02F3193B634303F6C413534343436E
:107A400093FBF1F3034921F812300132072AEDD1FB
:107A500010BD00BFAE110020104B043033F91000F0
:107A6000B0F5617F05DB40F633039842A8BF1846A6
:107A700001E04FF461700A7819235A4302F283320D
:107A8000824208DA4A78534303F283338342B4BF15
:107A90000020012070470020704700BFD828002038
:107AA00010B500F1500302788A4203D18478C2787D
:107AB000944204D304309842F5D1002010BD012037
:107AC00010BD00BF0028114AB8BF404290FBF2F33E
:107AD00030B50F4C3C2504FB030068430D4D90FB73
:107AE000F2F22D682D7B25B903EB830303EB8303AF
:107AF00001E0C3EB031302EB830304FB02020B80E0
:107B00004FF47A7392FBF3F24A8030BD809698006E
:107B1000806967FFBC100020022803D0431E584232
:107B200058417047064B1B681B7823B1054B1868FA
:107B3000C0F3C0407047044B1878C0F38000704712
:107B4000140E0020C80F0020E5330020A0F17D03B3
:107B5000012B70B504460D460A4E05D830687D21CC
:107B600005F0FFFB84F020043068214605F0F9FBA6
:107B700035B12B881C4404EB142404F0FF042C8042
:107B800070BD00BF7C11002010B50A4C5E28014674
:107B9000206805D15D2105F0E4FB20683E2105E069
:107BA0005D2903D105F0DDFB20683D21BDE81040D3
:107BB00005F0D7BBBC11002037B51A4B1A4C1B4936
:107BC0001B4A20B11B480088B0F5805F21D209888C
:107BD0001278154D9B79ADF804108DF8062001A898
:107BE000291D04228DF807300FF096FBC0B10198D3
:107BF000686053200AF022FCA0880AF051FCA079AA
:107C00000AF04EFCE0790AF04BFC0A4B00221A8085
:107C100006E0098812789B79A180A271E371E8E7F8
:107C200003B030BDB4330020BC1100208C11002003
:107C3000CC100020903200202DE9F84305460E4676
:107C40000D4B002493E88003B44213DA7B1933F917
:107C5000140008EB050333F9142009EB050333F98D
:107C6000143001341344022293FBF2F3C01A0AF0D9
:107C700026FCE9E7BDE8F883EC30002030B585B09C
:107C800004AC002524F8025D0091ADF80600214601
:107C90001020FFF75BFF9DF806002146FFF756FF17
:107CA0009DF807002146FFF751FF9DF8000021468F
:107CB000FFF74CFF9DF801002146FFF747FF9DF8B5
:107CC00002002146FFF742FF9DF803002146FFF71F
:107CD0003DFF9DF80E002946C043C0B2FFF736FFB6
:107CE00005B030BD10B5054C206805F037FB18B164
:107CF000206805F030FBF6E710BD00BF50110020F2
:107D000010B50446C0B2FFF73FFFC4F30720BDE83B
:107D1000104039E7024B5E21186805F022BB00BF16
:107D2000BC11002038B50546054C5E21206805F0E1
:107D300018FB20682946BDE8384005F012BB00BF9B
:107D4000BC11002013B5044601A90068FFF7BAFE74
:107D50001320FFF7E7FFBDF90400FFF7D1FF1B2059
:107D6000FFF7E0FFBDF90600FFF7CAFF2320FFF78A
:107D7000D9FF2368002BB4BF53204E20FFF7C0FF6C
:107D800001A96068FFF79EFE1220FFF7CBFFBDF947
:107D90000400FFF7B5FF1A20FFF7C4FFBDF9060086
:107DA000FFF7AEFF2220FFF7BDFF6368002BB4BFD3
:107DB00057204520FFF7A4FF02B010BD674B73B5F5
:107DC0001878FFF7A9FE664D04462B78834220D031
:107DD000C8B1644B1B68E3B193F900000223009320
:107DE000614B04211B6800225B78003318BF01231C
:107DF00001934FF41653FFF79DFC5C4B186040B1A4
:107E000001232B7005E0594E3068FFF77FFC34608A
:107E10002C70574B574D1878FFF77EFE2B78044691
:107E2000834218D088B1544B1B68A3B100220124AF
:107E300093F9000008214FF4964300940192FFF754
:107E400079FC4E4B186028B905E04C4E3068FFF7BE
:107E50005DFC34602C704A4B4A4D1878FFF75CFE8D
:107E60002B78044683422E4643D0002838D0464B18
:107E70001A68002A3DD0D37992F90000002B4FF008
:107E80000202424C08BF02230092002254F8233021
:107E900001921021FFF74EFC3D4B0546186040B3A0
:107EA0003C4C94F84A30022B0BD094F89620022ACE
:107EB00001D14C3405E023B1002A04F14C0418BF71
:107EC0000024354B1C6044B1204600214C220FF0A9
:107ED0003EFA0223256084F84A300123337008E01B
:107EE0002B4E306808F08CFF3068FFF70FFC3460D1
:107EF0002C702A4B2A4D1878FFF70EFE2B7804467B
:107F0000834229D000B3274B1B682BB3264A93F931
:107F100000001268032352782021002A0CBF082297
:107F20000922009301924FF461430022FFF702FC03
:107F30001E4B186080B11E4A012313702B701D4B1D
:107F40001A681D4B1A6007E0184E3068FFF7DEFB19
:107F5000174B34601C702C7002B070BD1C0E0020DA
:107F60008C100020180E0020BC100020BC11002036
:107F7000240E0020DC100020200E002050110020D4
:107F8000300E0020621100202C0E0020F0A4010809
:107F9000641100208C170020681100203C0E002086
:107FA00078110020380E0020340E00207C110020B3
:107FB00080110020C0280020841100202DE9F74303
:107FC00005F0D6F8924CA368C31A002BC0F2618367
:107FD00000F5433303F5A073A3608E4B1D78237B1C
:107FE000C5F38005EB1A18BF012325734DB1002B93
:107FF00000F04F83884B5A789A7001225A701A7099
:108000002BE0854A2BB1D37843F00203D3709378E9
:108010005370D67806F0020101F0FF0339B97E49AA
:108020008968411A002903DB06F0010300E00123FF
:1080300003F00107784917707BB1F2070DD50A7973
:1080400005230132D2B2B2FBF3F303EB8303D31A5D
:10805000724ADBB20B71D35C4B706F4EDFF8088253
:1080600033787BB3F37823F00203F3706C4B034453
:10807000AE20B36006F04DFF08B106F04FFF88F860
:108080000000002800F00583B02006F042FF4020E9
:1080900006F03FFF002006F03CFF102006F039FFFD
:1080A0004FF48067013F0020BFB206F009FF002FA8
:1080B000F8D1384606F0A1FF72785A4B53F82200E7
:1080C00006F01EFF98F80030002B00F0E282737873
:1080D000062B00F2B382DFE813F00700B1021800AC
:1080E00078006B018801ED014F49504A504B5148CF
:1080F00000F0B1FD012006F080FF4E4806F000FFC1
:10810000022006F07AFF4C48ADE14C4F3B689B07DC
:1081100035D5DFF858810A23B8F80010DFF8509100
:10812000B1FBF3F203FB121399F8001092B29BB269
:1081300000914048424900F08EFD01F005FF01200A
:1081400006F05BFF3B4806F0DBFE3E4B99F8002053
:108150001868B8F80030067902FB163164234B43E7
:10816000C17802208E1B5643B3FBF6F6F6B206F03A
:1081700044FF3146152001F0ABFE032600E0012646
:108180003B681F0540F15A822F4B30491F6864231A
:1081900097FBF3F2096803FB1273009125482C4901
:1081A00000F059FD01F0D0FE304606F026FF2148D0
:1081B00006F0A6FE08F08CFC0746701C06F01DFFBA
:1081C0001520394601F084FE38E20120214F06F0E7
:1081D00014FF214806F094FE3B6898074AD51F4AD1
:1081E0001448B2F90210B2F900300091B2F904203B
:1081F0001B4901921B4A00F02EFD01F0A5FE022052
:1082000006F0FBFE0B4806F07BFE032633E000BFC2
:10821000BC110020E5330020E823002049C30108F9
:10822000404B4C007CA401084EC3010857C3010811
:1082300041BC0108C91100205DC301089C28002031
:1082400064C30108B4100020C0100020C410002036
:108250007CC30108C810002091C3010896100020BB
:10826000A7C30108B6C30108C50A0020B810002042
:108270004D00002002263B68D9071AD57B4A7C486E
:10828000B2F90210B2F900300091B2F90420794934
:108290000192794A00F0DFFC06F1010801F054FE7A
:1082A000304606F0AAFE5FFA88F8714806F028FE0C
:1082B00046463B681A0718D5704A6D48B2F9021055
:1082C000B2F900300091B2F904206A4901926C4A77
:1082D00000F0C1FC771C01F037FE304606F08DFE41
:1082E000FFB2634806F00CFE3E46664A6149B2F9A9
:1082F0000030B2F902205E480092634ADFF8B09184
:10830000B2F90020771C0192604A00F0A4FC01F051
:108310001BFE304606F071FE554806F0F1FD54494B
:10832000D9F8000000F032FB51480FF054F8FFB2CA
:10833000C1B2092909D84B1CDBB2214420224A735F
:108340000021E21891731946F3E7DFF82481D9F888
:108350000400414400F01AFB01F0F6FD384606F037
:108360004CFE404606F0CCFD4146D9F8080000F02E
:108370000DFB40460FF02FF80236F6B2C7B2092FB8
:1083800009D87B1CDBB2274420227A730021E21833
:1083900091731F46F3E73E4BB3F900000BF0C4FAAC
:1083A00008EB070100F0F2FA01F0CEFD304657E08D
:1083B0000026384F3B78B34240F240810E2E00F049
:1083C0003D817008013006F018FE30460AF002FBCD
:1083D0003B78B34206D9202006F077FD701CC0B26E
:1083E0000AF0F8FA0236F6B2E3E72B4E2B4996F87C
:1083F000A8271F4800F02FFC012006F0FEFD1C48B6
:1084000006F07EFD264B27491F7819483A4600F0B2
:1084100022FC022006F0F1FD154806F071FD0C2348
:1084200003FB0766204996F8AB2796F8AA37104851
:1084300000F011FC01F088FD032006F0DEFD0C4881
:1084400006F05EFD96F8B01796F8AE2796F8AF37AF
:1084500007480091154900F0FEFB01F075FD04206E
:1084600006F0CBFD024806F04BFDE7E0E80F0020E8
:10847000C9110020A7C30108BAC30108EE0F0020EC
:1084800051D9010894280020A4100020BEC301087F
:10849000B423002088330020FC280020C2C3010838
:1084A000C0260020CEC30108DFC30108F0C30108C5
:1084B000A8230020784B1B681B0640F1BB80636A31
:1084C000A16A764A8B421CBF936292F82C304FF01F
:1084D00001011CBF013303F003034FF0000018BF7C
:1084E00082F82C3006F095FD94F82C306C4A00266A
:1084F000D05C06F0EAFC0220012106F08AFD694BFF
:108500003620F35C0136C3EBC30393FBF0F0C0B23B
:10851000062828BF06206038C0B206F0D6FC102E10
:10852000EDD1614B61491B78614813F0020F614B3B
:108530001A7814BF59234E2300F08DFB01F004FD7F
:10854000022006F05AFD5A4806F0DAFC5A495B4B05
:108550004E680A68564892FBF3F2594996FBF3F3CA
:1085600000F079FB01F0F0FC032006F046FD5048D6
:1085700006F0C6FC534B54491A884D4800F06BFB7B
:1085800001F0CFFC042006F038FD494806F0B8FCA5
:108590004E4B4F491A88464800F05DFB01F0C1FC84
:1085A00004210A2006F035FD414806F0A9FC49499E
:1085B000226B3F4800F04FFB474E01F0B2FC052014
:1085C00006F01BFD3A4806F09BFC7268B36843490D
:1085D000374800F040FB01F0A4FC05210A2006F01A
:1085E00018FD334806F08CFC3369F2683C49D21A16
:1085F0002F4800F030FB01F094FC062006F0FDFC53
:108600002B4806F07DFCB2683649294800F023FB70
:1086100001F087FC06210A2006F0FBFC244806F046
:108620006FFC3149152222480EF000FF01F079FC61
:10863000072015E7F37843F00203F3704DBB2B4B93
:1086400000219B791220032B97BF294A3F259B18B5
:108650001D7F06F0DEFC284606F037FC13200021C3
:1086600006F0D7FC234B1B78002B14BF522021208F
:1086700006F02BFC1420002106F0CBFC94F83450BB
:10868000074B585D013505F0030506F01EFC84F824
:10869000345003B0BDE8F0839C280020BC110020BA
:1086A00002C4010879100020CC10002007C4010882
:1086B000C9110020D2100020D4100020809698000C
:1086C00018C40108CE10002025C401083010002075
:1086D0002DC4010834C40108300200203BC4010845
:1086E00044C401084BC40108D40A0020B43300205C
:1086F0007CA401088A330020F0B50124B0FBF4F516
:108700008D4201D34C43F9E70026D4B1B0FBF4F518
:1087100004FB1500B4FBF1F41EB9002D01DC002CA4
:10872000F3D1092D03F1010EEFB204DD002A14BFCD
:108730003725572500E030253D441D70013673462E
:10874000E3E71C70F0BDF0B50124B0FBF4F58D42F9
:1087500001D34C43F9E70026D4B1B0FBF4F504FB98
:108760001500B4FBF1F41EB9002D01DC002CF3D18F
:10877000092D03F1010EEFB204DD002A14BF3725E5
:10878000572500E030253D441D7001367346E3E770
:108790001C70F0BD03685A1C0260197070472DE907
:1087A000F843089E002B074688461446334614BFFC
:1087B0004FF030094FF0200913F8012B0AB9254674
:1087C00003E0002CFBDD013CF6E7002D04DD38461C
:1087D0004946C047013DF8E7354624EAE474A01B4A
:1087E000284415F8011B11B13846C047F7E7BDE82A
:1087F000F883024B186804F0B4BD00BF780E002067
:10880000F8B507460C464868002115461E460BF091
:1088100073FA58B128460BF087F810490BF0D8F8D6
:1088200001464FF07E500BF087F96060616830467A
:108830000AF0C6FF014630460BF07EF92568064671
:10884000294638460AF0BAFF014630460BF0C0F818
:10885000014628460AF0B4FF2060F8BDDB0FC9408E
:108860002DE9F04102780346202A00F10100F9D0F9
:10887000092AF7D02D2A02D10346414D04E02B2AC4
:1088800008BF03464FF07E551C460026234614F8C9
:10889000012BA2F13007F9B209290DD83949304628
:1088A0000BF096F8064638460BF03EF80146304687
:1088B0000AF086FF0646E9E72E2A17D1314F2346F4
:1088C00014F8010B3038C2B2092A0FD80BF02CF87B
:1088D00039460BF031F9014630460AF071FF29495B
:1088E000064638460BF074F80746E8E71A7802F0B7
:1088F000DF02452A39D15A782D2A02D102330127C5
:1089000004E02B2A14BF013302330027013B00246B
:1089100013F8012F303AD1B2092903D80A2101FBFB
:108920000424F5E7B4F59A7F28BF4FF49A74A04663
:108930004FF07E53B8F1070F07D9184612490BF0D4
:1089400047F8A8F108080346F4E704F0070434B137
:1089500018460C490BF03CF8013C0346F7E7194672
:108960002FB130460BF0E8F804E04FF07E5130466E
:108970000BF02EF8014628460BF02AF8BDE8F081EE
:10898000000080BF0000204120BCBE4C30B5054631
:1089900087B00C4603A800210C220EF0D8FC284614
:1089A00000210BF0D1F920B1284628490AF008FF30
:1089B00003E0284625490AF001FF25490BF008F895
:1089C0000BF0CCF9054680EAE0706946A0EBE57053
:1089D0000AF026F8002DACBF20232D2368468DF821
:1089E0000C300EF0F8FC012807D130238DF80D3043
:1089F0008DF80E308DF80F300CE0022805D13023B1
:108A00008DF80D308DF80E3004E0032804BF3023BC
:108A10008DF80D30694603A80EF0C0FC03A80EF0D7
:108A2000DAFC0338C5B22A4603A920460EF0FEFC44
:108A300000236355204607490EF0B0FC03AB2046E7
:108A400059190EF0ABFC204607B030BD6F12033A47
:108A500000007A4484C4010870B50646B6FBF2F4FF
:108A60000846154614B12046FFF7F6FF05FB1464CF
:108A7000024B1B5D00F8013B70BD00BF86C40108BE
:108A80002DE9F04F81468A4616461C4689B00025DE
:108A90003178002900F0DB80252902D001364846D4
:108AA00074E072784FF00008302A0CBFB278B71C1F
:108AB000A2F1300312BF4FF0000BF71C4FF0010B77
:108AC000092B19D8A2F13003D9B2092905D80A22F5
:108AD00002FB083817F8012BF4E7A2F16103052B1C
:108AE00002D8A2F1570305E0A2F14103052B03D8F8
:108AF000A2F137030A2BEADD6C2A30D13A787E1CCA
:108B0000642A00F083800BD8252A3DD003D8002AA0
:108B100000F09D80BCE7582A0CD0632A19D0B7E733
:108B2000732A22D002D86E2A37D0B1E7752A5CD0DA
:108B3000782AADD1271D2068A2F1580462424FF077
:108B40001001624155E02CD9582A32D0632A2AD12B
:108B50003E4648462178271DD04701350FE0642A5C
:108B600063D00ED9732A14D13E4623684846009339
:108B7000514642460023FFF712FE271D05443C469E
:108B800086E7252ADFD13E4648462521D0470135D4
:108B90007EE70AD86E2A06D13E46236804341D605B
:108BA00076E7002A53D03E4672E7752A26D0782A07
:108BB000F9D1A2F1580304F1040C5A422068CDF80F
:108BC0000CC04FF010015A4105ABFFF795FDDDF8E1
:108BD0000CC03E46644605AB0093484651464246AB
:108BE0005B46FFF7DCFD054452E72068271D0A219C
:108BF000002205ABFFF7A7FD3C46ECE704F1040CAF
:108C0000CDF80CC020680A210022DDE72068271D6E
:108C1000002808DA2D238DF8143040420DF1150399
:108C20000A210022E6E705ABFAE7206804F1040C0C
:108C300000280ADA2D238DF8143040420DF1150377
:108C4000CDF80CC00A210022BFE705ABF8E72846A3
:108C500009B0BDE8F08F0EB40FB505AB53F8042B87
:108C60000190064901A80393FFF70AFF019B002228
:108C70001A7004B05DF804EB03B0704795870008E4
:108C80000FB413B50B4904AB08680B4953F8042B18
:108C900009680193FFF7F4FE0446084B186804F0D6
:108CA00054FB0028F9D0204602B0BDE8104004B0C3
:108CB000704700BF5409002050090020780E0020A2
:108CC00080EAE073A3EBE0738B4206DB002801DD52
:108CD000401A704702D0084470470020704770B5B2
:108CE00004460BF03BF82030402857D820462C494A
:108CF0000BF02AF828B120462A490AF05FFD044605
:108D0000F4E7204628490BF001F828B12046254910
:108D10000AF056FD0446F4E7204624490BF014F807
:108D200030B1224920460AF049FD01461F480AE0B9
:108D300020461F490AF0EAFF40B11C4920460AF0CC
:108D40003FFD01461A480AF039FD044621462046F7
:108D50000AF03EFE0546204629460AF039FE15492E
:108D6000064628460AF034FE13490AF027FD01465C
:108D700028460AF02DFE11490AF022FD0146284638
:108D80000AF026FE0E490AF019FD014630460AF0A7
:108D90001FFE014620460AF013FD70BD002070BD85
:108DA000DB0F4940DB0FC940DB0F49C0DB0FC93F78
:108DB000DB0FC9BF9A7C2E36FAAF4F393587083C96
:108DC000A4AA2A3E08B503490AF0FAFCBDE8084007
:108DD00085E700BFDB0FC93F2DE9F04F056885B07F
:108DE000814628460C46FFF7EDFF80462846FFF7F0
:108DF00076FFD9F8045006462846FFF7E3FF0746FA
:108E00002846FFF76CFFD9F8089005464846FFF75B
:108E1000D9FF82464846FFF762FF414681465046E9
:108E20000AF0D6FD4146834648460AF0D1FD514638
:108E3000019030460AF0CCFD4946029030460AF0D7
:108E4000C7FD3946039050460AF0C2FD49462060EE
:108E500007F100400AF0BCFD29466060A560029859
:108E60000AF0B6FD014601980AF0AAFC2946E06026
:108E700003980AF0ADFD014658460AF09FFC3946BA
:108E8000206106F100400AF0A3FD294660615846C2
:108E90000AF09EFD014603980AF090FC2946A06165
:108EA00001980AF095FD014602980AF089FC4146B6
:108EB000E06138460AF08CFD206205B0BDE8F08F15
:108EC0002DE9F04107688AB046688568044608467F
:108ED00001A9FFF781FF019938460AF079FD04994D
:108EE000804630460AF074FD014640460AF068FCB0
:108EF0000799804628460AF06BFD014640460AF075
:108F00005FFC0299206038460AF062FD05998046B0
:108F100030460AF05DFD014640460AF051FC0899D2
:108F2000804628460AF054FD014640460AF048FCB7
:108F30000399606038460AF04BFD069907463046B3
:108F40000AF046FD014638460AF03AFC0999064601
:108F500028460AF03DFD014630460AF031FCA0608B
:108F60000AB0BDE8F081074B10B51A881C4622EA0A
:108F700000009042188002D0012004F083F920887C
:108F800010BD00BF8C110020064B10B51A881C467E
:108F900010439042188002D0012004F073F9208819
:108FA00010BD00BF8C110020024A936823EA000024
:108FB00090607047FC28002008B5104B1A780023F9
:108FC000D9B2914207D20E49002051F82310013343
:108FD00009680880F4E7322004F0F1F8094B1B68B7
:108FE0005A0309D5084B9B685B0305D4BDE80840CC
:108FF00040F2DC5004F0E3B808BD00BFE0260020DA
:10900000E42600209C280020FC2800204B4A6823EE
:109010002DE9F341137040F2D4735380BE231371D2
:10902000EF2382F8D13700231946164682F8D2374B
:10903000F25C0133514040F2D4729342F8D13F4B7D
:109040003F4A83F8D2173F4B04275A6002F1883217
:109050005A600020013F17F0FF075ED0394B3422E1
:10906000394CDA6004F17848A8F5FC38C8F30903F4
:1090700053B100234FF4005056F80880019307F0D5
:1090800093FA0428E6D11CE04FF4302007F08CFA64
:109090000428DFD12B4D4FF430202B6943F002031D
:1090A0002B616C612B6943F040032B6107F07CFA64
:1090B00041F6FD732A69042803EA02032B61D8D024
:1090C000C8E7204D4FF400502B6943F001032B619A
:1090D0001FFA88F3238007F067FA042813D1A31C32
:1090E0000193019B4FEA1848A3F800804FF4005009
:1090F00007F05AFA41F6FE732A69042803EA0203CC
:109100002B6106D0A6E741F6FE732A6913402B6156
:10911000A0E70E4B04349C42A4D10A4A04281369E8
:1091200043F08003136102D108F066FE10B90A20F3
:1091300004F0C0F802B0BDE8F08100BFFC280020B8
:10914000230167450020024000F80108D4FF010810
:109150002DE9F04108F050FE10B90A2004F0AAF8F9
:10916000B74CB84940F2D47220460EF0E5F894F8B6
:10917000A8374FF4CC71022B84BF002384F8A837A2
:1091800094F8A827B04D01FB02F303F53870204492
:109190002344286093F8340301FB0242022803F5BC
:1091A0004C7384BF0020187192F83433A74A1370AF
:1091B0000C2202FB0343A64A03F2AA73136046F291
:1091C0000902A3681A401AB99D4A43F400539360F8
:1091D000A368DF0703D54FF40050FFF7E5FEA3684F
:1091E0005E0409D50820FFF7DFFE4FF40050FFF7BB
:1091F000DBFE0120FFF7D8FEA368180706D54FF461
:109200000050FFF7D1FE0120FFF7CEFEA3689904BE
:1092100013D54FF40040FFF7C7FE894B93F8843114
:10922000012B03D14FF40060FFF7BEFE4FF48030F6
:10923000FFF7BAFE4020FFF7B7FEA3685A0603D532
:109240004FF48030FFF7B0FEA36803F40852B2F584
:10925000085F0AD11B0508D5794B93F88431012B9F
:1092600003D14FF40060FFF79FFE94F8D221744BB6
:109270002AB193F8D62112B1002283F8D6214FF0FB
:10928000000C6746734E744B1E6004EB0C03B3F87E
:10929000EAE14FEA5E0101F077314FEA9E0303F005
:1092A0003333C1EB0E00C11A4FEADE0303F0113372
:1092B000CB1A03EB231303F00F32FF2392FBF3F3DC
:1092C0001EF00108C3EB032318BF0137A2EB030311
:1092D00018BFFFB2012B0ADD022B40F0AE80B8F1BF
:1092E000000F00F0AA801EF0BC0F00F0A6800CF169
:1092F000080CBCF1280FC8D1013F012F00F29D805E
:1093000008F056FD3022002154480EF020F8544F4A
:10931000544BD5F800801F60534B002108F17900B1
:10932000C3F80080FEF7BCFB504B80F001001870C2
:109330004F4B07F126021A604E4B07F1CC021A6020
:1093400098F8000004F036FC28684B4B00F5C57215
:109350001A6003F0C3FA494B07F18A021A60484BBE
:1093600000221A809A71474B2D6807F12A021A6071
:10937000454B05F219121A60444B05F289121A6026
:10938000434B07F108021A60424BDFF844811F602B
:10939000414B07F192021A6007F19C03C8F80030B4
:1093A0003E4BB4F866011E600AF0BAFAC8F808002D
:1093B000B4F868010AF0B4FA95F85C3008F10402D8
:1093C00088F8043095F87830C8F80C0088F8053033
:1093D00094F8D531286E88F81030314BC8F8145005
:1093E0001A60304B05F164021A602F490AF0F0FA56
:1093F00001464FF07C500AF09FFBB5F816412B4B0D
:10940000186020460AF090FA014629480AF094FBB9
:1094100028490AF0DDFA284A284B1560284A1860C6
:1094200005F168031360274A05F211151560264AF5
:109430001760264A1360BDE8F08101F0CBFD5FE7BD
:10944000FC28002000F8010804100020C02600209D
:109450002C100020842A0020F4320020F80E002076
:10946000402A00202C0F0020300F00200800002090
:1094700058020020140E00203C0F0020E40E0020B3
:10948000B4330020AC0200202C24002084040020EF
:10949000082300200C230020980300205C040020F7
:1094A00090230020D0230020DB0F4940CC23002054
:1094B000000061444C3D0F4424020020940300202E
:1094C00018020020840300208C03002020010020CB
:1094D000F411002008B5FFF799FDFFF739FEBDE84C
:1094E0000840012003F0CEBE426A806A131A584237
:1094F000584170474171704743799B070AD5436AC9
:109500008269D154436A01690133B3FBF1F201FB73
:10951000123343627047437913F001031FBFC368DE
:1095200003F1FF32C369006A1DBF181A1040C0B2B0
:1095300018467047437910B513F0010304460DD067
:10954000FFF7E9FF58B1236A6269E168D05C013333
:10955000B3FBF1F201FB1233236210BD184610BDBC
:1095600090F83B3210B57BB990F83A3290F8394216
:10957000A34209D2B0F8401201229A400A430133B3
:10958000A0F84022DBB2F3E710BD8379DB0748BFC8
:10959000B1FA81F1D0F8343148BF49095A681B89C2
:1095A00009B1136170475361704710F80A3C0133E9
:1095B000DBB20A2B84BF10F8131C054A00F80A3CE2
:1095C00082BF002322F8113000F80A3C704700BF28
:1095D000DC320020334A70B5136C9068194440F6B1
:1095E0008C23081A98429160D060516013463BD991
:1095F000127893F9451010468A420BD1111F0829A1
:1096000008D893F84610182901D8013103E083F8EF
:10961000442002E0002183F8461093F94440214998
:10962000A24219D191F84740B4B10C3100249442C0
:1096300006DA51F8046F1C4D25F814600134F6E782
:109640000C2805D01849002421F810400130F7E714
:10965000164801780131017083F84520002201216C
:109660001A7083F8471070BD92F84710C9B140F2E4
:10967000DA51A0F2EF248C4208D811780B2905D8D2
:109680000B1D0131117042F8230070BD002283F8D8
:109690004720074B03F13002002143F8041F934297
:1096A000FAD170BD7C090020DC320020E1000020EE
:1096B00088090020024A136C013319441164704771
:1096C0007C090020024B53F820301B68198070473A
:1096D000E4260020074BA1F57A7153F820301A6870
:1096E0001B8959434FF47A7391FBF3F189B21180CE
:1096F000704700BFE42600201FB50123ADF80830F5
:10970000ADF80410002301A9ADF80A30ADF80C3013
:10971000ADF8062006F059FF05B05DF804FB38B53A
:10972000A0F513746379A579DB0745D594F8383231
:1097300005F00105F3B1226B1068838DC3F34E036E
:10974000838494F83C3223B1B4F842320133A4F854
:109750004232917A6A00FFF7CFFF012384F83B324F
:10976000002384F8393284F83A3284F83832A4F885
:10977000403238BD94F83B322046012B04BF94F8A8
:10978000393284F83A32FFF7EBFE94F83B22236B30
:109790003AB9012284F83B221868997A05FA02F254
:1097A00007E0002284F83B2295421868997A08BFA6
:1097B0000222BDE838409FE738BD10B5A0F512740D
:1097C00094F83C22BAB9A36A616A994228D0591C1C
:1097D000A069A162C35C2069DBB25B0043F4007343
:1097E0008142A4F83E324FF00A0384F83D3228BF8C
:1097F000A262012312E094F93D327BB1B4F83E122B
:1098000020464B08A4F83E3201F00101FFF7BDFEEF
:1098100094F83D32013B84F83D3201E084F83C325B
:1098200094F83832002B4ED194F839320133DBB240
:10983000092B84F8393203D12046BDE810408FE669
:109840000A2B40D194F83B322BB9B4F8403243F0A4
:109850000103A4F840326379D9071CD5B4F840025B
:10986000820501D4C30705D4B4F844320133A4F807
:10987000443210E0E36AC0F347000BB198470AE0B6
:10988000E3696269D054E369E1680133B3FBF1F243
:1098900001FB1233E361012284F8382294F83B2261
:1098A0000023012A84F839320DD1A27984F83B32A1
:1098B000236B12F0010F1868997A0CBF0222002264
:1098C000BDE8104018E710BDF0B5046D8279A3899A
:1098D000467923F4005312F0020F4FEA03434FEA94
:1098E00013430CBF00214FF4005112F0040FA38169
:1098F00014BF4FF4806E4FF0000E16F0010F876812
:10990000054614BF04200020B307238A48BF40F057
:1099100008029BB223F4405343EA01032382A18946
:1099200048BF90B289B221F4B05121F00C014EEA47
:10993000010140EA0102A281A38A87B023F44073A7
:109940001B041B0CA38201A806F0E4FD039B049EEC
:10995000254A944218BF1E46A389192272431BB29E
:10996000002BB4BF7E00BE00B2FBF6F66427B6FB48
:10997000F7F00001010907FB1163A28912B2002A66
:10998000B7BFD9001A013231B1FBF7F2A7BF3232AB
:10999000B2FBF7F302F007021043A8BF03F00F0376
:1099A000AA79A8BF184380B212F0010F20812B6D55
:1099B00006D00E498B4202BF042001F548410861E0
:1099C00012F0080F9A8A0BBF22F0080292B212041A
:1099D00042F0080208BF120C9A829A8992B242F4AD
:1099E00000529A8107B0F0BD0038014000440040A9
:1099F0002DE9F04F504C4FF4147685B080469146D7
:109A00001D4606FB0046274608B94C4B02E00128DC
:109A100004D14B4B33631033C6F834314FF4147315
:109A200003FB08F3474AFC18FA50032262712246EE
:109A300003F59C733B44E162A36100214FF4807005
:109A4000D4F8343134324FF0010B62612162E161AC
:109A5000A162616284F83C1284F83912A4F84212BF
:109A6000A4F84412C4F80890A571E060206184F85D
:109A700038B284F8468258681B890222ADF80C304F
:109A800003A910238DF80E308DF80F20019205F0F8
:109A900084F8236B019A597B58681B898DF80E1046
:109AA00003A9ADF80C308DF80F2005F076F830469C
:109AB0005946FFF76AFD322003F081FB224BD4F8B0
:109AC00034A11B681A46B2FBF9F1B1F5803F03D30C
:109AD000012AF8D95208F6E71C4A5046B3FBF2F2C5
:109AE00089B2D2B202F0E2F84FF4147000FB08F031
:109AF000174B07EB000800F512703C180022C8F85D
:109B000048325046214602F019F9D8F8307015F065
:109B1000010F0CBF022200223868B97AFFF7ECFD72
:109B20000C4B3846C8F84C32211D002202F006F9D1
:109B3000304605B0BDE8F08F0C12002048BF010888
:109B400068BF01089CA401085800002040420F0093
:109B5000BB9700081F97000803460A4690F8460284
:109B6000D96A9B7944E71FB50123ADF8083000237B
:109B7000ADF80C30ADF80A30084BADF804101B7886
:109B800001A9012B08BF0323ADF8062008BFADF8DB
:109B90000C3006F01AFD05B05DF804FB78090020D2
:109BA00038B510F80E2C044650F8043C52B9012286
:109BB00000F80E2C20F80C1C997A18680222BDE8D7
:109BC0003840D0E730F80C2C20F80A1C891A89B2EA
:109BD00020F8081C074A10F80F0C002522F8101076
:109BE00004F80E5C1868997A2A46FFF7BCFF04F85F
:109BF000065C38BDDC320020044B53F820301BB12A
:109C000007289CBF1B681980704700BFA40A00206A
:109C10002DE9F7438E460546DFF8A092114699F8E4
:109C2000A0440068164698467246631C89F8A03422
:109C300001F0E8FF2B8901A9ADF8043018238DF855
:109C40000630686802238DF8073004F0A6FFAB7A6F
:109C500009F2A447240127442A6849460C2B00F244
:109C6000F680DFE813F00D00F400F400F40051007A
:109C7000F400F400F4008A00F400F400F400C200E0
:109C8000138CDFF83CC223F001031B041B0C13846C
:109C9000138CB2F804E0108B624520F073004FEA99
:109CA00000404FEA10409BB21FFA8EFE40F0700059
:109CB00014D00CF5006C624510D00CF5406C624578
:109CC0000CD00CF5806C624508D00CF5806C6245B8
:109CD00004D023F0020343F0030307E023F00E0354
:109CE0002EF4407E43F003034EF4807EA2F804E09D
:109CF0001083A2F834801384138B23F008031B0411
:109D00001B0C43F0080336E0138CDFF8B4C123F0DA
:109D100010031B041B0C1384138CB2F804E0108B8B
:109D2000624520F4E6404FEA00404FEA10409BB203
:109D30001FFA8EFE40F4E04008D00CF5006C62453E
:109D400004D023F0200343F0300307E023F0E003C6
:109D50002EF4406E43F030034EF4806EA2F804E01F
:109D60001083A2F838801384138B23F400631B0440
:109D70001B0C43F40063138369E0138CDFF840C1CC
:109D800023F480731B041B0C1384138CB2F804E0BF
:109D9000908B624520F073004FEA00404FEA10407C
:109DA0009BB21FFA8EFE40F0700008D00CF5006CDC
:109DB000624504D023F4007343F4407307E023F4B6
:109DC00060632EF4405E43F440734EF4805EA2F86C
:109DD00004E09083A2F83C801384938B23F0080363
:109DE0001B041B0C43F0080330E0138CDFF8D0C0D9
:109DF00023F480531B041B0C1384108CB2F804E072
:109E0000938B20F4005023F4E6431B0400041B0C46
:109E1000000C62451FFA8EFE43F4E04340F44050CC
:109E200003D00CF5006C624503D12EF4804E4EF445
:109E3000804EA2F804E09383A2F840801084938BB4
:109E400023F400631B041B0C43F4006393832B7BFC
:109E500043B1B2F844306FEA43436FEA53439BB2D5
:109E6000A2F8443013889BB243F001031380AB7A0D
:109E70000C2B19D8DFE803F0071818180B1818185E
:109E80000F18181813000B1902F134000AE00B190F
:109E900002F1380006E00B1902F13C0002E00B1958
:109EA00002F14000C3F8A40438460C44A4F8AC64A2
:109EB000C4F8A82403B0BDE8F08300BF0C12002052
:109EC000002C014004F038BD04F036BD04F034BD70
:109ED000642928BF6421F8B501FB00F5642495FBD3
:109EE000F4F40646E4B20027FBB2A34204D29F205A
:109EF00004F0EBFF0137F7E7B4420BD2142195FBD6
:109F0000F1F5C4EB8410663DC4EB80002844C0B278
:109F100004F0DBFF0134E4B2B44201D29A20F7E747
:109F2000F8BD08B507480DF056FAC0B20928024638
:109F3000044B04DC01302021C0B29954F6E7002222
:109F40001A5408BDC911002008B507480DF043FA9E
:109F5000C0B21428044B04D8421C20211954D0B29A
:109F6000F7E700221A5408BDC91100202DE9F74F68
:109F700003F0FEF8A64C804626686568A768861B35
:109F8000F643451BC71BED43FF43F60FED0FFF0FD5
:109F90002EB93FB9002D00F08782B9462CE04FF072
:109FA000000929E0B14627E003EB8A0BBBF8023039
:109FB0001A050ED413F4805F1DBF964A9BF801105A
:109FC0001268954A954B14BF52F82120126843F845
:109FD0002A20BBF80230D80516D499050AD5904B33
:109FE0001B7813F0040F0CBF8E4A8F4A8B4B1268FC
:109FF00043F82A2009F10109207B5FFA89FA8B498D
:10A0000082450B68D0D326E0894A5046594607F06E
:10A010008BFA884B1B885A0603D550465946864A08
:10A0200016E0580703D550465946844A10E01907F0
:10A0300003D550465946824A0AE09A0703D550464E
:10A040005946804A04E0DB07D4D5504659467E4A3B
:10A0500007F06AFACEE7DFF808E20093BEF90630AF
:10A060007822A3F57A7353434FF47A7293FBF2F399
:10A07000F34603F22B13019300225FFA82FE86451A
:10A0800017D2009B03EB820EBEF802E01EF4806F35
:10A090000DD040F2671ADFF88491019B39F822E075
:10A0A0009E449EFBFAFC0AFB1CEE29F822E00132DA
:10A0B000E3E74DB308F5C333A0336360637B544AD1
:10A0C00013BB9373614B1B6813F0020F0AD0DFF8C8
:10A0D00094E19EF800E0BEF1000F03D04FF0010EB6
:10A0E00082F80EE0DA0506D5594B5B791BB1A37BEC
:10A0F00043F00203A3734A4B1B7813F0050F02BF12
:10A10000A37B43F00403A37394F80EE0BEF1000FA9
:10A1100003D13F4B5B7B002B4FD094F80DC01CF05C
:10A12000010FACF10C031DD1BCF1030F07D8DFF810
:10A13000E8901EF0040F3B4A08BF4A4600E0364A4A
:10A14000ACF1040CBCF1070F05D8DFF81CC11EF000
:10A15000010F18BF6246DBB2032B0ED81EF0020FB0
:10A160003C4B06E0DBB2032B06D82F4B2A4A1EF0ED
:10A17000020F18BF1A4600E0274A4FF0000C5FFAA2
:10A180008CF383420DD20B6803EB8C035B881B06B8
:10A1900042BFD2F80090214B43F82C900CF1010CF7
:10A1A000EDE785B1BEF1000F08D0637B184A01339B
:10A1B000DBB2142B06D1002304E025B1637B002B16
:10A1C000F3D100E05373002E52D0234A3223B2F968
:10A1D0000250B2F90020002DB8BF6D42002AB8BF6E
:10A1E000524295FBF3F592FBF3F2EDB2D3B2AB42E0
:10A1F00038BF2B46194A13B192FBF3F300E0134624
:10A2000043442360E37B024A83BB01232FE000BF6A
:10A21000701700202824002008BC0108CA0800206C
:10A22000E5330020DCBB0108CCBB01089011002005
:10A23000B4A401088C110020BAA40108C0A401082C
:10A24000C6A40108CCA40108D2A401089C280020BF
:10A25000B4330020E4BB0108AC100020400D030023
:10A26000D828002018110020ECBB01080023D3736C
:10A270008F4D904B2D78E27BADB9002F00F00F8110
:10A280008D4B267B1A788D4B02F0040293F800C0A8
:10A290008B4BD2B2D3F800E00B680021894D03EB61
:10A2A00086060F46B5E01AB9874A1A61002508E00C
:10A2B000864AFAE70A68AB00D6187688760604D490
:10A2C0000135EBB28342F5D3D7E7814EB6F9006092
:10A2D000192E25DD12F803E094F814C00EF00F09D2
:10A2E000E14526690CDCDFF8CCC19CF815C0BCEB5D
:10A2F0001E1FDEBFD6F800C0DFF8D8E143F80EC05D
:10A3000012F803E094F816C00EF00F09E14533DBB4
:10A31000DFF8A0C19CF815C0BCEB1E1F2CDC26E0AA
:10A32000193629DA12F803E094F814C00EF00F0978
:10A33000E14526690CDCDFF87CC19CF817C0BCEB5A
:10A340001E1FA2BFD6F800C0DFF888E143F80EC098
:10A3500012F803E094F816C00EF00F09E1450BDB8C
:10A36000DFF850C19CF817C0BCEB1E1F04DBD6F809
:10A3700000E0584E43F806E0554EB6F90260192E3B
:10A380001BDD12F803C094F814E00CF00F09F1453E
:10A3900026690CDCDFF81C9199F81590B9EB1C1FAD
:10A3A000DEBFD6F80090DFF82CC143F80C90D25CE9
:10A3B00002F00F0CF4451EDD82E7193680DA12F840
:10A3C00003C094F816E00CF00F09F14526690CDB88
:10A3D000DFF8E09099F81590B9EB1C1FDEBFD6F8B6
:10A3E0000090DFF8F0C043F80C90D25C02F00F0C44
:10A3F000F445FFF665AF94F817E0BEEB121FA2BF5D
:10A400003668344A9E505BE75888000504D404330C
:10A410000435B342F8D122E04AB101EB0C0A062020
:10A420009AFBF0F900FB19A001280DDC01E057B9F7
:10A43000012793F801900EEB89003EF829A090F8CF
:10A440000290C07803E01746002081468246013121
:10A4500025F802AC85F800906870C9B2D7E7174AB2
:10A460001378013B13F0FF0308BF06231370124B50
:10A470001B785B0741BFBBF906304FF47A72A3F536
:10A480007A7303EBC30348BF93FBF2F3124A46BF50
:10A490000133DBB2012392FBF3F34344A36003B027
:10A4A000BDE8F04F04F086BA03B0BDE8F08F00BFFE
:10A4B0008A33002070170020E533002020000020A0
:10A4C00028240020CC080020E8BB010808BC0108B3
:10A4D000AC100020CA080020400D0300344B354A60
:10A4E0001B68126810B51A60334A116859605168C8
:10A4F00092689960DA60314A11681961516892680E
:10A5000059619A612E4A1168D9615168926819623D
:10A510005A622C4A11881985518859859188D288A8
:10A520009985DA85284A1188198651885986928832
:10A530009A86264A1188D9865188928819871946A1
:10A5400021F83A2F224A10780022824206DA214C62
:10A5500034F81240013221F8024FF6E71E4A128801
:10A56000A3F864201D4A1288A3F866201C4A1188AB
:10A57000A3F86C1051889288A3F86E10A3F870208D
:10A58000184A3B2112689A66174A126892FBF1F248
:10A59000B2F5967FC8BF4FF0FF325A67134A128850
:10A5A000A3F87820124A5289A3F85E2010BD00BF9C
:10A5B000EC300020C4330020302200203C22002058
:10A5C00048220020AC100020E80F00209610002048
:10A5D000E026002008100020E02500206C0E00205E
:10A5E000EE0F0020A0100020000000202810002006
:10A5F000F40F002070B5472007F020FF174B1B68B1
:10A600001B0307D5164B174A5B6810681B68C01AF6
:10A6100007F046FF144E154C154D307807F040FFFB
:10A6200023682868C01A07F04AFF63686868C01A80
:10A6300007F045FF0F4B188807F032FF0E4B1888C4
:10A6400007F02EFF0D4B188807F02AFF337823748C
:10A650002B68A3606B68E36070BD00BF70320020A0
:10A66000EC300020C4330020D2100020D83000206D
:10A67000D4100020D0100020CE1000203010002078
:10A680000A4A138801331380094A1368013313609F
:10A69000084A138801339BB2202B01BF002313808B
:10A6A000054A138808BF0133138070479032002099
:10A6B000783200207C3200207E32002038B53A4BC0
:10A6C00005461B780C46083B012B6BD8452007F04C
:10A6D000B5FE284607F0B2FE0C2D23D004D80A2D73
:10A6E0000AD014D835B138BD0E2D4BD02ED3FF2D46
:10A6F00050D038BD206849E0207807F09FFE62798D
:10A700006378002A14BF80200020184300E02078DE
:10A7100007F094FEA07807F091FEE07807F08EFE37
:10A7200020793BE0B4F9000007F0B0FEA07807F014
:10A7300085FEE07807F082FEB4F9040007F0A6FE7B
:10A74000B4F90600BDE8384007F0A0BE6378207871
:10A750008BB180F0800007F071FEA468E0B207F0D2
:10A760006DFEC4F3072007F069FEC4F3074007F04D
:10A7700065FE200E12E007F061FE6068BDE838401B
:10A7800007F09DBE206807F08BFE6068BDE838408A
:10A7900007F086BE054807F0D5FD0020BDE838402B
:10A7A00007F04CBE38BD00BFD0300020ABC401085C
:10A7B0002DE9F04FBF4B8BB018880193002840F073
:10A7C000A380BD4EFDF7F8F9FFF788FE34684920F5
:10A7D000254607F033FEB94B04F11C08186807F052
:10A7E0005FFE55F8040B07F05BFE284600F0A6FB61
:10A7F00004F1100000F0A2FB1027B14D01232A68DC
:10A80000BB40134203D0D8F8000007F058FE0137D0
:10A81000132F08F10408F0D1AA4F04F1280000F02A
:10A820007DFBB7F84431B4F92E00B846C01A07F0E2
:10A8300037FE2B6813F4805F08D0A34BB4F8640094
:10A840001B88181AC0F30D0007F02AFE2B68990424
:10A8500003D5B4F8660007F023FE2B685A0503D52C
:10A8600004F16C0000F05AFB2B681B0502D5A06EAA
:10A8700007F025FE2B685F0402D5606F07F01FFE0E
:10A880002B68180403D5B4F8780007F009FE2746B2
:10A8900004F1300000F042FB04F1360000F03EFB12
:10A8A000B8F8443137F93C0F4FF00108C01A07F0EF
:10A8B000F7FD864B1B78984509DA37F9020FB4F992
:10A8C0003C3008F10108C01A07F0F9FDF1E72B68E8
:10A8D000990505D5B4F95E00A0F2DC5007F0EFFD54
:10A8E00032687B487260B260121A9110794A4A430A
:10A8F000531C032293FBF2F202EB42029A1A7C23CE
:10A9000003FB0203336068E2734B744A1B681168EF
:10A910008B4206D00AA941F8203D00201360FFF7C2
:10A92000CDFE684A019B92F8CE171B8892F8CF079C
:10A930000B44013BB3FBF0F200FB12338B4280F07F
:10A9400017825D4F0120FDF737F9FFF7C7FD502053
:10A950003E687D6807F072FDBA683B6810681B6846
:10A960007A6803441068A3EB400007F0A8FD6A680A
:10A97000736802A89B1A0293AA68B3689B1A039390
:10A98000EA68F3689B1A049300F0D8FA2A693369DD
:10A990009B1A02936A6973699B1A0393B369AA6944
:10A9A0009B1A04930023194602AA52F8212002F1AF
:10A9B00020003F2842D802F108000F2806D80232B2
:10A9C000032A04D9002B08BF012300E00223013130
:10A9D0000329E9D1012B02980ED0022B21D0039B31
:10A9E00000F0030003F003039B0043EA0010049B04
:10A9F00003F0030318430CE000F00F0040F04000A8
:10AA000007F01CFD0498039B00F00F0040EA0310C0
:10AA1000C0B207F013FD06F11C0B05F11C08102451
:10AA20006FE000F03F0040F0800007F007FD9DF868
:10AA30000C0007F003FD9DF81000EAE702224FF03A
:10AA4000000802AB53F822304FEA880803F1800176
:10AA5000FF2910D903F50041B1F5803F02D248F03B
:10AA6000010808E003F50003B3F1807F34BF48F02C
:10AA7000020848F0030812F1FF32E2D268F03F000A
:10AA8000C0B207F0DBFC02AC0DF1140A08F00303BE
:10AA9000022B207807D0032B22D0012B29D107F0DD
:10AAA000CDFC607825E007F0C9FC607807F0C6FCB3
:10AAB000A0781EE07C320020EC30002078320020AC
:10AAC00070320020FC2800206C320020E02600209C
:10AAD000F8300020DF7BEFBD843200208032002080
:10AAE00007F0ACFC607807F0A9FCA07807F0A6FCA2
:10AAF000E078043407F0A2FC54454FEAA808C5D119
:10AB000089E7B84901220B68A2401A428A4606D05A
:10AB1000DBF80000D8F80030C01A07F0D0FC013490
:10AB2000132C0BF1040B08F10408EAD106F12600FE
:10AB300005F12601002331F9024F30F9022F121BD3
:10AB400002AC44F823200133042BF4D103214FF04D
:10AB500000094FEA89035FFA83F902AB53F8212019
:10AB60006AB102F108000F2802D849F0010906E095
:10AB70008032FF2A94BF49F0020949F0030911F11C
:10AB8000FF31E6D24846002407F058FCA0460DF1FC
:10AB9000080B09F00302022A16D0032A1DD0012A4D
:10ABA00038D1B8F1000F05D1DBF800409046240100
:10ABB000E4B22FE0DBF800004FF0000800F00F00D7
:10ABC000204307F03BFC25E0B8F1000F0CD0DBF888
:10ABD0000000C0F30310204316E0B8F1000F08D1C5
:10ABE0009BF8010007F02AFC9BF8000007F026FC08
:10ABF00010E0DBF80000C0F30330204307F01EFC38
:10AC0000DBF80000C0F3071007F018FCDBF8004089
:10AC10002401E4B20BF1040B06AB9B454FEA990902
:10AC2000B7D1B8F1010F02D1204607F007FCDAF8DE
:10AC3000003013F480541FBFB6F86420B5F86410D8
:10AC40000124521A18BF02929A040AD50AAA02EBEA
:10AC50008401B5F86600B6F866200134121A41F88E
:10AC6000202C580513D502AA02EB840C06F16A0EBB
:10AC700005F16A0000223EF9021F30F9028FC8EB8D
:10AC800001014CF822100132032AF4D103341905D2
:10AC900008D50AAA02EB8400A96EB26E0134521ADA
:10ACA00040F8202C5A0408D50AAA02EB8400696FE8
:10ACB000726F0134521A40F8202C18040BD50AABDD
:10ACC00003EB8402B5F87810B6F8783001345B1ADB
:10ACD00042F8203C00E0FCB1012C03D1029807F0BF
:10ACE000EEFB19E0631E002002AA52F82320400068
:10ACF000C0B20AB140F00100013BF5D507F09EFB60
:10AD00004FF0000802AB53F8280008B107F0D7FB5A
:10AD100008F10108A045F5DB30200321FCF78CFF8A
:10AD200036200321FCF788FF2F4B3C201978FCF7D5
:10AD300083FFDAF80030990506D5B6F95E00B5F95B
:10AD40005E30C01A07F0BBFB3A6828487B687A601F
:10AD5000121A9110264ABB604A43531C032293FBEC
:10AD6000F2F202EB42029A1A7C2303FB02033B60DD
:10AD7000204B1B681A0630D51F4C204D22682B68CB
:10AD80009A420BD162686B689A4207D1019B1B887B
:10AD9000102B11D11A4B1B885B060DD1482007F0F0
:10ADA0004DFB206807F08BFB606807F088FB236889
:10ADB0002B6063686B600EE0124A104B11782A7C9E
:10ADC000914208D1104A99681068884203D15268AC
:10ADD000DB689A4201D0FFF70DFC07F0A1FA0BB037
:10ADE000BDE8F08F70320020E0260020F83000200F
:10ADF000DF7BEFBD9C28002034100020D8300020DD
:10AE00007E320020D2100020D41000202DE9F84F0F
:10AE10000C9EC2EB030B394C0B9B002914BF4FF067
:10AE2000060A4FF0040AF61A636805460133904695
:10AE300013D1236853455ED2314A032B98BF29466C
:10AE400052F823202F4807F0E7FA63680022013305
:10AE500063602D4B05461A7013E0002511E02B4A64
:10AE60001278954240DA0B9BE3B109FB06F2995C3C
:10AE700001228A40264909680A4213D163680133D6
:10AE80006360D4F804900A9B1C4F9945E7DB2BD1F3
:10AE90000A2007F0D3FA3B6801333B604FF0FF33E1
:10AEA0007B6021E0184A117821B12C2007F0C6FA06
:10AEB000013501E00121117009FB0BF3226808EB59
:10AEC000030752B958F8030007F03CFA97F9041049
:10AED00005444B1CD2D00F4802E03A440E48117989
:10AEE00007F09AFA0544C9E7206850452CBF0020B6
:10AEF0000120BDE8F88F0020BDE8F88F88320020DF
:10AF0000D8A40108B6C40108881700205C000020FE
:10AF100070320020C5C4010831C4010810B50446D0
:10AF2000B0F9000007F0CBFAB4F9020007F0C7FA55
:10AF3000B4F90400BDE8104007F0C1BA10B50446EA
:10AF4000006807F0BCFA606807F0B9FAA068BDE8CD
:10AF5000104007F0B4BA2DE9F74F0120FCF714FDBB
:10AF6000002480B3012C2ED84FF04C0A0AFB04F7C2
:10AF7000DFF85C8008EB070B0BF14806B57815B1DC
:10AF80000134E4B2EDE790F9003090F804E018469F
:10AF90000E4B03228DE8240001212A4653F82E305F
:10AFA000FCF7C8FB814650B15846294652460CF082
:10AFB000CEF901231C4448F80790B370E4B2012095
:10AFC000FCF7C8FCCDE703B0BDE8F08FF0A40108A2
:10AFD0008C17002000212A2210B511480CF0B7F977
:10AFE000104B0022194610480424105C013283F8EB
:10AFF000E801052083F8ED4182424FF0000483F818
:10B00000EC0183F8EF4183F8EE0103F10803EAD184
:10B010000123A1F8EA31522381F8E63110BD00BFC7
:10B02000E22A0020FC280020E9C4010870B5064689
:10B03000441E14F8011F89B1094D28460CF0BDF9D2
:10B040000028F6D005F1080398423FBF054B401B8E
:10B05000C018A31B38BF80F88831EAE770BD00BF75
:10B060005ED90108FC2800202DE9F04FB34C8BB0CD
:10B070009A469DF85430019205460C220E4604F182
:10B080009800002100930CF062F90021142204F1D1
:10B09000A4000CF05CF9002384F8B830A84B1F78AA
:10B0A0009846A84B03F11802012F88BF1346C4F835
:10B0B000BC30F9F71CFA8146834670B3A24BB5F554
:10B0C000807FC4F8A430A14BC4F8A830A04BC4F8CA
:10B0D000B030A04BC4F8B4309F4B01D1002216E031
:10B0E000BB2D01D9012212E0612D01D902220EE00F
:10B0F000292D01D903220AE0132D01D9042206E0EB
:10B10000092D01D9052202E0002DE7D006221A7090
:10B11000012384F8B83002236DE0192002F04FF8C3
:10B12000682015214A46F9F723F878B38B4B622D36
:10B13000C4F8A4308A4BC4F8A8308A4BC4F8AC30A9
:10B14000894BC4F8B030834BC4F8B430824B0FD075
:10B1500004D80A2D13D0142D0FD00CE0BC2D05D02F
:10B16000B5F5807F07D183F801900AE0012200E065
:10B1700002225A7005E00322FBE70422F9E70522C8
:10B18000F7E7012384F8B830042334E0032F40F0BC
:10B19000E0830122752004A9F9F74AF99DF81020EF
:10B1A000702A40F0D683714BBB2DC4F8A430704B8D
:10B1B000C4F8A8306F4BC4F8B030664BC4F8B43054
:10B1C000654B01D901220EE0612D01D902220AE06E
:10B1D000292D01D99F700AE0132D01D9042202E024
:10B1E000092D02D905229A7001E00622FBE701230E
:10B1F00084F8B8300723604A604913700B68604FC9
:10B2000043F001030B6000233B709146082E33D8B6
:10B21000DFE806F0373237101D22102D2D004FF0D9
:10B22000000B0AAB03F818BD532059460122F8F76A
:10B2300089FD58BB434B98F8001003F1180201290F
:10B2400088BF1346C4F8BC30F9F751F970BB98F8C1
:10B250000030012B40F29E8000210AAB03F8181D3C
:10B2600018200122F8F76EFD002840F0B28098F80F
:10B270000030032B00F0BC80012E40F2D38000266A
:10B280003E7098F80030012BD4D8C8E79DF81030F4
:10B29000E52BCFD13B4B84F8C0B0C4F898303A4B83
:10B2A000C4F89C3004233B700223B4E006210A4614
:10B2B00004AB6820F8F746FD9DF8151001F0010277
:10B2C0009DF8131001F001014B0043EA82019DF843
:10B2D000112002F001030B430AD05BB2012B01D114
:10B2E000002302E0022B0FD1012384F8C13012E0C9
:10B2F0000C210DEB010368200122F8F723FD9DF8D6
:10B300000C3013F00F0303D1052001F0D3FF02E04E
:10B31000042BE9D1E4E71D4BC4F898301C4BC4F86A
:10B320009C3094F8C130002B0CBF6F236E2384F83F
:10B33000A03001233B7003236DE000BF8C17002079
:10B34000E733002010A501084D420008FD3E00082B
:10B35000DD3E000890C1793D21000020C542000873
:10B36000CF3F00089D3F00087D3F0008E13B0008FB
:10B37000774400085944000850000020C8100020FD
:10B38000E6330020C9430008A9400008193D000821
:10B390003D3F000800220AAB03F8182D1C200D21A8
:10B3A0000122F8F7CFFC00283FF456AF9DF810308B
:10B3B0002A2B02D01A2B7FF44FAFD24A84F8C23026
:10B3C000C4F89820D04A02233B70C4F89C20042380
:10B3D00021E09DF81030FB2B7FF449AFCB4BC4F834
:10B3E0009830CB4BC4F89C3001233B70052312E00E
:10B3F000752004A90122F9F71BF89DF81030702B75
:10B400007FF43AAFC34BC4F89830C34BC4F89C30B8
:10B4100001233B700823C14A89F80130136843F0C7
:10B420000203136098F80030012B05D107F0C8F82B
:10B43000BB4B4FF400525A610A2001F0C0FE772046
:10B44000A021012203ABF8F77DFC30B994F8D48039
:10B45000B44EB8F1000F6FD073E21E2101227720A5
:10B46000F8F786FE4FF42F6001F09EFE0027A7F14B
:10B4700060010026C9B2022204AB77208DF810606B
:10B480008DF81160F8F75EFC9DF811309DF81020E2
:10B4900043EA0222A34B03F1C4017A520237102F70
:10B4A000E5D1B3F8D210324601F00F0701F47F4125
:10B4B000A3F8D21033464FF0010E22F001002044D1
:10B4C000B0F8C400002818BF4FF0000ED60703D50F
:10B4D000C0B24340082002E083EA1023FAE71E04CA
:10B4E00048BF83F4C05301384FEA4303F7D1013218
:10B4F000102AE2D139438B4AA4F8D210BEF1000FD2
:10B50000A4D1C3F303339F42A0D142F21073A2F837
:10B51000FC30A2F8FE30844BC2F80031834BC2F8F5
:10B520000431834BC2F80831824BC2F80C31824B94
:10B53000C2F8103103234FE1794C07F041F84FF482
:10B540008047042303A92046ADF80C708DF80E3017
:10B5500003F023FB4FF400532361784801F0E0FE31
:10B560000E21022003F004FB0823049704A80127FE
:10B570008DF815308DF814808DF816704FF0030992
:10B5800005F036F9282302A88DF808308DF80990C7
:10B590008DF80A808DF80B7006F098FF142001F0EA
:10B5A0000EFE7720D0213A4603ABF8F7CBFB0028FC
:10B5B00000F090809DF80C30A6F8F890552B86F896
:10B5C000EF3040F08780D1213A4603AB7720F8F77F
:10B5D000B9FB9DF80C30772003F00F021B0986F8A9
:10B5E000F02086F8F130162204ABAA21F8F7AAFB66
:10B5F0009DF810209DF8113043EA0223A6F8D830B8
:10B600009DF812209DF8133043EA0223A6F8DA30A1
:10B610009DF814209DF8153043EA0223A6F8DC308B
:10B620009DF816209DF8173043EA0223A6F8DE3075
:10B630009DF818209DF8193043EA0223A6F8E0305F
:10B640009DF81A209DF81B3043EA0223A6F8E23049
:10B650009DF81C209DF81D3043EA0223A6F8E43033
:10B660009DF81E209DF81F3043EA0223A6F8E6301D
:10B670009DF820209DF8213043EA0223A6F8E83007
:10B680009DF822209DF8233043EA0223A6F8EA30F1
:10B690009DF824209DF8253043EA0223A6F8EC30DB
:10B6A00041F2707386F8D470A6F8FC3046F6781331
:10B6B000A6F8FE30224BC6F80031224BC6F8043102
:10B6C000214BC6F80831214BC6F80C31204BC6F887
:10B6D000103136E11F4A136823F480431360114B85
:10B6E000164AD3F81411914209D0D3F81811914297
:10B6F00032D0D3F81C11914234D102222DE0002225
:10B700002BE000BF154300080D400008A5430008CA
:10B7100065400008B13A0008B3440008C810002092
:10B72000001001408C17002005420008013E00086F
:10B73000FD410008F13D0008B1350008793B0008E3
:10B7400039420008A93E0008154200085D3E000885
:10B75000D539000800040140012203EB82020021D8
:10B76000C2F8141193F820314FF4005262617B4CFF
:10B770008BBB142001F023FD04F221137620D0218D
:10B780000122F8F7DFFA94F82131582B2BD104F578
:10B790009273882118227620F8F7D4FA7620F421C3
:10B7A0003122F8F7E5FC012384F820316C4BA4F832
:10B7B000FC80C4F804316B4BC4F8003145F6D81353
:10B7C000A4F8FE30684BC4F80831684BC4F80C315B
:10B7D000674BC4F810310423664A9370664A1368B5
:10B7E00043F004031360644E5C4C336813F0020FA3
:10B7F00002D0D4F898309847009B63B315F0FF0F40
:10B80000336809D140F2596213F0020F40F27123FC
:10B8100018BF13467D2208E09A0759BF4FF47A7388
:10B820001A464FF4FA634FF47A721499994205DB81
:10B83000B1F57A6F0B46A8BF4FF47A63511E0B44E3
:10B84000B3FBF2F3013BDBB203FB022284F840318D
:10B85000C4F8442106E09DF8003084F84031149B80
:10B86000C4F84431D4F8A4309847444B019F93F86E
:10B870000090434B03F11802B9F1010F94BF9946B0
:10B880009146404D00232B700FB1022F55D14FF040
:10B8900000080AAB03F8188D1E200A210122DFF8E8
:10B8A000BCB0C4F84891F8F74DFA98B19DF8103043
:10B8B000482B48D1344B0222CBF84C31334BCBF8D8
:10B8C000503103232B702B4BDA70336843F008039D
:10B8D000336001E0804636E02D4B93F858210AB1E1
:10B8E00084F8B82093F859210AB12A490A7093F8CC
:10B8F0005A3103B12B7033681B0718D564269AFBA5
:10B90000F6F5284608F010F8074606FB15A000B229
:10B9100008F00AF8204908F05BF80146384607F0BD
:10B920004FFF1E4908F054F8C4F8540102E0002308
:10B93000C4F854314FF0010B0BE0012FCCD91F4656
:10B940009FE7022348E7012FC6D9002785F800802A
:10B950009DE758460BB0BDE8F08F00BF8C17002064
:10B96000D1390008D33900080D420008113E000803
:10B970006D37000850000020C8100020E733002079
:10B9800040A50108E8330020FFEB0008A5E8000807
:10B99000FC280020E63300208988883C00002041F4
:10B9A0000120002105F07ABA174AF0B5164692F840
:10B9B0005831D2F85CE1042B10D85C1C0EEBC303A9
:10B9C0009D1CE4B208D09A88D10705D5104203D057
:10B9D00008E00131052907D12346ECE786F8583104
:10B9E0000020F0BD9F7800210C2202FB01F3064DE0
:10B9F00005F5B07C1CF803209742EAD12B4485F86A
:10BA00005841D3F86401F0BD8C1700208A6810B546
:10BA10000C6A036814430A6923F4FF4314434A6918
:10BA200023F0700314438A691443CA6914434A6AB1
:10BA300014438A6A224313430360CB6843600B6854
:10BA400083604B68C36010BD026D70B515880446F5
:10BA5000ADB2A90613D5036B8BB9C36A1BB190882D
:10BA600080B298470BE0E169928840694E1CD2B2DF
:10BA7000E6614254E169E268914228BFE3612B0626
:10BA800013D5636AA26A9A42236D0AD0511CA06939
:10BA9000A162825C9A802369994206D30023A36243
:10BAA00070BDDA6822F08002DA6070BD026B034676
:10BAB000C16810B5406942B11A6C8C1A013A08BFCE
:10BAC0000A46005D1A64C0B210BD1A6A805C013279
:10BAD0008A4228BF0022C0B21A6210BD436B13B164
:10BAE00090F844007047836A406A1B1A58425841D4
:10BAF0007047036B13B15B68016C01E0C369016AB5
:10BB00008B423CBFC2689B18581AC0B27047836A08
:10BB10008169426B1944D160416A994297BF0169BA
:10BB2000CB1ACB1A536096BF0023536083624FF049
:10BB3000000380F84430136888BF816243F001033A
:10BB400013607047436A8269D154436A02690133C2
:10BB5000934228BF00234362436B1BB11B68DB0782
:10BB600005D4D4E7026DD36843F08003D3607047F7
:10BB70004171FDF7A9BE8160FDF7A6BE2DE9F04138
:10BB800005460E46078A83899BB21F40002F37D097
:10BB9000B7FA87F24FF00043D340DB4399B21F401E
:10BBA000A2F11B032982042BF0D8DFE803F0221F47
:10BBB0001C190300746A24B1013C0023A4B273620F
:10BBC00001E0AC8DA4B2D6F82080B8F1000FDDD032
:10BBD000D8F80030404621469847D8F80480F4E76A
:10BBE0003068A98E08E07068298F05E0B068A98FD9
:10BBF00002E0F068B5F84010036889B29847C5E7DD
:10BC0000BDE8F081254B10B55A43254B254C1B68E8
:10BC10000139B3FBF2F20388013AA04289B292B231
:10BC20009BB212D004F50064A0420ED0B0F1804F58
:10BC30000BD0A4F59834A04207D004F58064A0424C
:10BC400003D004F58064A04202D123F070039BB2BC
:10BC5000154CA04206D004F58064A0421CBF23F41A
:10BC600040739BB203800F4B8185984202850FD0B1
:10BC700003F5006398420BD003F54063984207D068
:10BC800003F58063984203D003F58063984201D1A5
:10BC9000002303860123838210BD00BF40420F00B2
:10BCA00058000020002C01400010004073B50546EC
:10BCB0000068FFF7A7FF2A680124138800269BB2BB
:10BCC00043F001031380EB7A01A88DF804308DF85E
:10BCD00005408DF806608DF8074006F0F7FBEB7A1B
:10BCE0001B2B0BD1192301A88DF804308DF80540CA
:10BCF0008DF806608DF8074006F0E8FB02B070BDD5
:10BD00000C4B800A98420CD004D8B0F5801F0CD19F
:10BD100001207047084B984205D04933984206D01D
:10BD200003E00220704703207047FE207047002088
:10BD3000704700BF01001000020010002DE9F84319
:10BD400004680746204688469146FFF7D9FF032836
:10BD50004BD8BA7A9108B8F1000F06D1A589AEB2D6
:10BD600002258D4026EA0505A5810A2303FB001361
:10BD70001F4A42F82380043342F82390B8F1000FA1
:10BD800007D0BD7AA189AD080223AB400B439BB21B
:10BD9000A3812823434303F120011144EFF31286CA
:10BDA000502585F3128803F10C051C331544134408
:10BDB00055F8047F17B10F60296804319D42F7D10F
:10BDC00000230B60F3B283F31188282303FB0020C8
:10BDD000036A23B1A3899BB243F0010304E0A38962
:10BDE00023F001031B041B0CA381BDE8F88300BFF3
:10BDF00068220020004827E628190020004823E692
:10BE00007C19002000481FE6D01900200B4B4FF48E
:10BE100000525A604FF6FE730948D0F8DC201168D2
:10BE20000B401360D0F8CC20D0F8D0309A4201D02B
:10BE3000A8306CE6012380F8EC3070470000024027
:10BE4000281900202DE9F0431D46A64B8DB09842DD
:10BE5000884617469DF850605CD1A34BA34AA4497D
:10BE6000C3F8A82003F1FC02C3F8BC2003F5FE725E
:10BE7000C3F8C0204FF48072C3F8B420C3F8B820D0
:10BE80009C4AC3F8B070C3F8D820A2F54842543A8F
:10BE9000C3F8F420C3F8F020C3F8F800C3F8DC10AE
:10BEA000954B9A6942F480429A615A6942F00102C4
:10BEB0005A6102238DF803304FF40073ADF800305F
:10BEC000330701D51C230FE0AC0706D518238B4898
:10BED00069468DF8023002F060FEE8070AD54FF49B
:10BEE0008063ADF800304823844869468DF80230FD
:10BEF00002F053FE0E238DF804300022012301A826
:10BF00008DF805308DF806208DF807307C4C06F052
:10BF1000DDFAA1E07B4B98424ED1734B734ADF654B
:10BF20005A654FF480721A665A6603F53F729A6634
:10BF300003F57F72DA66744AC3F8A400C3F89C2044
:10BF4000C3F8A0206C4B3107DA6942F40032DA61A1
:10BF50005A6942F001025A614FF002038DF8033032
:10BF60004FF00403ADF8003001D51C230EE0AA0702
:10BF700006D51823614869468DF8023002F00DFE9F
:10BF8000EB0709D50823ADF8003048235B48694624
:10BF90008DF8023002F001FE26238DF804300022D5
:10BFA000012301A88DF805308DF806208DF80730A3
:10BFB000564C06F08BFA4FE0554B984240F0ED801E
:10BFC000494B4A4A9F601A6003F2FC425A6103F2ED
:10BFD000FC529A614FF48072DA601A614D4A18651A
:10BFE0009A64DA64444B3407DA6942F48022DA61F5
:10BFF0009A6942F008029A614FF002038DF803300B
:10C000004FF48063ADF8003001D51C230FE0A80782
:10C0100006D51823404869468DF8023002F0BDFD70
:10C02000E9070AD54FF40063ADF8003048233A48D9
:10C0300069468DF8023002F0B0FD27238DF80430F8
:10C040000022012301A88DF805308DF806208DF817
:10C05000073006F03BFA244C4FF00009012384F826
:10C060004430C4F82090C4F81C90C4F82890C4F858
:10C070002490C4F82C806571A760A6712046FDF756
:10C0800023FCEA0752D5206B002847D0E36CCDF89B
:10C090000C9001934FF480530A9380230693E36836
:10C0A000CDF814900493202309936369CDF81C9074
:10C0B0000293CDF82090CDF82C9004F0B3F901A9AB
:10C0C000206BFFF7A3FC226B216D136843F0010383
:10C0D00013608B8A9BB243F040038B8253689BB200
:10C0E000236423E0003801402819002070A50108CE
:10C0F0004400024058000240001002400008014085
:10C10000D019002000440040044400407C19002065
:10C110000048004004480040000C01404FF6DF7228
:10C12000236D1A80DA6842F02002DA60AB072CD562
:10C13000606B28B3A36C002501934FF480530A93DE
:10C140008023069323690295049310230393059596
:10C150000795089509950B9504F064F9606B01A9A2
:10C16000FFF754FC636B1A6842F002021A60226DFA
:10C170005D605D60938A9BB243F08003938204E02C
:10C18000226DD36843F08003D360226D20469389EB
:10C190009BB243F40053938100E000200DB0BDE852
:10C1A000F08300BF10B507F0BFFB0021044607F085
:10C1B000CBFD08B1204601E004F10040054907F03D
:10C1C000BBFC054907F004FCFCF7FCFD034B1860C1
:10C1D00010BD00BF8096184B35FA8E3C48000020F9
:10C1E000F8B59C4B04461B68187818B1012800F07C
:10C1F0006A819AE2242C984D0CD006D80A2C00F0C3
:10C20000D9800D2C00F0D68048E12A2C06D02C2CA9
:10C2100004D043E128706870A87050E18F4B6978B2
:10C220002F7800208C4A58542FBB1978D770472993
:10C2300021D1597850291ED19978472907D1D97829
:10C24000472904D11979412901D10121D170997867
:10C25000824A522903D1D1784D2900F06882997819
:10C260007E4A472907D1D178532904D11279562A19
:10C2700004BF0322EA70EA78774E022A39D0032AF3
:10C280004CD0012A40F08580BA1E072A00F2818036
:10C29000DFE802F004080F131A257F2A06F014FBCA
:10C2A000686076E01B78532B73D16B685B426B60E0
:10C2B0006FE006F009FBA8606BE01B78572B68D194
:10C2C000AB685B42AB6064E01B78302B644B1A7840
:10C2D0008CBF42F0020222F002021A7059E00020E4
:10C2E00006F052FB287354E0002006F04DFBE88175
:10C2F0004FE0072F06D0082F4BD1012006F044FB5A
:10C30000708246E0012006F03FFB41F2184358439B
:10C310004FF47A73B0FBF3F030823AE0022F07D08B
:10C32000032F0AD1002006F02FFB4E4B187030E08F
:10C33000002006F029FB30752BE02AD93A1F921015
:10C34000337D0132D2B2013B02EB8303DBB2102B0F
:10C350001FD8F91EC2F1010201EB8202D2B2012AFA
:10C360000BD0042A11D100205E1E06F00DFB3E4BBF
:10C37000002298553D4B9A5507E03D4A5E1E00202D
:10C38000935506F001FB3B4B98553B4A136801332C
:10C390001360314B2A2C18BF9A7807F101074FF030
:10C3A00000000CBF012254402F7068700CBF5A75FA
:10C3B0009C7084E0687D002848D0304B13F8012D34
:10C3C0002F495A708B42F9D1244A234C1378527862
:10C3D000402B85BF373B1B011B01DBB298BF03F02D
:10C3E000F003402A8CBF373A303AD2B21344AA78CD
:10C3F000DBB29A4227D121230B702249E0780B68E7
:10C40000012803F101031E4A0B600AD002281CD147
:10C4100072231370228A1C4B1A80628A1B4B1A806B
:10C4200013E0672313700E4B1B789F070ED5184B34
:10C4300062681A60A2685A60227B164B1A70E28901
:10C44000154B1A8002E03F230B70002000236B7510
:10C4500035E000BF5002002024200020C828002022
:10C46000CC10002048100020791000206910002016
:10C470004910002059100020E0110020E80A002097
:10C48000D40A0020EC110020CE1000203010002033
:10C49000D4100020D2100020D01000206B78687DCE
:10C4A0000E2B9FBFA54A591C5170A54A98BFD45462
:10C4B000A24A18B993785C40947000E000200030E4
:10C4C00018BF0120F8BD9D4B0022997D082900F27C
:10C4D0002C81DFE801F0050B0F15202B475D67006D
:10C4E000B52C40F02281DA75012239E0622C08BFB8
:10C4F000022235E003229A751C765C769C7614E164
:10C5000004229A755A7E997E2244D2B25A760A44FF
:10C510009A76DC7609E105229A755A7E997E224444
:10C52000D2B25A760A449A769C83FEE006229A7525
:10C530005A7E997E2244D2B25A760A449A769A8BCF
:10C5400002EB0424A4B2B4F5AC7F82BF7B4A012184
:10C55000D17500229C83DA83002C40F0E68007220C
:10C560009A75E2E05A7E997E2244D2B25A760A4403
:10C570009A76DA8BB2F5AC7F3EBF7049891881F8A4
:10C5800020400132998B92B29142DA83E7D9CCE014
:10C5900008229A755B7EA34200F0C780674B012298
:10C5A000DA750DE0674D9A7515F8012D6A70664AC7
:10C5B0009542F9D1997E614AA14206D03F232B7062
:10C5C000624A536801335360AFE06148016801314A
:10C5D0000160D07D10B13E232B70A6E0212129708F
:10C5E000D17E062941D004D8022907D0032923D0BF
:10C5F000F8BD122959D0302967D0F8BD5021546AAE
:10C60000297054494C60946A0C60116B4FF47A7431
:10C6100091FBF4F1504C218092F878114F4A19B1F6
:10C62000117841F0020102E0117821F0020111704D
:10C63000012283F8792169E05321297092F82510AD
:10C64000CE0705D592F82420D51E6A426A4100E043
:10C65000024602F0010183F87811002A56D13F49C1
:10C660000A7822F002020A7050E04F21297092F8F5
:10C670002B10CC0705D592F82A20D11E4A424A41F8
:10C6800000E0024602F0010183F8781122B9334933
:10C690000A7822F002020A7093F84F10304A1170A3
:10C6A000B3F84C102F4A118030E05621546B29709A
:10C6B0002D490C8042F21074916B91FBF4F12B4CDC
:10C6C0002180012182F87A1120E04921297092F815
:10C6D0002410274A102988BF102111702549147889
:10C6E0000022A2420ED20E7A234D56554E7A234D89
:10C6F0005655CE7A224D565511F80C6F214D565590
:10C700000132EEE720490A6801320A6093F8793174
:10C710000A4A002B3AD092F87A31BBB3002182F852
:10C72000791182F87A111846F8BD0020F8BD127907
:10C73000432A7FF494AD0222EA7090E52420002081
:10C74000C8280020E80A0020D40A00203002002077
:10C75000EC110020D4100020D0100020CC100020BC
:10C76000D21000204E000020CE10002030100020FB
:10C7700048100020442000204910002059100020BB
:10C780006910002079100020E0110020F8BD044954
:10C79000044B0968002218705A6199611A77704732
:10C7A000C028002030020020F8B5101A0D461F46A0
:10C7B00007F0BAF80446781B07F0B6F8174B079E47
:10C7C000196807F005F921460546204607F000F9EB
:10C7D00029460746284607F0FBF80146384606F08A
:10C7E000EFFF0BF025FA0E4907F0F2F807F0DCFA3C
:10C7F000069B2946186004F100400BF08DF80949AA
:10C8000007F0E6F8084906F0DBFF07F0A7FA002872
:10C81000BCBF00F50C40A0303060F8BD48000020DF
:10C820002C7D8E3FA00CB34500A00C4644F2506313
:10C83000984203DDA0F50C40A0387047034B9842A6
:10C84000BCBF00F50C40A030704700BFB0B9FFFF7F
:10C85000F7B50368174C184D23600B68174E6360DB
:10C860000068FFF79FFC95E80300154B01960093C5
:10C8700094E80C00FFF798FF3668124B60681E6062
:10C880006B68114FC01A07F04FF8104B196807F08A
:10C890009FF807F063FA2A68236878609B1A3B6068
:10C8A0000B4B1E600B4B1B68DA880B4B1A8003B0D6
:10C8B000F0BD00BFA8270020D4100020B42700201E
:10C8C000B0270020F0270020B827002048000020D3
:10C8D000E82700203C0F0020E427002070B5044624
:10C8E000407907F01DF81E4907F026F91D4D1E4E30
:10C8F0002860E07B07F014F8194907F01DF9EE6095
:10C900006860A07907F00CF8184907F015F9184D80
:10C910002860207C07F004F8114907F00DF96860E1
:10C92000A07E06F0FDFF134907F006F9EE60A8604F
:10C93000E07906F0F5FF0D4907F0FEF80E4D28608E
:10C94000607C06F0EDFF064907F0F6F86860E07ECF
:10C9500006F0E6FF074907F0EFF8EE60A86070BD4B
:10C960000000C842C02700200000FA440000204117
:10C97000D027002000007A44F427002010B50C4C8A
:10C9800023789B0713D50B4B1B78042B0FD90A4A2E
:10C990000A4B1068526818605A60FFF703FC084B96
:10C9A0001A88084B1A80237843F00103237010BDC6
:10C9B000CC100020D2100020D41000203410002011
:10C9C000A410002004280020044B1A78044B0AB15C
:10C9D000044A00E0044A1A60704700BF9228002011
:10C9E000982800200000A0410000A0C1164B13B5FC
:10C9F0001B681B0325D5154B154C1B7815498DF865
:10CA00000030154B20681B788DF8013006F0E0FFF0
:10CA100007F0CAF911498DF80200606806F0D8FFE6
:10CA200007F0C2F98DF80300A06807F0BDF90C4BC0
:10CA30008DF804001B780A2069468DF80530FDF753
:10CA40003DFE02B010BD00BF9C2800208E280020B3
:10CA5000B028002000002041AC28002000007A44CB
:10CA600092280020054A137883F001031370044ACA
:10CA700000231360034A1360B8E700BF9228002028
:10CA8000A8280020A4280020094A13781844134637
:10CA9000C0B210F0800F18BF80381070054A1978A6
:10CAA0001378994201BF00231370014A1370704735
:10CAB000092800200828002010B50A4B0A4A1B78D4
:10CAC00042609C18094A046012789A4225BFD31A22
:10CAD0000B60C3F1800300232EBF4B600B604A60E4
:10CAE00010BD00BF092800200A28002008280020C7
:10CAF0001FB5684602A9FFF7DFFF044B02981B68C9
:10CB000003440398184405B05DF804FB400E002070
:10CB10002DE9F04F89B00193002382469946029196
:10CB20000392039A934205DA029A52F823200133C2
:10CB30009144F6E7019B4D46002B56D102F066F971
:10CB4000002852D101987DE00222404E8DF81C2031
:10CB50001A0C4FF480578DF81D2006201A0A8DF804
:10CB60001E208DF81F3002F075F97761062005F060
:10CB700001FD374B01223761D0461A707761264696
:10CB8000002007A9042205F0BFFC029F4FF0000B14
:10CB9000039B9B451EDABC4657F8042B4FEA8B03D8
:10CBA000002A48D0B24236D332465AF80310002049
:10CBB000CDF814C0049305F0A7FC049BDDF814C065
:10CBC0005AF8032032444AF80320DCF800309E1B58
:10CBD000CCF800601D4B4FF480521A611D4A2D1B8A
:10CBE00013681C44019B146053B34DB3194B1B686D
:10CBF000DCB22A19B2F5807F174A88BFC4F5807469
:10CC0000D26898BF2C4693429ED3144A00231370D7
:10CC1000134A137014E00020D8F8001005F074FCDB
:10CC200057F8043CD8F80020F61A1344C8F800302E
:10CC3000002347F8043C0BF1010B08F10408A7E7B7
:10CC4000C5EB090009B0BDE8F08F00BF000C014042
:10CC50003D0E0020400E00200C000020082800207F
:10CC60000928002030B50B4C0B4D22782B7885B06D
:10CC70009A420CD0684602A9FFF71EFF01236846BE
:10CC800002A90222FFF744FF00232B70237005B096
:10CC900030BD00BF092800200828002030B50E4D07
:10CCA0000E4C2A78237885B09A4211D0684602A9A2
:10CCB000FFF702FF002302A902226846FFF728FFC0
:10CCC000FFF7E2FE20782B781B1A5842584100E00B
:10CCD000012005B030BD00BF092800200828002031
:10CCE00038B50E4C4FF4805545F2082002F0B2F8EA
:10CCF0006561062005F03EFC094B01222561C72035
:10CD00001A70656105F036FC064A00232561137030
:10CD1000054A1370054A136038BD00BF000C01407E
:10CD20003D0E00200828002009280020400E002089
:10CD300001480249FEF722BF00080040E02200201F
:10CD400001480249FEF71ABF00040040B822002043
:10CD50004FF080400149FEF711BF00BF9022002034
:10CD600001480249FEF70ABF002C0140682200205A
:10CD700001480249FEF702BF002C01406822002052
:10CD8000034B4FF4805208B11A6170475A617047E3
:10CD900000080140034B4FF4805208B15A617047BC
:10CDA0001A617047000801402DE9F84F2E4E0446E5
:10CDB00037683846FCF706F805463846FBF78FFF1C
:10CDC000766880463046FBF7FDFF83463046FBF72A
:10CDD00086FFD4F8049006462946484606F0F8FD3A
:10CDE000A76882464146384606F0F2FD01465046A5
:10CDF00006F0E4FC21688246584606F0E9FD41460B
:10CE00000446484606F0E4FD314606F0E1FD0146E1
:10CE1000204606F0D5FC31460446384606F0D8FDDB
:10CE2000294606F0D5FD0146204606F0C9FC01461C
:10CE300050460AF071FD0D4906F0CAFD0C4906F096
:10CE40007BFE0C4B196806F0BBFC0B4906F074FE28
:10CE50000AF08AFC83B21A0444BF00F5B47083B2AE
:10CE600018B2BDE8F88F00BFA02100200000E14407
:10CE7000DB0F4940E0180020000020412DE9F04F71
:10CE800087B003939A4B80461B889346980737D503
:10CE900040F2E632109B9748DC89B0F900301B1B4A
:10CEA00003F2F315954203D8002BB8BF5B4201E0B3
:10CEB0004FF4FA73B0F9022040F2E630121B02F28E
:10CEC000F314844203D8002AB8BF524201E04FF461
:10CED000FA729342B8BF13460522C3F5FA7393FB67
:10CEE000F2F30A22643B534398F81C20D2105343B8
:10CEF000642293FBF2F3134423EAE373DBB200E012
:10CF00006423C1460093CB1C02930025029B022D93
:10CF100013F8016F784F02934FEA450A05D1B7F92C
:10CF200004301B365E43761149E0744B37F9152007
:10CF300033F9153003EB4202CBF100039A4203DBD5
:10CF40005A451346A8BF5B466D4A32F90A40039A18
:10CF50001B1B32F915402344019306F015FA019B7F
:10CF600088B1684A1846545D06F0DEFC664906F052
:10CF7000E3FD0146204605F03FFB634906F028FD2E
:10CF800006F0ECFE03465A4A1288D10713D437F94B
:10CF90000A401B36664392074FEA26160FD598F8CB
:10CFA00012409DF9002063435343642293FBF2F344
:10CFB00006EB231603E098F808405C432611534B18
:10CFC000042433F90A3099F8017093FBF4F4341B0C
:10CFD0004F4E674306F10803EB5C98F851205F431E
:10CFE0000193642397FBF3F7FF117AB1384604925B
:10CFF00006F09AFC06F10C030C2101FB0531049AA2
:10D00000336BFBF7FDFB06F0A9FE0746414B99F891
:10D010000B6019883E4B01FB04F203F1340E5EF8FD
:10D020002500D21206FB02063B4AB6F5001FA8BF38
:10D030004FF40016964203F14000B8BF164650F870
:10D04000252040F825404FF6FF700909B0FBF1F1AB
:10D05000A21A4A4303F14C0103F158044EF825602B
:10D0600051F825E054F8250044F825E098F85040A0
:10D07000921170444FEA850C7613104441F8252034
:10D0800094B1CDF810C0059306F04EFC059B0C2121
:10D0900003F1640201FB05211B6B2246FBF7B0FB89
:10D0A00006F05CFEDDF810C099F81530BA19584347
:10D0B000019B013543431846642390FBF3F0174B63
:10D0C0000012024423F80A2003F108024CF802700F
:10D0D000032D03F1140203F120034CF802604CF815
:10D0E000030009F101097FF411AF07B0BDE8F08F2B
:10D0F0008C110020D8280020AC100020E033002044
:10D100009428002088A5010800002041E80F002095
:10D11000A0210020C40F00200000E0FF28220020F2
:10D120001FB5084B1B681B0309D58DF8040003913C
:10D1300001230D2001A98DF80530FDF7BFFA05B0D8
:10D140005DF804FB9C2800201FB5084B1B681B03DF
:10D1500009D58DF80400029100230D2001A98DF856
:10D160000530FDF7ABFA05B05DF804FB9C28002004
:10D1700010B50A4A0A4B11689B6812689142F8D1AF
:10D18000084A4FF47A70D2F8B44000FB04F2D31A84
:10D19000B3FBF4F300FB013010BD00BFC02800203A
:10D1A00010E000E0A021002038B50446FFF7E0FFC2
:10D1B0000546FFF7DDFF401BA042FAD338BD10B58E
:10D1C00004462CB14FF47A70FFF7EEFF013CF8E70C
:10D1D00010BD024A1368013313607047C028002055
:10D1E00010B50024044B53F8243003B198470134A0
:10D1F000032CF7D110BD00BFA0180020014B1B6805
:10D20000184700BFCC33002010B50020FFF7F6FF11
:10D21000074B00241C7006F093F8064B83F8B840C7
:10D22000C3F8BC40A3F8C040C3F8C44010BD00BF61
:10D230008B330020A021002010B510B9BDE81040AC
:10D24000E2E700230C225A430C4C1119125D824272
:10D2500003D00133102BF5D110BD094BD3F8C40016
:10D2600018B14A784078824206D20022C3F8C4102E
:10D27000A3F8C020C3F8BC2010BD00BF9CAC0108BF
:10D28000A021002010B540001428A8BF14200023BE
:10D29000074A022199540B4499181424834201F837
:10D2A000014CF5DBFF21D1540F20BDE81040C3E74E
:10D2B0002427002038B540F2DB156843134B1022B9
:10D2C0005A6108221A61851E0B24013C14F0FF04E8
:10D2D00015D00E4B2846DA6882F01002DA60DA6860
:10D2E00082F00802DA60FFF76AFF0120FFF786FF8D
:10D2F0001920FFF764FF0020FFF780FFE5E7044AED
:10D30000044B1A60044A054BDA6038BD000C01403A
:10D31000EFBEADDEF04F00200400FA0500ED00E0A6
:10D32000074B1A6832B15A681AB19A682AB90222B0
:10D3300000E0012243F8220070470F20BAE700BF47
:10D34000A018002003685B69184703681B69184729
:10D350000368DB68184703689B68184703685B68C5
:10D36000184703681B681847B0F902302DE9F74FDA
:10D3700093421CBF0023037090F800A004460E46A1
:10D380009146BAF1000F40F0AB80104606F0CCFA9F
:10D39000864906F01DFB864906F01AFB4FF07C51CA
:10D3A00006F016FB0AF040FA0146054606F010FBAF
:10D3B00080498346284606F00BFB0346584619462B
:10D3C000019306F0FDF94FF07E5106F0F9F90146A0
:10D3D0004FF07E5006F0B0FB2946804606F0F8FA82
:10D3E000294606F0F5FA07460146606006F0E8F9BE
:10D3F000E7604FF07E572946A0602761284606F077
:10D40000DFF9294606F0E4FA4FF0804106F0D6F93C
:10D410000146404606F0DCFA019B60611946584619
:10D4200006F0CCF9394606F0CBF90146404606F045
:10D43000CFFA40F2DC53A0462746554663651023D9
:10D44000A4F852301823A061A4F850304FF097414F
:10D45000D8F8100006F0BCFA0021824606F056FC0F
:10D4600028B150464FF07C5106F0A8F904E0504630
:10D470004FF07C5106F0A4F906F0D2FCC7E90E018A
:10D480004FF09741D8F8040006F0A2FA0021824636
:10D4900006F03CFC28B150464FF07C5106F08EF966
:10D4A00004E050464FF07C5106F08AF906F0B8FCD3
:10D4B0000135032DC7E9080108F1040807F1080741
:10D4C000C4D1A6F2DC531B042367E3676367C4F887
:10D4D0008030A367C4F884300123A4F8029023703D
:10D4E000D4F85490B4F95280C9EB0606636A06FA80
:10D4F00008F67343276A4FEAE67B206F07FB0B337E
:10D500002667A7FB0667E26F1F44636CD4F840C030
:10D5100053434FEAE27B0CFB0B3ED4F88010C4F877
:10D520008020ACFB02237344B61A67EB0307E36A5F
:10D53000A26A43434FEAE07B02FB0B3EA2FB0023BF
:10D540007344B6185F41E36C656F4B436067A06C32
:10D550004FEAE17B00FB0B33C4F88410A0FB010110
:10D560001944636B361A05FB03F3206B4FEAE57B26
:10D5700000FB0B3367EB0107A0FB05018019194481
:10D580007941B4F95020A56706F006F908F1FF3299
:10D5900001239340E067C01841EBE371424606F077
:10D5A000FBF8484403B0BDE8F08F00BF6F12833A28
:10D5B000DB0F4940F404B53F2DE9F0410024234B33
:10D5C000E0B21E78B0420CD2214B33F81010214B40
:10D5D00053F820301BB10B2801D8DB689847013481
:10D5E000EDE71D4B1B685B032ED500242346E2B2FA
:10D5F000B24229D2174F4FEA840857F824205568C1
:10D600009D4219D02846FEF77BFBEFF31283502290
:10D6100082F3128811494FF0280EAA8C0EFB0010DD
:10D6200092B20132C0F8EC20AA8ADBB292B242F088
:10D630000102AA8283F3118857F8083000221B6880
:10D6400001341A802B46D2E7BDE8F081E0260020A5
:10D6500008100020E42600209C280020A0210020A3
:10D6600008B50E4B1B6813F4805F0D4B14BFD3F845
:10D670006831D3F86C319A880A4B19780023D8B2F4
:10D68000884204D2084820F813200133F7E7FFF757
:10D6900093FFBDE80840322091E500BF9C280020A0
:10D6A000A0210020E0260020081000200A4B30B501
:10D6B0001A680A4B02F48052D3F86841D3F86C51CF
:10D6C00000230AB1A18800E0A988054820F81310BA
:10D6D00001330C2BF5D130BD9C280020A021002067
:10D6E000C226002070B5124D0024214605F27110AB
:10D6F000702285F8704109F02AFE2146D5F8E43100
:10D700000B4A0B4493F9020088B11E6802F27114AF
:10D710000E5108199C88073184809B797029837188
:10D7200092F8703103F1010382F87031E6D170BDD7
:10D73000A0210020094B1A680E2303FB0020437A26
:10D74000FF2B07D0064A12789A4203D9054A32F8CD
:10D75000130000E0808800B2704700BF2C24002036
:10D7600088330020D82800202DE9F04F91B0FFF732
:10D77000FFFC8C4C0546D4F8E8614FF00008831B91
:10D780001846019306F0CCF8D4F8EC11029006F09C
:10D790001FF9C4F8E8514546D4F8F071824E97F865
:10D7A00000B00390814A0DF11C0A32F9150006F011
:10D7B000BBF8039906F00CF94AF82500BBF1000FFD
:10D7C0002BD0584606F0B0F801464FF07E5006F0D8
:10D7D000B3F90246DFF8009211464FF07E500592F1
:10D7E00005F0ECFF59F8251006F0F2F809F10C01EC
:10D7F000049031F9150006F097F8059A114606F0E5
:10D80000E7F8DDF810C00146604605F0D9FF49F899
:10D81000250006F0A3FA708003E0654A32F815206F
:10D82000728036F9022F0135032D02FB0288B9D12F
:10D83000642303FB08F85F4B5F481B8807A95B4321
:10D8400098FBF3F8A8F149081FFA88F8FBF738FBB2
:10D85000B8F13B0F7D6810D9524BB3F91402D3F8DD
:10D86000105206F061F80146284606F06DFA534B57
:10D8700068B31A7842F008022CE04FF07E51284637
:10D8800005F09EFF01464FF07E5006F055F98146A7
:10D890004FF00008DFF820B128465BF8281006F0AA
:10D8A00097F8474A039032F9180006F03DF8039BB9
:10D8B0000146184605F084FF494606F089F84BF802
:10D8C000280008F10108B8F1030FE3D1C4E71A7882
:10D8D00022F008022946D4F80C021A700AF01CF84B
:10D8E00081462060D4F80802D4F810B200F1004557
:10D8F000D4F80C02014606F06BF8594680465846AB
:10D9000006F066F80146404605F05AFF0AF090F925
:10D91000014628460AF000F82A49804660604846D9
:10D9200006F056F809F020FF274D2649288040468A
:10D9300006F04EF809F018FF244B68801B681B079F
:10D940004CD5234807A9FBF7BBFABD684FF07E51C1
:10D95000284605F035FF01464FF07E5006F0ECF802
:10D9600082464FF0000B1A4B284653F82B100493B5
:10D9700006F02EF81749039031F91B0005F0D4FF8B
:10D98000039A0146104605F01BFF514606F020F8A9
:10D99000049B43F82B000BF1010BBBF1030FE2D109
:10D9A000184652E0A021002094100020E80F00202B
:10D9B000A02300201C000020A8230020CC10002061
:10D9C000961000204C3D0F4494280020C8100020E1
:10D9D000B8230020EE0F0020942300206C4D514608
:10D9E0002846FBF76DFA28686B680146039305F03B
:10D9F000EFFF039B82461946184605F0E9FF0146F2
:10DA0000504605F0DDFED5F808B082465946584626
:10DA100005F0DEFF0146504605F0D2FE0AF008F997
:10DA20000021824606F068F970B92868514606F070
:10DA300083F851462860686806F07EF851466860B1
:10DA4000A86806F079F8A8605148FFF7ADF9514B86
:10DA500051491880029805F0BBFF4E4B08F1004871
:10DA6000054609F10049B3F90000CDF82C80CDF846
:10DA7000289005F059FF494900F1004005F0A8FF42
:10DA8000DFF82C810C90B8F9000005F04DFF0D90E7
:10DA9000B8F9020005F048FF0E90B8F9040005F04F
:10DAA00043FF0AA90F900DA8FBF70AFA7B78012B18
:10DAB0001AD13B4B3B4F1B7813F0040F0ED1D7F814
:10DAC0002402402390FBF3F3C01A05F02DFF0F99B9
:10DAD00005F076FE06F042F9C7F82402D7F82402D2
:10DAE000402390FBF3F001E02F4B188805F01CFF5A
:10DAF00001460F9805F062FED4F82C120F902846CC
:10DB000005F05EFE0146284606F016F8D4F82872A5
:10DB1000054639460F9805F051FE0146284605F0A6
:10DB200057FF0146384605F04BFE0746C4F8280269
:10DB30000D9809F019FED4F830522978FBF7C0F897
:10DB4000D4F834321844C4F834020E9809F00CFEAC
:10DB50002978FBF7B5F8D4F838321844C4F83802FD
:10DB6000384609F001FE6978FBF7AAF8D4F83C3290
:10DB70000E4A184401991368C4F83C021944D4F8B9
:10DB8000403211600133C4F8403211B0BDE8F08F6B
:10DB900024000020A4100020BD37863535FA8E3CC5
:10DBA000E5330020A02100201C000020C833002005
:10DBB0009610002001380A4B042804D8DFE800F052
:10DBC0000507090B0D00074A08E0074A06E0074A67
:10DBD00004E0074A02E0074A00E0074A1A6070477B
:10DBE00054000020A5FE00087DCE0008AD330108DA
:10DBF00067FB0008D1F7000835F2000838B50024AB
:10DC00000B4D6059254403F0EBF9696811B10948DF
:10DC1000FBF736F8A96811B10748FBF731F8074858
:10DC2000103403F0DDF9B4F5F07FE9D138BD00BF61
:10DC30008CA50108EEC40108F4C4010829CF01082D
:10DC400070B50546284609F0C6FB064658B91A4B7A
:10DC50001A485A791A4BBDE8704003EB8203D3F897
:10DC6000DC11FBF70DB828461649324609F0BCFB1B
:10DC700060B9154803F0B4F9144C54F8041F19B1F5
:10DC80001348FAF7FDFFF8E7124805E00024124BAD
:10DC900053F8241021B91148BDE8704003F0A0B931
:10DCA0002846324609F0A0FB01340028EFD1024B90
:10DCB0000B4D5C71C6E700BFFC280020FAC40108C8
:10DCC0008CA5010806C501080BC5010868A7010855
:10DCD0001EC5010829CF01086CA70108C6C20108AA
:10DCE0001CC00108F0B585B0044609F074FB082893
:10DCF00026D1621EE01D1F4912F8013F0968194430
:10DD0000497801F00301022908BF203B82421370C9
:10DD1000F1D1254604F1080715F8016B1648314684
:10DD200009F04BFB20B12846314609F046FB10B103
:10DD3000F9F724F91CE0BD42EED12046FDF776F953
:10DD40000E4803F04DF900230D4A04A91A4492F835
:10DD500088210A440849595C0133082B02F80C1C3D
:10DD6000F2D10023074801A98DF80C30FAF788FF9B
:10DD700005B0F0BD600000205ED9010822C5010891
:10DD8000FC280020CDCD01082A4B2B4C1E6880B505
:10DD90002068F9F797FC3046F9F794FC2068417940
:10DDA0008D0703D441F00201FFF7CCFA234B082280
:10DDB0001A61234D10221A612B689A0341BF062372
:10DDC0006371E37923F0010344BF43F00203E3717D
:10DDD0002068FFF7C3FA90B1184F08237B61164BF8
:10DDE0001868FFF7B8FA8046FEF7FAF908B103F0B1
:10DDF00065FC30464146FFF7B4FA08233B613046E4
:10DE0000FFF7ACFA78B10D4F4FF01008C7F8148047
:10DE10003046D4F80090FFF79EFA01464846FFF7D7
:10DE2000A0FAC7F810802B689B03D1D5FAF7C6F883
:10DE3000CEE700BFDC260020E4230020000C0140D8
:10DE40009C2800202DE9F047054609F0C4FA2F4E22
:10DE50000446D6F8088090B92D4803F0C1F82D4B40
:10DE600053F8241049B10123A34013EA080F02D04C
:10DE70002948FAF705FF0134F1E7284822E028464F
:10DE80002749224609F0B0FA58B9264803F0A8F805
:10DE9000254C54F8041F0029EFD01F48FAF7F0FE74
:10DEA000F7E72B784FF000092D2B03BF013504F164
:10DEB000FF344FF0010A4FF0000A164B53F8297057
:10DEC00027B91A48BDE8F04703F08AB82846394612
:10DED000224609F089FAA8B9012000FA09F0BAF13E
:10DEE000000F03D0FBF760F8114803E040EA080098
:10DEF000B060104803F074F83946BDE8F0470E48AA
:10DF0000FAF7BEBE09F10109D7E700BFFC280020DF
:10DF100028C50108D4A701081EC5010829CF01089A
:10DF200006C5010832C50108D0A70108C6C201080C
:10DF30003EC5010847C50108CCCD010810B5084809
:10DF400003F04EF8074B00241C741C64064B1C7035
:10DF5000FFF7ACFB03F0B6FA044B1C6010BD00BF2A
:10DF60004FC50108E4230020E9330020DC2600200F
:10DF700070B5064600240A4BE518AA8816420AD056
:10DF8000E1580848FAF77CFE2846002102F0B9FF64
:10DF9000054803F025F81434B4F5486FEBD170BD93
:10DFA0003CAE01087BC5010829CF010808B5084827
:10DFB000FAF766FEFEF794FE00F028FF18B9642019
:10DFC000FFF7FDF8F8E70348BDE80840FAF758BE48
:10DFD00085C5010892C501082DE9FF410A48068858
:10DFE00085684488B0F80480C768FEF781FDCDF8E5
:10DFF00000800290019731462A4623460348FAF7EB
:10E000003FFE04B0BDE8F0810C0000209AC5010875
:10E01000F0B504788BB005460CB1002436E04A4BCD
:10E0200019680E2303FB0411B1F91D51B1F919212F
:10E03000B1F91B31009591F8205101F58C700195D3
:10E0400091F8215101F59071029590F90700039024
:10E0500091F902103D48049121460134FAF710FE6F
:10E06000082CDCD16DE02D2B14D1072C1BDC2846AD
:10E0700009F006FA0AAB661C03EB440424F8100C02
:10E0800015F8013F303B092BFAD934462B78002B89
:10E09000E9D104E0A3F13002092A09D8E5E7082C08
:10E0A000BDF8182009D00BB0BDE8F040F8F766BF06
:10E0B000202BF8D101352646E7E7072AF3D840F2AE
:10E0C000DC55BDF81A00204BA0F2EE2189B2A9421E
:10E0D0001B68E8D8BDF81C10A1F2EE24A4B2AC4233
:10E0E000E1D8BDF81E7004B23EB2A642DBDB0DB231
:10E0F000AE42D8DCA542D6DBBDF92440642CD2D197
:10E10000BDF8266034B2112CCDDCBDF82050B42D02
:10E11000C9D8BDF82240B42CC5D812B24FF00E0EAB
:10E120000EFB0233A3F81B116421A3F81901A3F815
:10E130001D7183F8205183F8214183F81F1183F862
:10E1400022610BB0F0BD00BF04100020F7C501082C
:10E15000F0B504468FB0204609F03DF9C5B21DBBAD
:10E16000AB4802F03DFFAB4C94F8D61009B9AA4871
:10E1700053E049B294F8D42094F8D530009194F843
:10E18000D710A648019194F9D8100734029194F958
:10E19000D210039194F8D310049129460135FAF76F
:10E1A0006FFD102DE0D1E2E720469D49052209F0E0
:10E1B0001BF90546B8B929469A48702209F0C7F8F4
:10E1C0002846994B19680E2303FB001301300022E7
:10E1D000082883F8232183F8242183F8252183F854
:10E1E0002621F0D112E120469049042209F0FCF8E2
:10E1F00005462046002D4AD1202109F0DEF80028EE
:10E2000000F00481461C304609F0E5F82C4607462C
:10E21000874B53F824502DB986480FB0BDE8F04025
:10E22000FAF72EBD30462946FAB209F0DDF801347E
:10E230000028EDD1774A164602F17001002382F8DA
:10E24000DA3082F8D63082F8D53082F8D43007320E
:10E250008A42F3D1784901EBC40191F8A02293429C
:10E2600010DAD1F8A472C3EBC302B0183A441768AD
:10E2700000F1D401C0F8D47090880133888092797D
:10E280008A71E7E729466D48FAF7FAFC8FE06C4996
:10E29000072209F0A9F805462046002D49D1202182
:10E2A00009F08BF8064609F096F8C4B26CBB6548D5
:10E2B000FAF7E6FC214664480134FAF7E1FC0E2C3B
:10E2C000F8D15548FAF7DCFC002460482146FAF7FB
:10E2D000D7FC0025544A012311680E2202FB0412C8
:10E2E000D2F82321AB401342594B5A495A4808BF30
:10E2F00019460135FAF7C4FC0E2DEBD1464801341E
:10E30000FAF7BEFC082CE0D180E03046534909F012
:10E31000BBF82C4600284CD0022C4FD009F0B0F8A6
:10E3200006AB43F824004D49002009F0ADF8013454
:10E33000F0E74A4909F0A8F8002460B1082C38D069
:10E3400009F09EF806AB43F824004449002009F088
:10E350009BF80134F1E7082C2BD1069B0F2B28D812
:10E36000DDF81CE0BEF1070F23D8089F0D2F20D841
:10E37000099E06F16402C82A1BD80A9DFF2D18D8F1
:10E380000B98642815D80C99642912D8884210DAA1
:10E390000D9C032C0DD8324AC3EBC303134483F8FE
:10E3A00004E05F719E71DD71187259729C722D4C80
:10E3B000D1E60FB0BDE8F040F8F7E0BD069B072BB3
:10E3C00020D807990D291DD80278722A0DD06E2AFF
:10E3D00018D1154A0E20126800FB032301228A403F
:10E3E000D3F8231121EA020209E00F4A0E20126835
:10E3F00000FB032301228A40D3F823110A43C3F808
:10E40000232101E0F8F7BAFD0D4CA4E60FB0F0BDF2
:10E410001FC60108FC28002029CF01084AC60108B0
:10E4200096C20108D029002004100020C1C20108B2
:10E430006CA70108C6C201088CA50108D5C2010855
:10E4400017C60108F8C4010866C6010831C40108EE
:10E450005ED20108A4D101086BC601086FC601088D
:10E46000CC2900201CC001082DE9F743047805469B
:10E470008CB9324D95F8A312B5F8A02295F8A232C6
:10E480002F48009121460134FAF7FAFB102C05F1D0
:10E490000405EFD14FE008F0F3FF0F28044636DC07
:10E4A0002846202108F089FF264EE4B2D6F84480A1
:10E4B000451CA4000027284608F0E2FF5FFA87F910
:10E4C000B9F1010F83B208D0B9F1020F0BD0B3F547
:10E4D000B47F25D2726C13530AE0FF2B20D8736CE3
:10E4E0002344987004E0FF2B1AD8736C2344D8702F
:10E4F00028462C2108F061FF054608B1013502E0ED
:10E50000B9F1020F0CD10137032FD4D113E00E481B
:10E510000E4900220F2303B0BDE8F043FAF7B0BB69
:10E5200008EB04000021042208F011FF03B0BDE84D
:10E53000F043F8F723BD03B0BDE8F083FC280020CA
:10E5400071C60108E423002035C2010854C2010845
:10E550002DE9F04FAC498BB0044608F001FFAB4900
:10E56000002820460CBF0125072508F0F9FEA84920
:10E570000028204608BF022508F0F2FE002808BF48
:10E580000425E90740F1FB80A24802F029FD0020A4
:10E5900002F032FBA04CA14802F022FDA04802F09C
:10E5A0001FFD62799F4BA04803EB8203D3F8DC1177
:10E5B000FAF766FB9D48FAF763FB26460027D6F874
:10E5C00014800021404605F097FB20B19848FAF7E7
:10E5D00057FB002669E039469648D6F818B0D6F8B9
:10E5E0001CA0D6F82090FAF74BFB4046002105F01E
:10E5F0008DFB10B1202002F0EBFC06A94046FAF793
:10E60000C5F901468C48FAF73BFB5846002105F056
:10E610007DFB10B1202002F0DBFC06A95846FAF77A
:10E62000B5F901468448FAF72BFB5046002105F066
:10E630006DFB10B1202002F0CBFC06A95046FAF782
:10E64000A5F901467C48FAF71BFB4846002105F076
:10E650005DFB10B1202002F0BBFC06A94846FAF78A
:10E6600095F9013701467548FAF70AFB0C2F06F1B8
:10E670001006A4D1AAE749B294F8D42094F8D53072
:10E68000009194F8D7106E48019194F9D81007348E
:10E69000029194F9D210039194F8D3100491314669
:10E6A0000136FAF7EDFA102E03D094F8D6100029AF
:10E6B000E1D100260E2777430024624A0123926CA1
:10E6C000A3403A44D2F80A20134240F09480013427
:10E6D0000E2CF2D10136082EECD15B4802F080FC02
:10E6E0004D4B5A4C9F6854F8041F19B15848FAF71B
:10E6F000C7FAF8E70E46574B53F826404CB10123B2
:10E70000B3403B4203D054482146FAF7B9FA0136E8
:10E71000F1E7524802F064FC21463F4B0AAA0B4441
:10E7200093F8883113444E4A8A5C0131082903F872
:10E73000102CF2D1002306A94A488DF82030FAF7B0
:10E740009FFA494802F04CFC4848F9F757F8484806
:10E7500002F046FC4548F8F717FC464802F040FC3A
:10E760004248FFF781FE4448FAF78AFA4020FFF753
:10E77000FFFB424802F034FC3C48F8F73BFFAA0795
:10E7800026D53F4802F02CFC3E4802F029FC3748D1
:10E7900002F072FA3C4802F023FC3448F8F775FBAB
:10E7A0003A4802F01DFC3148F8F774FE3848FAF791
:10E7B00067FA2E48F8F7F6FC364802F011FC2B48B1
:10E7C000FFF726FC2C48FAF75BFA8020FFF7D0FB16
:10E7D0006B0716D5304802F003FC304802F000FC0D
:10E7E000224802F023FA2448FAF74AFA4FF48070DC
:10E7F000FFF7BEFB05E0314622462948FAF740FA0A
:10E8000065E70BB0BDE8F08F85C60108F9CA0108BD
:10E810008CC6010892C60108FC280020A0C6010889
:10E82000B2C601088CA50108BEC60108C9C6010808
:10E83000D6C60108E3C60108F7C40108CDCD01081A
:10E84000EBC60108E42300200AC70108D0A701088D
:10E850001AC70108D4A7010828C7010835C701084D
:10E860005ED9010841C701084AC701081CC0010858
:10E8700059C7010865C7010829CF010873C70108F6
:10E8800080C7010893C70108A1C70108ABC70108E9
:10E89000BAC70108C8C70108D4C70108E5C70108FD
:10E8A000F7C7010837B50622044603216B461E2030
:10E8B000F5F748FA9DF801309DF80000154D43EA40
:10E8C000002000B205F030F8296805F081F805F065
:10E8D00045FA9DF8033020809DF8020043EA0020AD
:10E8E00000B205F021F8A96805F072F805F036FAD3
:10E8F0009DF80530A0809DF8040043EA002000B296
:10E9000005F012F8696805F063F805F027FA6080F1
:10E9100003B030BD3000002010B5054C23681869E5
:10E9200001F096FF18B123681A69024B5A6110BDB5
:10E93000D41800200004014038B50D4B0D4D9968E6
:10E940000D4B1A681C465288114203D0FEF710FC8A
:10E95000286007E0FEF70CFC2B68984282BFC01AC3
:10E96000064B186023685A68054B5A6138BD00BFD2
:10E97000000C0140302400202C0200200000002068
:10E9800000040140084A13689B020BD5074B002185
:10E9900019704FF6FE730649086803400B604FF488
:10E9A00000135360704700BF00000240E4330020B2
:10E9B0006C0002402DE9F047664D6B686649581CB3
:10E9C0000A788E4602F0FF060AB10346F6E737469C
:10E9D0006B60687CEB6895F81080AA7C39B22029BE
:10E9E00000F09C80DFF880C10CEB8103DC789B7821
:10E9F0003CF82110C3F1FF039BB2002B65D04FF010
:10EA00003C0CB1FBFCF9C3F1FF0363431B12B9F1EA
:10EA1000050F5DD8DFE809F0030B1A293A4AE01A1E
:10EA20004143B1FBFCF0DAB21044C0B251E0B1FB9B
:10EA3000FCF00CFB101189B2DAB2C1F13C01E31A0F
:10EA40004B43B3FBFCFC204694442CE0B1FBFCF0B0
:10EA50000CFB1011E21A89B24A43B2FBFCF25FFAD6
:10EA600083F84244D2B2204632E0B1FBFCF90CFB01
:10EA7000191189B2E01AC1F13C014843B0FBFCF026
:10EA80005FFA83F84044C0B2224621E0B1FBFCF8B3
:10EA90000CFB1811D8B289B2E31A01FB03F2B2FBE6
:10EAA000FCFC224684445FFA8CF412E0B1FBFCF8D3
:10EAB0000CFB181189B2D8B2C1F13C01E31A4B43E7
:10EAC000B3FBFCF20244D2B203E02246204600E04F
:10EAD00044464FEA042C4CEA004C4CEA020C172343
:10EAE0004FF0010808FA03F806F1170118EA0C0FB5
:10EAF000A1EB0301DFF8748014BF4FF011094FF050
:10EB0000090989B213F1FF3308F80190E8D21836E9
:10EB10000137B6B2BFB2114BA0465FE7EB600123ED
:10EB20008EF8003040F22A33AA740D4A69810D49EB
:10EB300085F8108068742E81536000238B840B88C5
:10EB40009BB243F001030B80136843F00103136091
:10EB5000BDE8F08730240020E4330020402400206A
:10EB60006C00024000040040CA080020E90A0020AE
:10EB700001F0030301F0FC0101F1804101F5803156
:10EB800010B59B008C680F229A4024EA02028A602A
:10EB90008A68984002438A6010BDF0B5B1F800E081
:10EBA00000234EFA03F2D50725D58E784FEAD30C11
:10EBB000F40648BFCC7806F00F0203F0070748BF01
:10EBC0002243BF0050F82C500F24BC4025EA040417
:10EBD000BA402243282E40F82C2005D1C4680122D7
:10EBE0009A4024EA020205E0482E04D1C4680122BA
:10EBF0009A402243C2600133102BD2D1F0BD2DE9DF
:10EC0000F0437A4A87B01368904693B11A681AB1F4
:10EC10007749886902438A619A889868ADF800202C
:10EC200002228DF80320694604228DF80220FFF7A6
:10EC3000B4FF3220FEF7C3FA002111221E20F5F79F
:10EC400097FA012160221E20F5F792FA6420FEF760
:10EC5000B6FA002402A8FFF725FE274626460A2515
:10EC6000022101221E20F5F783FA3220FEF7A7FACF
:10EC700002A8FFF717FEBDF90820BDF90A101444D9
:10EC80008A42A8BF0A46BDF90C300F4493421E4485
:10EC9000A8BF134613F5805F09DD564A013DD368CE
:10ECA00083F01003D360DBD14FF0010901E04FF096
:10ECB00000091E2000211222F5F75AFA0A25022126
:10ECC00001221E20F5F754FA3220FEF778FA02A846
:10ECD000FFF7E8FDBDF90820BDF90A10A41A8A4221
:10ECE000A8BF0A46BDF90C307F1A9342A6EB030673
:10ECF000A8BF134613F5805F07DD3E4A013DD36888
:10ED000083F01003D360DAD101E04FF00009204610
:10ED100004F00AFE0146384804F00EFF374D20F09B
:10ED200000402860384604F0FFFD0146324804F0F8
:10ED300003FF20F000406860304604F0F5FD014616
:10ED40002F4804F0F9FE20F00040A8600021702256
:10ED50001E20F5F70DFA012120221E20F5F708FAF2
:10ED60001E2002210022F5F703FA6420FEF727FA9D
:10ED7000B9F1000F04D14FF07E532B606B60AB6094
:10ED8000D8F80030194E1A7B62B31A7D52B3184975
:10ED900000258A69012442F001028A61187B197DED
:10EDA000FFF7E6FE1748FEF7BBFA3368164A1B6901
:10EDB00004A8536104930C238DF815308DF814507A
:10EDC0008DF8164001F014FD336801A85B7D8DF8C5
:10EDD00006508DF8043003238DF805308DF8074078
:10EDE00003F074FB07B0BDE8F08300BFD418002027
:10EDF00000100240000C014000406F46300000202F
:10EE000001C05E4619E90008000401400F4B73B5CC
:10EE100018781C4698B105230D4D8DF800304FF43D
:10EE2000805600238DF8013001A86E6169460222E8
:10EE300003F06AFB2E619DF8050000F0010000F070
:10EE40000100207080F0010002B070BD3D0E002076
:10EE5000000C0140064B70B506461C461D68FFF7C6
:10EE6000D5FF18B923685B1BB342F8D970BD00BF4A
:10EE7000C0280020F7B503238DF80430030C8DF86B
:10EE800005308DF80700030A06200F4614468DF85A
:10EE90000630FFF7DFFF78B1084D4FF4805601A927
:10EEA00004226E61002003F02FFB38460021224629
:10EEB00003F02AFB20462E6103B0F0BD000C014098
:10EEC000024640213C20F5F753B970B500EB8000B5
:10EED000094CA0F1A1059C3825440444074B15F8C2
:10EEE000010F1E787040FFF7EBFFA542F6D13046C8
:10EEF000BDE87040E4E700BFBCA90108EA33002088
:10EF000010B5441E14F8010F10B1FFF7DEFFF9E74A
:10EF100010BD024680213C20F5F72AB910B5D42057
:10EF2000FFF7F7FF8020FFF7F4FFA820FFF7F1FFBE
:10EF30003F20FFF7EEFFD320FFF7EBFF0020FFF7A6
:10EF4000E8FF4020FFF7E5FF8D20FFF7E2FF1420E8
:10EF5000FFF7DFFFA120FFF7DCFFC820FFF7D9FF95
:10EF6000DA20FFF7D6FF1220FFF7D3FF8120FFF74B
:10EF7000D0FFCF20FFF7CDFFD920FFF7CAFFF12048
:10EF8000FFF7C7FFDB20FFF7C4FF4020FFF7C1FFFB
:10EF9000A420FFF7BEFFA620FFF7BBFFAF20FFF7BF
:10EFA000B8FFA620FFF7B5FFAE20FFF7B2FF202085
:10EFB000FFF7AFFF0020FFF7ACFFB020FFF7A9FF7E
:10EFC0004020FFF7A6FF0020FFF7A3FF1020FFF768
:10EFD000A0FF4FF48064013C0020A4B2FFF770FF53
:10EFE000002CF8D18120FFF794FFC820FFF791FF94
:10EFF000AF20FFF78EFF012010BD08B55038C0B21A
:10F00000FFF787FF0020FFF784FFBDE808401020CE
:10F010007FE710B504465039C8B2FFF77AFF04EB1A
:10F020004400400000F00E00FFF773FF062060432D
:10F03000BDE81040C0F3031010306AE7012828BF74
:10F0400001202DE9F04F0646734F142000FB067196
:10F05000724BD1F8A4421E765C61714BD1F8B42298
:10F06000DD69B1F8AC822A43DA61A288B1F8AEA2B8
:10F0700022F44072D1F8A852120489B0120C4AEA64
:10F080000809A28003A9C5F8109002228DF80E008D
:10F0900028460193ADF80C908DF80F20FFF77DFD09
:10F0A000019B00971F464FF0080BAA6818EA020F51
:10F0B00003D10A20FEF778F8F7E70A20C5F8148094
:10F0C000FEF772F8C5F810800A20FEF76DF8BBF164
:10F0D000010BEAD1C5F814A00A20FEF765F8C5F8BF
:10F0E00014800A20FEF760F8C5F810800A20FEF7A9
:10F0F0005BF80222C5F810A0284603A98DF80F205E
:10F100001C228DF80E20ADF80C90FFF746FD454A05
:10F1100003A894423A690BBF42F4001242F4800201
:10F120003A613A610BBF3A693A6922F4001222F45B
:10F1300080023A61A38823F440731B041B0CA38054
:10F1400023889BB243F001032380A58801F0E2F9F4
:10F150000599354B25F03F05B1FBF3F32D042D0C3C
:10F160001D43ADB2A5802288002522F001021204C1
:10F17000120C22802D4A03A8B1FBF2F100298AB2B9
:10F1800008BF012242F400414FF4967253434FF4FA
:10F190007A7293FBF2F301339BB22384A183238819
:10F1A000009A9BB243F001032380238823F48163F8
:10F1B00023F002031B041B0C23804FF480432381A4
:10F1C000142303FB062696F8B13201248DF80C3087
:10F1D0008DF80D508DF80E508DF80F4003F076F934
:10F1E00096F8B0329DF80F208DF80C308DF80D5048
:10F1F0008DF80E501AB103A803F068F908E05A0917
:10F2000003F01F039C4002F12003094A42F8234007
:10F2100009B0BDE8F08F00BFBCA901083024002070
:10F22000001002400054004040420F00804F120086
:10F2300000E100E02DE9F04F054690F850008DB058
:10F2400008910592099318B13228A8BF322000E036
:10F25000012004F069FB0146AA4804F06DFCAA4BAA
:10F2600004461888002808BF012004F05DFBA74968
:10F27000069004F0ADFB01900199204604F0A0FA3D
:10F280000146019804F058FCA14B07901B889A078F
:10F2900024D5A049B1F90030B1F9020083EAE37244
:10F2A00080EAE071A2EBE372A1EBE07191420C46BF
:10F2B000B8BF1446B4F5E17F12DA914203DD0028AD
:10F2C000D8BF404203E0002BCCBF1846584204F0A0
:10F2D0002BFB914904F030FC064603E0002601E0D8
:10F2E0004FF07E564FF0000903950024CDF80890AA
:10F2F00063000493894B33F9140004F015FB88492B
:10F3000004F066FB04F02AFD04F00EFB854904F0CE
:10F310005FFB804B824633F9140004F005FB7C4B05
:10F3200007461B889B077ED0014604F049FA7E4BB6
:10F33000804633F9140004F0F7FA0146404604F021
:10F340003FFA04F00BFD059B5B42984203DB059BF3
:10F350008342A8BF0346754A0499885E099A1B1A1E
:10F3600032F91400184404F0DFFA804604F00CF877
:10F3700070B16F4B40466F4914F8039004F0DCFB0A
:10F380000146484603F038F96A4904F021FB8046FB
:10F39000287F04F0C5FA684904F01AFB8346287AEE
:10F3A00004F0BEFA0146404604F012FB634904F043
:10F3B0000FFB04F0D3FC81460BF1004004F0CEFCBF
:10F3C000814505DB584604F0C9FC4845A8BF4846BE
:10F3D00004F0AAFADFF8889102900199404604F0FF
:10F3E000F7FA59F8241004F0EBF955494FEA840B69
:10F3F000804604F08BFC38B94046524904F0A4FC26
:10F4000020B1DFF8408101E0DFF8348149F80B805A
:10F41000A87C04F085FA0146404604F0D9FA4A492E
:10F4200004F0D6FA81463A4BB3F800B01BF0010F56
:10F4300040F09880394B049ADFF81C81D35E002B92
:10F44000B8BF5B42B3F5206F4FEA84030A9303DD34
:10F45000002348F824302AE03C49384604F0B8FA42
:10F46000039B0B90587804F05BFA0B9A0146104608
:10F4700004F062FB514604F0A1F9019904F0A8FAE6
:10F4800058F8241004F09CF93149804604F03EFC01
:10F4900038B940462F4904F057FC20B1DFF8B4805A
:10F4A00001E0DFF8AC802C4A0A9B42F80380039B02
:10F4B000D87A04F035FA284B53F8241004F088FA6F
:10F4C000264904F085FA1BF0020F80464CD03846DE
:10F4D000029904F073F90146304604F079FA0146C6
:10F4E000029804F06DF949460746404604F066F973
:10F4F0000146304604F06CFA0146484604F060F9D3
:10F50000804631E083F9223EC40F0020BD378635A6
:10F510008C110020AC1000200000E143E80F002017
:10F520000000A03ECDCC4C40E033002094280020C9
:10F5300088A50108000020410000A0406F12033C94
:10F540000000F0C10000F0410AD7A33D0000A04335
:10F55000000040C300004043542400200AD7233C4D
:10F560004C240020C846029F874B185D04F0DCF94C
:10F570000146504604F02CFA844904F029FA014669
:10F58000384604F01BF995F85120034642B1804BF0
:10F590000C2101FB04317F4B1B68F9F731F903465D
:10F5A0007D4F504657F824100A9304F007F901994B
:10F5B00004F0C2FA47F824A007F1080A5AF824B068
:10F5C0001037594604F0FAF80146079804F000FA9B
:10F5D0000146584604F0F4F883464AF82400385DA2
:10F5E00004F0A2F90146584604F0F2F96B4904F020
:10F5F000EFF907460A9B4146184604F0E1F8394600
:10F6000004F0DCF808F0B0F8654A049B0492D0528C
:10F610000A9BDFF8B0B1184604F0A0FB4BF82400B9
:10F62000404604F09BFBDFF8A0A1DFF8A0814AF878
:10F63000240007F1004004F091FB039B049A01337E
:10F6400048F82400039317460CB9012450E6089AA1
:10F65000544B9479B3F90430640028345C43524B22
:10F660006411B3F9040004F05FF94FF07A5104F02B
:10F67000AFF908F079F8201A04F056F9002CB8BF59
:10F680006442322C0646494C02DD0023A36025E08B
:10F69000069804F063FB20F0030004F045F90190A4
:10F6A000687B04F03DF90146304604F091F9019B76
:10F6B00081463F49184604F03FFA0146484604F0A7
:10F6C00087F904F04BFBA36818443A4B9842A8BF53
:10F6D0001846394B9842ACBFA060A360A3686FF096
:10F6E000FF005B13B3F5807FA8BF4FF4807398428F
:10F6F000B8BF184604F018F98146304604F02EFBD6
:10F70000EB785843801104F00FF92C4B04461B781A
:10F71000032B11D9B5F84E60B6F5FA7F0CD204F080
:10F720001DFB7342984203DBB0420346A8BF334639
:10F73000184604F0F9F8044695F8512032B1154BFB
:10F7400020461F491B68F9F75BF8044649462046E6
:10F7500004F036F804F002FB80B2B88000B204F086
:10F76000E3F808F001F8B880204604F0F7FACBF887
:10F770000800484604F0F2FA0023CAF80800C8F866
:10F7800008300DB0BDE8F08F60240020A69B443BFC
:10F79000AC210020D021002064240020F7CC923836
:10F7A00028220020AC100020E80F0020D4210020E7
:10F7B00000803B45FEFFFF0F020000F0E026002026
:10F7C000C4210020302200203C22002048220020BA
:10F7D0002DE9F04F89B00593BF4B0026B3F9029095
:10F7E000B3F90030B9F1000FB8BFC9F10009002B1F
:10F7F000B8BF5B429945B8BF99468046B246344689
:10F80000B9F5FA7F04910392A8BF4FF4FA790190F9
:10F8100000960296B14D2B88990754D0AE4B6100EB
:10F8200033F91420AE4B33F9143003EB4202039B3F
:10F830005B429A4203DB039B9342A8BF1346A94A4B
:10F840008F5E059ADB1B32F914001F1803F09CFD34
:10F8500090B1A54B384613F804A004F065F8A3490D
:10F8600004F06AF90146504602F0C6FE9F4904F0D2
:10F87000AFF804F073FA074698F8083064227B4327
:10F8800093FBF2F398F81C206FF0040A0AFB02FACB
:10F89000534504DB02EB820A9A45A8BF9A4642F21E
:10F8A0001072934B53F8240038449042A8BF10467E
:10F8B000904A9042B8BF104643F8240098F812309E
:10F8C0005843031302932D8805F00303012B38D00E
:10F8D000814B894933F91430A6000093019B51F8FC
:10F8E000247093F801E0854B33F9140080EAE0734B
:10F8F000A3EBE073B3F5206F16DC009A50235A4354
:10F9000092FBFEF3042290FBF2F0181A0744B7F5BD
:10F910007A5F7B4BA8BF4FF47A579F42ACBF41F848
:10F92000247041F8243002E0002341F824308B5940
:10F930007D2693FBF6F6019BDB7A7343402693FB0F
:10F94000F6F6AA0712D5009A09FB06F509FB02F79D
:10F950000298C9F5FA7303FB0A7703FB00534FF4CF
:10F96000FA7297FBF2F193FBF2F505E0EB0755BF56
:10F97000354651460099029D604B042733F91430F7
:10F98000604A93FBF7F3A25C6FF04F07534393FB7E
:10F99000F7F398F851204FEA440BCF187AB1384664
:10F9A000069203F0C1FF584B0C2101FB0431574B69
:10F9B000069A1B68F8F724FF04F0D0F907464F4B6E
:10F9C000534A3BF803003BF9021003B25B1A0421CF
:10F9D00093FBF1F102F1040E5EF824302BF80200E3
:10F9E0000C3252F8240042F8243098F85020184481
:10F9F0004FEA840C08444EF824108AB1CDF81CC09C
:10FA0000069203F091FF434B0C2101FB04313F4B65
:10FA1000069A1B68F8F7F4FE04F0A0F9DDF81CC0A4
:10FA20003D4BDFF810E11B5D7A195843202390FB12
:10FA3000F3F3D21A2BF80E20384A5B424CF802300E
:10FA4000019B3748374901334CF801504CF800709E
:10FA5000019375460CB90124DCE61F4B0427B3F96A
:10FA60000440049B244E9B79D6F808E00F335B00DA
:10FA70006343224C5B11B4F90440002B94FBF7F76D
:10FA8000A3EB0707B8BF5B42322B98F80D400BDCA5
:10FA900004FB07E4244BA342A8BF2346234CA34204
:10FAA000ACBFB360B46001E00023B36098F80340DA
:10FAB00004FB07F31E4C9B112478032C3DD9B8F8A6
:10FAC0004E40B4F5FA7F38D26742BB4234DBA342E2
:10FAD000A8BF234631E000BFAC1000208C110020ED
:10FAE000E03300209428002088A501080000204170
:10FAF00078240020F0D8FFFFD4210020E80F002058
:10FB000080C1FFFF60240020AC210020D021002014
:10FB10008024002004220020742400204822002099
:10FB2000302200203C220020FEFFFF0F020000F0E8
:10FB3000E0260020282200203B46B4686FF0FF0634
:10FB400044F34F34B4F5807FA8BF4FF48074B442BF
:10FB5000B8BF344683601E190023AE808C6093606A
:10FB600009B0BDE8F08F2DE9F04F87B00393B54B96
:10FB700081461D88029105F00205ADB2019295B152
:10FB8000B14BB3F90250B3F90030002DB8BF6D424C
:10FB9000002BB8BF5B429D42B8BF1D46B5F5007F44
:10FBA000A8BF4FF40075CB460026A74BA74933F9F1
:10FBB0001620A74B4FEA460A33F91630520083EA63
:10FBC000E374A4EBE374B4F5206F4FEA860851F8B0
:10FBD000260011DC042493FBF4F3D31A0344B3F599
:10FBE0007A5F9C48A8BF4FF47A538342ACBF41F878
:10FBF000263041F8260002E0002341F8263051F873
:10FC000008709BF80B30FF119BF801405F438D4B50
:10FC100054431B88BF119B074FEAA41456D08E4B48
:10FC20003AF903301A44019B5B429A4203DB019B81
:10FC30009342A8BF1346894A3AF902209B1A039AB5
:10FC400032F916201A44049203F09EFB049A98B1EC
:10FC5000834B10469B5D049303F066FE814903F0DD
:10FC60006BFF049B0146184602F0C6FC7D4903F079
:10FC7000AFFE04F073F8024642F210707A4958F869
:10FC8000013013448342A8BF034678488342B8BF7B
:10FC9000034648F8013099F8081099F81C004A43C7
:10FCA00000EB8000D21141428A4203DB8242A8BFAE
:10FCB0000246114699F81220641A53431B13FF1A87
:10FCC0006F436C4303EB672701EB6424604B042212
:10FCD0003AF9033093FBF2F2654B9B5D534399F87D
:10FCE0005120A4EBA3147AB12046049203F01CFE29
:10FCF000604B0C2101FB06315F4B049A1B68F8F73F
:10FD00007FFD04F02BF8044651495C4B3AF80100A2
:10FD10003AF903E002B2CEEB02024FF0040E92FB7E
:10FD2000FEF22AF803009E440C3358F80EC058F82F
:10FD3000030048F80E206044104499F8502048F819
:10FD400003C08C4682B10591049203F0EDFD4C4B4B
:10FD50000C2101FB0631484B049A1B68F8F750FD53
:10FD600003F0FCFFDDF814C0464BDFF834E19B5D87
:10FD7000E21943435B11D21A2AF80E204248434944
:10FD8000434A5B4248F8004048F8017048F80230A6
:10FD90000BF1010B74460EB9012606E72A4B042726
:10FDA000B3F90450029B294E9B79D6F808E00F3333
:10FDB0005B006B43BCF904505B1195FBF7F7002B1C
:10FDC000A3EB0707B8BF5B42322B99F80D500BDC51
:10FDD00005FB07E52F4BAB42A8BF2B462E4DAB4290
:10FDE000ACBFB360B56001E00023B36099F8035085
:10FDF00005FB07F3294D9B112D78032D0CD9B9F87C
:10FE00004E50B5F5FA7F07D26F42BB4203DBAB42DF
:10FE1000A8BF2B4600E03B46B5686FF0FF0645F3F0
:10FE20004F35B5F5807FA8BF4FF48075B542B8BF98
:10FE3000354683605E190023A6808D60936007B00D
:10FE4000BDE8F08F8C110020AC100020D4210020E0
:10FE5000E80F002080C1FFFFE0330020942800203D
:10FE600088A501080000204178240020F0D8FFFF79
:10FE700060240020AC210020D02100209424002008
:10FE80000422002074240020302200203C22002084
:10FE900048220020FEFFFF0F020000F0E0260020B5
:10FEA000282200202DE9F04F89B00593A84B0026A9
:10FEB000B3F90280B3F90030B8F1000FB8BFC8F150
:10FEC0000008002BB8BF5B429845B8BF98468246F1
:10FED000B146B3463446B8F5FA7F0492A8BF4FF452
:10FEE000FA78029003969B4D2B88990757D0022CE5
:10FEF00055D0974B610033F91420974B33F91430E8
:10FF000003EB4202049B5B429A4203DB049B934255
:10FF1000A8BF1346914A8F5E059ADB1B32F9140085
:10FF20001F1803F031FA90B18D4B384613F804B026
:10FF300003F0FAFC8B4903F0FFFD0146584602F03E
:10FF40005BFB884903F044FD03F008FF07469AF87D
:10FF5000083064227B4393FBF2F39AF81C206FF085
:10FF6000040101FB02FB5B4505DB02EB82029342CD
:10FF7000A8BF13469B4642F210727B4B53F82400F5
:10FF800038449042A8BF1046784A9042B8BF104605
:10FF900043F824009AF81230584303130393298836
:10FFA00001F00303012B01D1022C3DD1684B704DB0
:10FFB00033F91490029BA00093F801E06D4B55F8C3
:10FFC000247033F9146086EAE673A3EBE673B3F5A5
:10FFD000206F1CDC022C14D0502303FB09F292FB8F
:10FFE000FEF3042296FBF2F69E1B3744B7F57A5FC8
:10FFF000614BA8BF4FF47A579F42ACBF2F502B5094
:020000040801F1
:1000000007E089EAE973A3EBE973642BE4DD0023DD
:100010002B50574B7D26C35893FBF6F6029BDB7A99
:100020007343402693FBF6F68A0713D5022C11D0B2
:1000300008FB06F508FB09F70398C8F5FA7303FBFC
:100040000B7703FB00534FF4FA7297FBF2F193FB2B
:10005000F2F508E0CB0704D5022C02D0039D5946E7
:1000600001E03546494663000193424B042733F9CA
:100070001430424A93FBF7F3A25C6FF04F075343EF
:1000800093FBF7F39AF85120CF187AB138460692CD
:1000900003F04AFC3A4B0C2101FB0431394B069A20
:1000A0001B68F8F7ADFB03F059FE0746314B019A88
:1000B0000198D15A344B0AB2C05E4FEA840C121A2E
:1000C000042092FBF0F20198C15203F108011433AD
:1000D00051F824E053F8240041F8242070441044DF
:1000E0009AF8502043F824E08AB1CDF81CC006925B
:1000F00003F01AFC254B0C2101FB0431214B069A1D
:100100001B68F8F77DFB03F029FEDDF81CC0204BCF
:10011000204A1B5D01995843202390FBF3F07B1983
:100120001B1A8B521C4B40424CF803701B4B013482
:100130004CF803501A4B032C4CF80300029B03F1BC
:10014000010302937FF4CFAE09B0BDE8F08F00BF8A
:10015000AC1000208C110020E033002094280020F7
:1001600088A501080000204178240020F0D8FFFF76
:10017000D4210020E80F002080C1FFFF6024002070
:10018000AC210020D0210020A8240020042200203F
:100190007424002028220020302200203C2200204D
:1001A00048220020084BDA68D10709D4DA685207E0
:1001B00008D4DB6813F0100F14BF0320042070472D
:1001C00001207047022070470020024003788B42D4
:1001D00086BF024B33F8110000207047C82400206E
:1001E0000022134670B5234914180C44247E83EA78
:1001F0000423082413F4004F4FEA430318BF83F489
:10020000815304F1FF3418BF83F0010314F0FF049D
:100210009BB2EFD10132192AE5D100F1190200F1A8
:100220001A050A440D44167E2A7E02EB062292B27B
:100230009A421ED10F4B93F83950E2B2AA4215D21E
:10024000431C03EB4203DBB2CA1801330B44127E9A
:100250001B7E03EB02239BB24FF4AF6253431B138D
:1002600003F5487321F814300134E6E7012381F8DF
:100270003A3070BDC824002003788B420BD9074B5D
:10028000890093F83B201944C86B02B1400800F57F
:10029000777080B270470020704700BFC8240020EC
:1002A00007299DBF034B03EB8101B1F86C000020CF
:1002B000704700BFC824002070B50546FCF758FF02
:1002C000314CD4F88C30C4F88C00C31AB3F5FA5F03
:1002D000C4F8903082BF002384F8943084F89530BD
:1002E00094F894302BB9A12D02BF274A012182F83E
:1002F000951094F89510244A29B1D118EDB2013324
:100300000D7682F8943094F8945094F89630AB427D
:1003100039D11D4B93F89730052B02D0062B03D013
:100320002CE00020FFF75CFF637E1E2B26D100200F
:100330000246C1B26B1E994219DA21440B7E082194
:10034000DBB283EA0206F60744BF83F01803C3F367
:10035000460301F1FF3154BF5B0843F0800311F005
:10036000FF01C2F34702ECD101301A46E1E7234412
:100370001B7E9A4202D10320FFF732FF002384F84C
:10038000953084F8943070BDC824002010B5044620
:10039000FCF7EEFE41F288310E4BE4B2D3F8982020
:1003A000C3F89800821A8A42C3F89C2084BF0022B6
:1003B00083F8A02093F8A02006490F2A134418BF01
:1003C000013283F8A14012BF81F8A020012381F8F7
:1003D000B13010BDC824002010B50446FCF7C8FE9B
:1003E00041F288310E4BD3F8B420C3F8B400821A1E
:1003F0008A42C3F8B82084BF002283F8BC2093F857
:10040000BC200749142A134418BF013283F8BD40A9
:1004100012BF81F8BC20012381F8D23010BD00BF8B
:10042000C82400204FF6FE730268134003600023C7
:10043000036043608360C360284B984201D1284A1F
:1004400027E0284B984201D1254A2AE0264B9842C2
:1004500001D1234A2DE0254B984201D1204A30E0BA
:10046000234B984201D11E4A33E0224B984204D1DB
:100470001B4A536843F470032EE01F4B984204D18B
:10048000174A536843F0706326E01C4B984204D12E
:100490001B4A536843F00F031EE01A4B984204D1E5
:1004A000174A536843F0F00316E0174B984204D103
:1004B000134A536843F470630EE0144B984204D11E
:1004C0000F4A536843F4704306E0114B984204D13D
:1004D0000B4A536843F4702353607047080002408E
:1004E000000002401C000240300002404400024074
:1004F000580002406C0002408000024008040240A4
:10050000000402401C040240300402404404024043
:10051000580402401F4A10B5536803F00C03042B23
:1005200003D0082B04D01C4B14E01C4B1B6811E0BB
:1005300053685168C3F38343C90303F1020301D431
:10054000174906E0516811F4003F1449096818BFC3
:1005500049084B43036053681249C3F30313CC5C4F
:100560000368E34043605468C4F302240C5D23FA3B
:1005700004F484605468C4F3C2240C5DE340C36097
:100580005268C2F381320A44127CB3FBF2F3036176
:1005900010BD00BF0010024000127A003C00002095
:1005A00000093D0088AC010810B50446FFF7FAFDCC
:1005B000012806D11CB1FFF7F5FD013CF8E7052045
:1005C00010BD002C08BF052010BD0A88F0B54B886F
:1005D0008E88B1F808E0CC88002A3AD1028C43F02A
:1005E000010322F001021204120C0284058B078C15
:1005F000ADB225F0F30545EA0E1189B241EA0602D3
:100600007A49BFB2884212D001F5006188420ED00B
:10061000B0F1804F0BD0A1F59831884207D001F599
:100620008061884203D001F58061884202D127F0C1
:10063000020701E027F00A071F4302830784038BA8
:1006400023F00C031B041B0C0383038B9BB21C4382
:1006500044E0042A44D1028C22F010021204120C4D
:100660000284018B058C21F440721205120D42EABE
:100670000E325E4992B242EA06228842ADB292B28E
:1006800012D001F5006188420ED0B0F1804F0BD03E
:10069000A1F59831884207D001F58061884203D0E6
:1006A00001F58061884207D125F0200141EA03135A
:1006B0009BB243F0100304E025F0A00143F01003C7
:1006C0000B4302830384038B23F440631B041B0C42
:1006D0000383038B9BB243EA0424A4B20483F0BDDA
:1006E000082A028C3ED122F480721204120C028479
:1006F000828B3E4D92B222F0F307018C47EA0E1234
:1007000092B2A84289B242EA060212D005F500650B
:10071000A8420ED0B0F1804F0BD0A5F59835A84275
:1007200007D005F58065A84203D005F58065A8428D
:1007300007D121F4007141EA03239BB243F4807393
:1007400004E021F4206143F480730B43828303842B
:10075000838B23F00C031B041B0C8383838B9BB2C2
:100760001C4341E022F480521204120C0284858B57
:10077000018C25F440752D052D0D45EA062545EA29
:100780000E321A4D89B2A84292B212D005F5006518
:10079000A8420ED0B0F1804F0BD0A5F59835A842F5
:1007A00007D005F58065A84203D005F58065A8420D
:1007B00007D121F4005141EA03339BB243F4805343
:1007C00005E047F6FF5543F480530D402B438283E9
:1007D0000384838B23F440631B041B0C8383838B70
:1007E0009BB243EA0424A4B28483F0BD002C0140F0
:1007F000016830B5CD43154B1C682C401C605A680D
:100800002A405A60027902F1804202F5823214686D
:100810002143116002689C68D5432C409C60D968D4
:100820002940D9604179102909BF996801F18043B5
:100830001143996015BF03F58233D96819680A43DB
:1008400016BF0A43DA601A6030BD00BF00040140E1
:10085000054B1A685B69034004D0104214BF0120A5
:10086000002070471846704700040140CA78F0B570
:10087000D40648BF8C780D8802F00F0348BF23438D
:1008800015F0FF0F1DD0016800240126A64006EADE
:100890000507B74211D14FEA840E0F2606FA0EF66D
:1008A00021EA0601282A03FA0EF641EA060101D1DF
:1008B000476102E0482A08BF07610134082CE4D1EF
:1008C0000160FF2D1FD94168002404F108070126AB
:1008D000BE4006EA0507B74211D14FEA840E0F2643
:1008E00006FA0EF621EA0601282A03FA0EF641EA74
:1008F000060101D1476102E0482A08BF07610134BF
:10090000082CE2D14160F0BD0F4B1A6842F00102A1
:100910001A6059680D4A0A405A601A6822F08472B7
:1009200022F480321A601A6822F480221A605A680F
:1009300022F4FE025A604FF41F029A60044B4FF0FB
:1009400000629A60704700BF001002400000FFF88C
:1009500000ED00E02DE9F8435B4C0368013AC4F870
:10096000D43083880D46A4F8D830072A42D8DFE86F
:1009700002F0040A101822292F35B4F8D4300B8065
:10098000B4F8D63013E0B4F8D6300B80B4F8D430D5
:1009900005E0B4F8D4305B420B80B4F8D6305B424B
:1009A00005E0B4F8D6305B420B80B4F8D4306B80ED
:1009B000B4F8D8301DE0B4F8D4305B420B80B4F802
:1009C000D63012E0B4F8D6300B80B4F8D4300CE056
:1009D000B4F8D4300B80B4F8D63005E0B4F8D63093
:1009E0005B420B80B4F8D4305B426B80B4F8D830F3
:1009F0005B42AB80354B1B79002B62D1B5F900000F
:100A000002F092FF8046B5F9020002F08DFF074622
:100A1000B5F9040002F088FFD4F8DC100646404621
:100A200002F0D6FFD4F8E8108146384602F0D0FF35
:100A30000146484602F0C4FED4F8F4108146304620
:100A400002F0C6FF0146484602F0BAFE06F08CFEF0
:100A5000D4F8E0102880404602F0BAFFD4F8EC1039
:100A60008146384602F0B4FF0146484602F0A8FE2F
:100A7000D4F8F8108146304602F0AAFF01464846F5
:100A800002F09EFE06F070FED4F8E4106880404646
:100A900002F09EFFD4F8F0108046384602F098FF2E
:100AA0000146404602F08CFED4F8FC100746304662
:100AB00002F08EFF0146384602F082FE06F054FE38
:100AC000A880BDE8F88300BFC82400203C000020B7
:100AD00038B50F4B1B689C890E4B186880F31000CB
:100AE000201A02F021FF0C4902F072FF0546204651
:100AF00002F01AFF0146284603F01EF803F02EF913
:100B00006428A8BF642020EAE070C0B238BD00BFEE
:100B1000B4100020C41000200000C84244F6FB714D
:100B2000084B1A68137803EB431300FB0313507848
:100B3000C0EB0030B3FBF0F39078B3FBF0F080B281
:100B4000704700BFB410002008B50A480A2290F888
:100B5000013100EB4303B3F8101100F5907089B236
:100B600020F8081CFCF700FC80B2FFF7D7FF024B0F
:100B7000188008BDC8240020B810002070B51B4B99
:100B8000002093F8A911B3F8AA5103EB410494F89B
:100B9000AF6194F8B02183F8A80142EA0622954299
:100BA0001A4622D193F8AD31012B02D0812B02D00D
:100BB00070BD184600E00320102984BF102382F87E
:100BC000A93192F8A9410A4A0023D9B2A14202F1FF
:100BD00002020AD212F8025C12F8011C41EA052155
:100BE000044D25F813100133EFE770BDC824002031
:100BF000772600209A26002007B5064B0649009369
:100C0000064B074A01930748074BF8F739F803B03A
:100C10005DF804FB6CBC01085DC3010841BC010820
:100C200057C301085CCD010860BC010808B5037812
:100C300033B90C4B0C481978BDE80840F8F720B8D8
:100C400006F01EFC02280CD8064B0C221870074B2D
:100C500002FB0030064B0230186001F0A9F805488D
:100C6000E5E708BDC02600207CCD0108A4300020A7
:100C70002C1000201CC0010808B503783BB90B4BB1
:100C80000B4893F8A817BDE80840F7F7F9BF06F03E
:100C9000F7FB022808D8054B83F8A807F8F7B6F940
:100CA000F8F756FA0348E8E708BD00BFFC28002023
:100CB00080CD01081CC0010838B5037803BB214B67
:100CC0001B6801330F2B07D81F490C2202FB0312AC
:100CD00095681C462DBB00E01C4601340F2C01DD3D
:100CE000002400E005D818490C2202FB0412956884
:100CF000BDB99C42F1D11548BDE83840F7F7C0BFF7
:100D000006F0BEFB0F28044605D80F4A0C2303FB50
:100D100000239D682DB92146BDE838400C48F7F7FF
:100D2000AFBF084B1C60FCF76FFA21462A46094802
:100D3000F7F7A6FF0C235C43034B185DBDE8384072
:100D4000FCF77ABA440000209CAC01088DCD010864
:100D5000A3CD0108BBCD010873B5037813B9F6F72D
:100D60000DF93FE001AA204906F0EBFB0024024602
:100D7000264625469AB134B1012C08D1104606F01A
:100D80007FFB064603E0104606F07AFB054601AA03
:100D90000020154906F0D5FB01340246EAE70B2D89
:100DA00003D9124812490C230CE0022C11D1A6F5EC
:100DB0007A73B3F57A7F08D90C480E494FF47A72EA
:100DC0004FF4FA63F7F75CFF0CE00B4B03EB4503C2
:100DD0005E80094B094803EB45032946B3F902201D
:100DE000F7F74EFF02B070BD6FC6010835C20108AB
:100DF00054C201081BCA0108C0260020D2CD010838
:100E000038B50D4C05462368834206D1F6F77EFCC3
:100E1000204600214C2206F09AFAE36CAB4209D13D
:100E20002846F6F773FCBDE83840044800214C2200
:100E300006F08DBA38BD00BF8C170020D8170020EF
:100E4000034B1A68D379591C1344D171187A70472F
:100E50006C11002010B5FFF7F3FF84B2FFF7F0FF2D
:100E600004EB002080B210BD10B5FFF7F3FF04467D
:100E7000FFF7F0FF04EB004010BD10B50446054B32
:100E800021461868FCF76DFA034B1B68987960409F
:100E9000987110BD701100206C11002038B5044607
:100EA0000D462420FFF7E9FF4D20FFF7E6FF002C59
:100EB000084C14BF21203E20FFF7DFFF23680022EB
:100EC00028469A71FFF7D9FF236893F84900BDE8D7
:100ED0003840D2E76C11002001460020DEE710B553
:100EE0000446C0B2FFF7C9FF200ABDE81040C4E7BE
:100EF00010B5044680B2FFF7F2FF200CBDE81040A9
:100F0000EDE737B582888368044610060D4641BF79
:100F100029494FF4CC7091F8A81700FB0133D10593
:100F200042BF26490C20097802F03F0248BF00FB6F
:100F30000133042A12D006D8012A0DD0022A2FD15B
:100F400093F900102DE0102A0AD0202A0AD0082A8E
:100F500026D1B3F9001024E0197822E0198820E0A6
:100F600019681EE069461868F7F710FD0146144835
:100F7000F7F786FEF5B1E06802F0D6FC6946F7F7B0
:100F800005FD01460F48F7F77BFE206902F0CCFC17
:100F90006946F7F7FBFC01460A48F7F771FE09E0DE
:100FA00000210948F7F76CFE25B10848E16822697D
:100FB000F7F766FE03B030BDFC280020C0260020F5
:100FC000F7C40108F0C4010831C40108E1CD0108EB
:100FD000024B0146D869FCF7C4B900BFC026002007
:100FE00010B5441E14F8011F21B1034BD869FCF75A
:100FF000B8F9F7E710BD00BFC02600202DE9F04F7B
:10100000037885B01BB96C48FFF7EAFFD0E006F023
:1010100037FA05460628694C99BF69482946694848
:101020000621F7F72DFE94F820200023D9B2914233
:1010300007D26549002051F8231001330968088060
:10104000F4E7013DEDB272B6604F6DB207EBC5013A
:1010500049684FF001085E4E57F8359008FA01FADA
:101060004FF480624FF400731FFA8AF172614FF0FF
:10107000480B73613046C9F8141003A9ADF80C2071
:1010800001938DF80EB08DF80F80FDF786FD019B62
:101090003046ADF80C3003A910238DF80E30ADB2F8
:1010A0008DF80F80FDF779FD484603A9ADF80CA037
:1010B0008DF80EB08DF80F80FDF76FFDE9007B18FD
:1010C0005A6857F83530D00803EB800E53F82030BB
:1010D00002F00702A3659200E36523660F239340A5
:1010E000DB43E06DC4F854E01840E065A06D0340B8
:1010F000A365E06D082393400343E365A06D08FA00
:1011000002F303433846A365B3685F05FCD4676DFB
:10111000A36D08223B604FF40073C9F814A07361FB
:101120002C4B1A6110225A6140F6B833B26852054E
:1011300013D4013BFAD14FF40073ADF80C301823EF
:101140008DF80E302248012303A98DF80F30FDF7EA
:1011500024FD236E3B6062B62AE0C9F810A0E36D5F
:1011600050F835E03B604318D3F804C0DEF80C209B
:10117000012303FA0CF31343CEF80C30154B102265
:101180001A61B268124B5205C2D5D9F808204FF443
:10119000007C1AEA020F0F4A4FF0080E15BFC3F881
:1011A00010C0C3F814C0C2F810E0C2F814E0E8E7B9
:1011B00005B0BDE8F08F00BFE8CD0108C0260020D3
:1011C0002FCE01085BCE0108E42600202CCD0108BB
:1011D00000080140000C0140F7B52949294B087867
:1011E000294D1C68294B05EB80001A88D0F8C010E7
:1011F000274B28481B7800914FF47A71B4FBF1F12A
:10120000F7F73EFD244B25481968254B0026B1FB16
:10121000F3F1F7F735FD234B1F68F3B205EB8302BB
:10122000D2F8D010E1B101249C403C4216D02207F4
:1012300014D01D4A0B20D25C00FB0323124A1B482A
:1012400002EB8303D3F8F020F7F71AFD022C05D147
:10125000174B197A11B11748F7F712FD0136DCE781
:101260001548FFF7BDFE154B15481A88154B92B26D
:10127000198840F2D47303B0BDE8F040F7F700BD21
:1012800018110020C02800209CAC0108B8100020D4
:101290004D00002086CE010858000020C9CE01086C
:1012A00040420F00C810002050000020D9CE010895
:1012B00024180020E1CE010829CF0108C60F002024
:1012C000E5CE0108C40F00202DE9F041002480463E
:1012D00025460F4E4146A759384606F0B9F858B191
:1012E00039460C48F7F7CCFC30190021FFF709FE0E
:1012F0000948FFF775FE01351434B4F5486FE8D19D
:101300001DB9BDE8F04105486AE6BDE8F08100BFBF
:101310003CAE01087FC5010829CF0108C6C20108FB
:101320002DE9F74F824606F056F8054628B1012808
:1013300018D19AF800302A2B14D15848FFF750FEE4
:101340000024574E5748A159F7F79AFC30192946FF
:10135000FFF7D7FD14345448FFF742FEB4F5486F49
:10136000EFD198E050463D2106F027F8002800F024
:101370008D8003461D4613F8012D202AFAD0441C07
:10138000204606F07DF881462046F7F769FA0746C1
:10139000CAEB05054FF0000B142404FB0BF4DFF837
:1013A000208108F5D073E6580193304606F013F813
:1013B0008446314662465046CDF800C006F014F827
:1013C000DDF800C0019B002856D1EAB2624553D136
:1013D0001D194444D4F8AC0102F0A6FA014638467F
:1013E00002F0A8FC002845D0D4F8B00102F09CFA25
:1013F0000146384602F094FC00283BD0B4F8A431F2
:101400009A0658BF4F46142202FB0B881C0648BFA1
:101410002648D8F8A82142BF90F8A8074FF4CC740A
:1014200004FB0022D80542BF21480C24007803F0B9
:101430003F0348BF04FB0022042B39460BD004D8DD
:10144000013B012B0CD817700AE0102B05D0202B84
:1014500005D0082B04D1118002E0176000E017606E
:1014600031461448F7F70CFC2846002103B0BDE8CC
:10147000F04F46E5104805E00BF1010BBBF1A00F62
:101480008AD10E4803B0BDE8F04FA9E5504603B03D
:10149000BDE8F04F18E703B0BDE8F08F17CF0108A3
:1014A0003CAE01087FC5010829CF0108FC280020B7
:1014B000C02600202CCF010837CF0108C6C2010882
:1014C0009CAC010808B50748FFF78AFD064BD869B0
:1014D000F6F7F8F8FCF7C4F8F7F76EFD034A044B8B
:1014E000DA6008BD57CF0108C02600200400FA05C5
:1014F00000ED00E008B50548FFF772FD00F09EFC26
:10150000F7F784FDBDE80840DCE700BF63CF0108C2
:1015100008B50448FFF764FDF7F778FDBDE808401B
:10152000D0E700BF79CF010810B54B88DC0641BF7A
:101530002F4B14791B6853F8244044BF2D4B43F8BC
:1015400020404B889B0641BF294B54791B6853F8B8
:10155000244044BF274B43F820404B881C070ED53E
:10156000254B0C781B78B3EB141FA1BF204BD4780C
:101570001B6853F82440A4BF1E4B43F820404B88FF
:101580009B070ED51D4B0C781B78B3EB141FDFBFE8
:10159000174B54781B6853F82440DCBF154B43F8B5
:1015A00020404B88DC070FD5154C0B78247803F0CE
:1015B0000F03A342DFBF0E4B14781B6853F824407F
:1015C000DCBF0C4B43F820404B885B070FD50B78F2
:1015D0000C4903F00F0309788B42A1BF044B9278AA
:1015E0001B6853F82220A4BF024B43F8202010BDF3
:1015F00028240020CA080020871700208517002013
:101600008417002086170020254A0023F0B51568AE
:101610001C461A462348244903700B702E197688FD
:101620004EB92F5D3FB9037000230A704B700778E5
:101630001C461A460CE0360548BF013204F104048A
:1016400003F1010348BFD2B2802CDBB2E6D1EAE756
:10165000E0B2B8420CD215F82400013406099E42CB
:1016600000F00F00A8BF731C9042A8BF421CEFE718
:101670008A704B70C2F3470102F001020A444C1E0B
:101680000A490B480A70C3F3470203F001031344ED
:1016900004700849501E084A08701370F0BD00BF5E
:1016A000901100207C1700203C2700208617002086
:1016B000841700208717002085170020924B2DE902
:1016C000F04FDA68914D1A612A6891B0DA60904A59
:1016D0000295136843F0200313608E4B1A78012A99
:1016E0000CBF002201221A708B4B1A78910740F12F
:1016F0004D838A490978042940F24883884909784A
:1017000001F0040101F0FF0011B922F001021A708A
:101710001B78DB0702D408B1FBF730F98149CA789E
:10172000531C052293FBF2F202EB82029A1A7E4BC3
:10173000CA701F7892000023DFF81082DFF8109241
:1017400058F82310794C91FBF9FE04F1080040F899
:1017500023E0774844F8231000FB0E1142F210708A
:1017600091FBF0F004F1100680B226F813004FF060
:10177000140C04F114060CFB036C04F13C0A5AF837
:1017800023605CF802504CF80210761B31440526A9
:101790004AF8231091FBF6F109FB0E114434012F96
:1017A00044F823104FEA830B444605D10238B0F5C4
:1017B000797F98BF4BF808100BB90123BCE7594E4D
:1017C000029BB2461868336DC01A02F0A9F8594955
:1017D00002F0B2F9029B4FF07E511B680746336559
:1017E00002F094FA08B94FF07E574B4BCAF8547088
:1017F0001B78514E13F00103504D12D00DAA0092E8
:101800004F4B0EAA01920CCB94E80300FAF7CCFFE1
:101810000D9A6421B2FBF1F20E9B328093FBF1F33F
:1018200000E033802B809AF858303E4D002B35D0A5
:10183000696D4FF07E5002F07FF90746EB6D20682E
:10184000C01A02F071F8394602F0C2F802F086FAC6
:101850002B6E86B2606836B2C01A02F065F8394B5A
:10186000196802F0B5F8394602F0B2F802F076FADB
:10187000B5F9662000B28118B5F964200220B318CA
:1018800091FBF0F193FBF0F389B29BB2A5F86A10DB
:10189000A5F86830A5F86610A5F8643001238AF829
:1018A0005830294B61681B88206803F030031D4EB7
:1018B000264DCAF86010CAF85C00002B00F0668262
:1018C00006F17403009306F178030193F26E336F0F
:1018D000FAF76AFF6B68306FC01A02F025F8194BEF
:1018E000196802F075F802F039FAF36E2A68C6F842
:1018F00080009B1AF3670C4B1B78012B2AD0022B1C
:1019000000F0E68042E200BF30020020C028002044
:10191000C810002032100020CC100020D21000206F
:10192000E53300203C270020380F0020402700200E
:10193000806967FF00007A444611002048110020AA
:1019400034100020480000208C110020D41000200A
:1019500080969800D6F88430D6F8A0400293D6F846
:10196000943004F100400393D6F89830776D0593D6
:1019700002F0F4F98146204602F0F0F9D6F89C30E6
:10198000BB4C0493BB4B06901B684FF0000B0793B6
:10199000B94E4FEA4B0356F82B80A6F1140240468D
:1019A00032F81B50089301F0BFFF029902F010F8C3
:1019B00002F0D4F9401B1FFA80FA283626F81BA043
:1019C0000FFA8AFA504601F0AFFF039902F000F8CF
:1019D00002F0C4F986B20AEB080001F0A5FF0599F0
:1019E00001F0F6FF394601F0F3FF216801F0E8FE4F
:1019F00002F0B4F9484504DB069B9842A8BF18469C
:101A000000E0484601F090FF206002F0A7F9079B34
:101A1000304486B2987801F083FF984901F0D8FFEE
:101A200001464FF07E5002F087F8394601F0C8FEBB
:101A30000146384602F080F809906068D4F808A0A2
:101A4000C0EB080001F070FF394602F075F851460E
:101A500001F0B4FE099A0146104601F0B9FF0146B3
:101A6000504601F0ADFE3135ADB2622D0146206128
:101A7000C4F80480A0600ED9049801F0A9FF02F018
:101A80006DF97F4AB0F5FA6FA8BF4FF4FA60904243
:101A9000B8BF104600E0002040F6B832064436B227
:101AA0009642A8BF1646774A089B9642B8BF16468C
:101AB000754A54F8140B9E52142202FB0BF2734920
:101AC0005050BBF1000F40F061814FF0010B5FE718
:101AD000684BB6F8A8401F68736F3D8902935B0896
:101AE0009D4228BF1D4623B29D4202DC1FFA85F9A4
:101AF0000AE06749706D01F06BFF02F02FF9204496
:101B00001FFA80F9A6F8A890DAF87860DAF8AC4005
:101B1000341B2046FAF78AFE41F293130028D8BFFF
:101B200040429842CCBF0020012078B3204601F00B
:101B3000FBFE584901F04CFFF7F7D1F80446029834
:101B400001F0EEFE0146204601F042FF02F006F9E8
:101B500040F6B83380B2AAF8B00000B29842A8BFED
:101B60001846484B9842ACBF3018F01848F6A043CE
:101B7000984203DDA0F50C40A03804E00028BCBF6B
:101B800000F50C40A030CAF8B40001E0CAF8B46017
:101B9000DAF8B4300026C3F50C502830039301F076
:101BA000C3FE3C4901F014FF0446F7F70BF90F9010
:101BB0002046F7F794F8DAF8B830DAF8C44005931D
:101BC000DAF8BC300E9004F10040089302F0C6F839
:101BD0000490204602F0C2F8DAF8C030DAF85480F7
:101BE0002A4C09900793730048460A9301F09CFE23
:101BF0000EAB53F8261001F0EBFEDFF8A0A005466F
